:020000040804EE
:100000000000082495780608E178060841B3050841
:1000100047B305084DB3050853B3050800000000B9
:100020000000000000000000000000009D680408BF
:10003000E1780608000000003769040847690408F1
:10004000E1780608E1780608E1780608E178060814
:10005000E1780608E1780608E1780608E178060804
:10006000E1780608E1780608E1780608E1780608F4
:10007000E1780608E1780608E1780608E1780608E4
:10008000E1780608E1780608E1780608998706080D
:10009000A9870608A5870608B5870608E178060837
:1000A000E1780608E1780608E1780608E1780608B4
:1000B000E1780608E1780608E1780608E1780608A4
:1000C000E1780608E1780608E1780608E178060894
:1000D000E1780608E1780608E1780608E178060884
:1000E000E1780608E178060800000000E1780608DB
:1000F000E1780608E1780608E1780608E178060864
:10010000E17806089D750608E1780608E17806089A
:10011000E1780608E1780608E1780608E178060843
:10012000E1780608E1780608E1780608E178060833
:10013000E17806088B980408E1780608E17806085B
:10014000E1780608E17806080000000000000000E1
:10015000E1780608E1780608E1780608E178060803
:10016000E1780608E1780608E1780608E1780608F3
:10017000E1780608E1780608E1780608000000004A
:10018000E1780608E1780608E1780608E1780608D3
:10019000E1780608E1780608E1780608E1780608C3
:1001A000E1780608E1780608E1780608E1780608B3
:1001B000E1780608E1780608E1780608E1780608A3
:1001C000E1780608E1780608E1780608E178060893
:1001D000E1780608E1780608E1780608E178060883
:1001E000E1780608E1780608E1780608E178060873
:1001F000E1780608E1780608E1780608E178060863
:10020000E1780608E1780608E1780608E178060852
:10021000E1780608E1780608E1780608E178060842
:10022000E1780608E1780608E1780608E178060832
:10023000E178060891780608E1780608E178060872
:10024000E1780608E1780608E1780608E178060812
:10025000E1780608E1780608E1780608E178060802
:10026000E1780608E1780608E1780608E1780608F2
:10027000E1780608E1780608E1780608E1780608E2
:10028000E1780608E1780608E17806080000000039
:10029000E1780608E178060810B5054C237833B9F3
:1002A000044B13B10448AFF300800123237010BD49
:1002B000E018002400000000D4D5070808B5034B5F
:1002C0001BB103490348AFF3008008BD00000000E4
:1002D000E4180024D4D50708154B002B08BF134B96
:1002E0009D46A3F5803A00218B460F461348144AD9
:1002F000121A30F05DF90F4B002B00D098470E4BCF
:10030000002B00D098470020002104000D000D486C
:10031000002802D00C481BF0CDFE2FF047FC200037
:10032000290008F0CFFC1CF0D9F800BF000008003D
:100330000000082400000000218C0408E0180024BC
:10034000981E0124B5C00508000000000020704779
:1003500070470000054B10B504460360806810B17B
:1003600003685B689847204610BD00BF707107089E
:10037000034B10B504460360FFF7ECFF204610BDA9
:10038000F067070810B50446FFF7F2FF102120467A
:100390001CF014F9204610BD10B50446FFF7DAFF33
:1003A000102120461CF00AF9204610BD70470000BD
:1003B00038B50B4B0546446903607CB16368013B6B
:1003C00063605BB9236820469B689847A368013B3C
:1003D000A3601BB923682046DB689847284638BDD0
:1003E000C070070806480023064A0749C0E90133E0
:1003F0004FF4FB738381054B03601BF059BE00BFB4
:10040000FC1800240000002471030408F0670708AA
:10041000014801F03FBD00BF1C2C0024014801F041
:1004200039BD00BF1C2C00240020704700207047FD
:100430000020704700207047002070470020704760
:1004400010B50446692006F0A1F82146C0B2BDE807
:10045000104006F0AFB90000044B10B5044640F858
:10046000043B05F0EDFF204610BD00BF18680708EB
:1004700008B5002006F08AF80021C0B206F09AF90B
:10048000892006F083F80021C0B206F093F9182005
:1004900006F07CF80121C0B206F08CF97D2006F050
:1004A00075F80121C0B206F085F90020FFF7C8FFFA
:1004B0000A2006F06BF80121C0B206F07BF9092092
:1004C00006F064F80121C0B206F074F98F2006F03E
:1004D0005DF80021C0B206F06DF98E2006F056F8E6
:1004E0000021C0B206F066F96E2006F04FF8012137
:1004F000C0B2BDE8084006F05DB900002DE9F0414A
:1005000086B0054601F076FC354B2420354E2B6035
:100510001CF020F804463449684605F0DCFF20460C
:10052000694640F8046B05F0F7FF0A23684623820A
:100530000023636105F084FF2C4BC5F8104128208F
:100540002360636943F0020363611CF003F804460F
:10055000274903A805F0BFFF0DE0684605F070FFCE
:10056000242120461CF02AF8284640F8046B05F0A8
:1005700067FF2CF09FFE274603A947F8046B384617
:1005800005F0CAFF0A2303A823820023636105F054
:1005900057FF184B4FF4647023601BF0DBFF80465D
:1005A000FFF704FF10E003A805F04AFF2821D8E771
:1005B0004FF4647140461CF001F826603846F3E7BA
:1005C000FBE7CDE7F2E7CFE763692846C4F824806C
:1005D00043F00203C5F81441636106B0BDE8F08141
:1005E0008468070818680708C8680708606807086B
:1005F000F76807083C68070808B5044801F0B8FB2D
:100600006420BDE8084006F00DB800BF7019002452
:10061000026810B542B1D0E90143A3423FBF5C1C60
:100620000968846042F8231010BD000008B4036814
:100630008B4277B50446164623DBC36821EAE17591
:1006400013B1294680689847237953B10F4BA068AE
:100650002B4413F8011C05F0CCFD0D49A06805F0F2
:10066000C4FD08AA07992046019201F0A1FA236966
:1006700013B12946A06898471EB10649A06805F045
:10068000B4FD03B0BDE8704001B07047AF68070823
:10069000D493070873970708436807B501220093AE
:1006A0000621044B0448FFF7C1FF002003B05DF8AA
:1006B00004FB00BFDA690708D42B002408B40368E0
:1006C0008B4277B50446164623DBC36821EAE17501
:1006D00013B1294680689847237953B10F4BA0681E
:1006E0002B4413F8011C05F084FD0D49A06805F0AA
:1006F0007CFD08AA07992046019201F073FA23694C
:1007000013B12946A06898471EB10649A06805F0B4
:100710006CFD03B0BDE8704001B07047A8680708E1
:10072000D49307087397070808B501220B460621E2
:10073000FFF7C4FF08BD000070B586B00546FFF79F
:1007400097FE0120FFF77CFE2749284801ACFFF700
:10075000EBFF274E274B0093331D0FCB84E80F0090
:10076000337D6A46244925488DF8143001F0B3FCE6
:10077000224801F0CFFC38B92149224805F048FD54
:10078000012005F04FFFFBE71C4801F0D5FB0228D4
:1007900003D11D491B4805F03BFD1C4802F0CEFA71
:1007A000FF211B4802F0B4FD20B91A49154805F095
:1007B0002FFDFEE700221648114602F007FD012139
:1007C0000022134802F002FD002319466A6A42F82B
:1007D00023106A6A1A440133642B82F8F411F5D1AC
:1007E000002006B070BD00BFF1680708D42B0024BC
:1007F0001C1900247C7C0708040000241C2C002405
:10080000FF680708B8330024456907080C1900245D
:100810003419002466690708B12337B5A82200936C
:10082000C0210123124805F075FC12480023124C28
:10083000124D22461249C0E901334FF4FB73838104
:10084000104B03601BF034FC284602F055FD28468F
:100850000D4D22460D491BF02BFC2846FFF74EFE9E
:1008600022460B49284603B0BDE830401BF020BCAF
:100870001C1900240C190024000000243419002441
:1008800071030408F0670708701900249D320408FA
:100890005904040873B51A4D04464FF4964118489C
:1008A00004F0D2F8164803F009FF20B9284603F0F7
:1008B000E5FF0028F6D00123114A0621114801F076
:1008C00080F80022104B06210E4802ADFFF7AEFE65
:1008D00004F12406D4F81031304645F8043D294689
:1008E000FFF796FED4F81431294630460193FFF7FE
:1008F0008FFE204601F09CF9002002B070BD00BFC1
:10090000B8330024D42B0024B668070808B504497E
:100910000448FFF709FF0448FFF7BCFF08BD00BF0C
:10092000F3690708D42B00247019002408B50C487B
:100930000C49FFF7F9FE0C4802F0D6FB60B10B49F9
:100940000748FFF7F1FE0021074802F05FFC28B1DD
:100950000749084816F010FD002008BD0021F8E7FF
:10096000D42B002489690708742D00249469070892
:100970003DCF733F881A002408B51D491D48FFF775
:10098000D3FEFFF775FD0120FFF75AFD092005F0A2
:10099000FDFD0021C0B205F00DFF8F2005F0F6FD32
:1009A0000121C0B205F006FF8E2005F0EFFD012108
:1009B000C0B205F0FFFE4FF4FA7300224FF4E131AC
:1009C0000D4800F0C7FC40F213434FF4964201215A
:1009D0000A4802F0ABFB20B909490A4805F018FCA7
:1009E000FEE701220021054802F0F0FB002008BDCF
:1009F000AB690708D42B0024401E0024742D00246A
:100A0000B7690708B833002410B586B0002218492A
:100A1000684601F0CDFC684601F006FD10B31549AB
:100A20001548FFF781FE6946144802F091FC134C0B
:100A3000684601F04DFD58B1204602F057FC0021F8
:100A4000204602F0E3FB0121204602F0DFFBEFE746
:100A50000B490948FFF768FE04E06846FFF7A8FC69
:100A60002CF028FC6846FFF7A3FC002006B010BD60
:100A70000C190024D2680708D42B00243419002450
:100A8000DD680708704710B504461C3019F060FB9C
:100A9000204610BD10B5044619F05AFB204610BD83
:100AA00010B504466C3016F0B9FC04F1480016F09D
:100AB000B5FC04F1240016F0B1FC204616F0AEFCA3
:100AC000204610BD38B504460D461C2200212FF0EB
:100AD0006FFD2046294619F0B7FB204638BD0000BF
:100AE00038B504463421FFF7EDFF352104F11C0031
:100AF000254DFFF7E7FF432104F13800FFF7E2FF40
:100B0000632104F15400FFF7DDFF372104F1700089
:100B1000FFF7D8FF762104F18C00FFF7D3FF972170
:100B200004F1A800FFF7CEFF7F2104F1C400FFF716
:100B3000C9FF7A2104F1E000FFF7C4FF042104F1AA
:100B4000FC00FFF7BFFF082104F58C70FFF7BAFF28
:100B5000262104F59A70FFF7B5FF2A4640F62301D7
:100B600004F5A87016F0DEF82A4640F6220104F5D6
:100B7000E07016F0D7F82A4640F6010104F50C7033
:100B800016F0D0F8204638BD0000C07F10B50446EE
:100B90001221FFF797FF862104F11C00FFF792FF57
:100BA000792104F13800FFF78DFF992104F15400F9
:100BB000FFF788FF422104F17000FFF783FF8321D4
:100BC00004F18C00FFF77EFF822104F1A800FFF7FB
:100BD00079FF332104F1C400FFF774FF0E2104F103
:100BE000E000FFF76FFF204610BD10B50446A430AB
:100BF00016F056FB04F1540016F052FB201D16F0BF
:100C00004FFB204610BD10B5044600F58470FFF779
:100C1000ECFF2046FFF7E9FF204610BD10B5044663
:100C200000F59E7016F00CF9204610BD2DE9F34139
:100C30004FF47A73002504464FF48072C56129464B
:100C400004F59E76058404F52777C0E90153224B0D
:100C500003602023C0E905358923283020F8063CAD
:100C60004FF6FF7320F8043C20F8023C2FF0A0FC64
:100C7000C4F8285184F838517D22C4F82C51182129
:100C8000C4F83051304616F07DF8284605F07EFC59
:100C900005468D2005F07AFC80468A2005F076FC1A
:100CA000009043462A462146384600F0D3FB04F51F
:100CB00034731C22002118462FF07AFC00220D21EB
:100CC00019F0ACFA04E0304616F0BAF82CF0F2FA5B
:100CD000204602B0BDE8F0815C78070837B50621F0
:100CE0004F4800F0D7F84F4A07214F4800F032FA3A
:100CF00036214E48FFF7E6FE84214D48FFF7E2FE1D
:100D00006A214C48FFF7DEFE2F214B48FFF7DAFE41
:100D10004A48FFF78BFF4A4A4A4948481BF0C8F93E
:100D20004948FFF7DDFE464A484947481BF0C0F9ED
:100D30009B21474816F054FBA121464816F050FB72
:100D40006721454816F04CFB2721444816F048FB24
:100D5000002401253A4A42493D481BF0A9F97B236A
:100D60007C2298213F48CDE9004500F04BF99A23B9
:100D700087222D213C48CDE9004500F043F90CE0E5
:100D8000354816F04BFB334816F048FB304816F058
:100D900045FB2CF08FFAF6E7F8E7294A334931484A
:100DA0001BF086F93248FFF7F1FE324800F0FEF9F9
:100DB000314800F0FBF97E213048FFF783FE3048D0
:100DC00000F0C6F91C2200212D482FF0F1FB012272
:100DD00019212B4819F020FA194A2A4928481BF0F2
:100DE00067F91C22002128482FF0E2FB00221E2177
:100DF000254819F013FA1C22002124482FF0D8FBB3
:100E00001F21224819F005FA0D4A21491E4803B056
:100E1000BDE830401BF04CB91248FFF7E6FEB8E7DA
:100E2000181B0024D4240024201B0024341B00247D
:100E3000501B00246C1B0024881B0024A41B0024CE
:100E4000000000241D0C040814220024850A040854
:100E5000881A0024AC1A0024D01A0024F41A0024A2
:100E6000A10A0408042000240C210024070C040813
:100E7000E81E0024901E0024E41F0024E81F002424
:100E8000941E0024950A0408B01E0024CC1E0024E1
:100E9000870A0408014A018042607047D424002474
:100EA000034B044A1A6001221A715A71704700BF3D
:100EB000B424002440420F007047D0F804310133BD
:100EC000C0F80431704738B50446043016F0BAF95A
:100ED000054604F1540016F0B5F9237840EA4500C0
:100EE000C4F8FC003BB903281ED1D4F8003101330B
:100EF000C4F8003107E0012B18D1D4F8F830032BE7
:100F000004D10028F1D0C4F8F80038BD13B9032883
:100F1000F9D1EAE7022B05D10128F4D1D4F8003148
:100F2000013BE5E7012BEED10228F6E7022BEAD1DF
:100F3000D4F8F83080EA0302032AE4D09842E2D0E1
:100F400083EA6003D4F8002113F0010308BF4FF0D7
:100F5000FF33D31ACCE70B6803604B6843608B68A0
:100F600083607047C3680BB19B681847704710B522
:100F70000446FFF7F7FF204610BD10B4D0E9003457
:100F800009686210E4075DF8044B01EB020044BFFE
:100F90008A58D35818470146043008B5FFF7EDFFCB
:100FA00008BD0000034A0346C26007C983E8070082
:100FB000704700BFFC69070810B586B0044603916E
:100FC000684606A980E80C0001E90C00204603A948
:100FD000FFF7E8FF204606B010BD37B56C46054662
:100FE00084E80C0094E80C00FFF7E6FF284603B005
:100FF00030BD08B5FFF7CFFF08BD08B5FFF7F9FF13
:1010000008BD00002DE9F0470446061D8EB01546C8
:1010100004F1540730469A469DF85C9016F01AF990
:101020002946384616F016F904F1A4085146404600
:1010300016F010F9002384F800903046C4F800310F
:10104000C4F80431169BC4F8F43016F0FBF80546DA
:10105000384616F0F7F8002340EA45003A4D21469D
:1010600001936B460095C4E93E000CCB0AA8FFF73C
:10107000B4FF0AA9304616F031F90AA8FFF777FF46
:10108000B9F1000F32D00023029521460AA803933C
:1010900002AB0CCBFFF7A1FF0AA9304616F03BF9D3
:1010A0000AA8FFF764FFB9F1020F1FD100230495CE
:1010B00021460AA8059304AB0CCBFFF78EFF0AA9C3
:1010C000384616F00BF90AA8FFF751FF00230695E2
:1010D0002146079306AB0AA80CCBFFF77EFF0AA9AF
:1010E000384616F018F90AA8FFF741FFBAF1FF3F9A
:1010F00010D0164B21460AA808930023099308AB89
:101100000CCBFFF76AFF0AA9404616F0E7F80AA8D9
:10111000FFF72DFF20460EB0BDE8F0870AA8FFF7C5
:1011200026FF404616F0BCF8384616F0B9F83046AF
:1011300016F0B6F82CF0BEF8F0E7EFE7EEE7EDE7D3
:10114000EFE7F1E7F3E700BFC70E0408BB0E0408A2
:1011500070470000C0E90112044AC260002210B5C5
:1011600002740122024C4274046010BD00093D006B
:1011700066660640064B074A1A6007225A60064A0E
:101180009A60064ADA6000221A7401225A74704783
:10119000BC24002466660640D424002400093D00D7
:1011A000014800F003B800BFD024002422230370BC
:1011B000704710B5C36886B001228DF80F100DF18D
:1011C0000F01186803680092DC680DF11703A0474F
:1011D0009DF8170006B010BDF8B5427A04460368C2
:1011E0000E46CFB29B680D0A62B93946984723680C
:1011F00060F3070629469B682046984760F30F2650
:10120000B0B2F8BD29469847236860F30F263946E7
:101210009B682046984760F30706F1E7C36813B55B
:10122000186803680092DC680B46A04702B010BD46
:10123000704770477047C36810B5044653B11868CB
:1012400040B103685B6898470421E0681BF0B6F979
:101250000023E36010BD10B5044618211BF0AEF961
:10126000204610BD436873B599426D4604460E464C
:1012700085E8060004D1BDF8042003899A420FD006
:10128000E36808219DF80420186816F008FBE3685D
:101290003146186816F021FB0098AB886060238106
:1012A00002B070BD73B5C568044625B904201BF0B3
:1012B00051F9E0600560E3681B6883B94FF0FF36C1
:1012C00074201BF047F9B4F91430B4F91020054626
:1012D000B4F91210009616F0E7FBE3681D6002B047
:1012E00070BD742128461BF069F92BF0E3FF000064
:1012F00038B50A2005F05EF90546082005F05AF9D0
:101300000446092005F056F9094B0A4A0121988242
:1013100018461A60002259725A601A72DA601D82E9
:101320005C82054A0549BDE838401AF0C1BE00BFDD
:10133000D4240024106A0708000000243512040891
:101340000268322313B50093946A40F21342A04717
:1013500002B010BD13B5046800931346A46A40F2AE
:101360001342A04702B010BD13B5322304680093A6
:10137000A46AA04702B010BD006903681B69184742
:10138000006903689B691847006903685B6918472F
:1013900000690368DB6818470120704770B5044690
:1013A0000D4616460499C5622286026A002A08BFC5
:1013B0001A46436A002B18BF1946026241628069CF
:1013C000002807DB0121C0B205F070F90021207E62
:1013D00005F0F0F9E069002807DB0121C0B205F053
:1013E00065F90121207F05F0E5F9002320693246E7
:1013F000294684F828300368BDE870401B6A184706
:1014000010B50446006903685B6A9847A069002824
:1014100007DB0021C0B205F0CDF90021207E05F0E8
:1014200045F9E069002809DB0021C0B205F0C2F9E6
:10143000207F0021BDE8104005F038B910BD0346FB
:1014400090F8280018B1186903681B681847012232
:101450005A60704770B500254FF47A768361049B1B
:10146000456280F82850C0E90156034EC0E90412D5
:101470000660C0E9073570BD4C6A070810B5044620
:101480008069002807DBC0B2012105F093F9206ACA
:1014900008B105F0C9F8012384F8283010BD10B553
:1014A000044600690368DB689847A369002B07DBE3
:1014B000606A08B105F0B8F80021207E05F07AF9DD
:1014C000002384F8283010BDC069002803DB002108
:1014D000C0B205F06FB97047C069002803DB012175
:1014E000C0B205F067B970470A4B00224FF47A7119
:1014F00001205A6283F82820C3E9012106491960B6
:10150000064919611521C3E905011421C3E9071230
:10151000704700BFEC2400244C6A07080430002404
:101520000368C9B21B68184749000023C161C0F8AD
:101530002C327047036801211B6B184710B40368F5
:101540009C6B0123A4465DF8044B6047D0F82C3215
:10155000B3F5807F1FBF5A1CC0F82C22C01880F83A
:101560002C1114BF012000207047D0F828017047CB
:101570007047C0F830127047C0F834127047D0F886
:101580002831A3B1D0F828318BB1D0F82431D0F86C
:1015900024210344013293F82030D2B2C0F8242130
:1015A000D0F82821013AC0F82821184670474FF09A
:1015B000FF307047D0F828312BB1D0F824311844CF
:1015C00090F8200070474FF0FF30704738B503683F
:1015D00004465B6A9847FC201AF0BCFFB4F91A2055
:1015E000B4F91810054615F0AFFD656138BDFC2152
:1015F00028461AF0E3FF2BF05DFE38B5D0F82C3208
:101600001446054600F596701A441844B2F5807FDA
:1016100088BFC3F5807422462EF0CCFED5F82C325C
:1016200020462344C5F82C3238BD38B504464069FD
:101630000D4608B115F0A1FC206920B12946BDE88E
:10164000384015F0D9BD38BD07B581F0010100F56E
:1016500096720091D0F82C32C169406915F0A0FC57
:10166000002814BF0220002003B05DF804FB10B571
:101670000446406920B10368DB6898470023636132
:1016800023699BB1D4F838021BF07BFAD4F83802F6
:101690001BF0FBFAD4F8380210B103685B68984776
:1016A0009C2120691AF08AFF0023236110BD70B5C8
:1016B000C2B083F001030446154602AE0093490010
:1016C00013464069324615F08AFCC8B9A84218D0C2
:1016D000D4F82831B3F5807F10D0D4F82031325CB3
:1016E000234483F82020D4F820310133DBB2C4F83E
:1016F0002031D4F828310133C4F828310130E5E72E
:101700000025284642B070BD30B50446BDB0002566
:10171000206915F07AFD0328FAD8DFE800F04A02C4
:101720001212D4F8343203B19847D4F82C22002A8C
:10173000EED004F59671206915F06BFDC4F82C52BB
:10174000E6E7C4F82051F022C4F824516946C4F8F1
:101750002851206915F05BFD002282421DDAD4F881
:101760002831B3F5807F18D0D4F82831B3F5807FC5
:1017700011D0D4F820311DF80210234483F8201032
:10178000D4F820310133DBB2C4F82031D4F8283149
:101790000133C4F828310132DFE7D4F82831002BB7
:1017A000B6DDD4F83032002BB2D0D4F828019847F7
:1017B000AEE704F049FFABE70022C26070470000CB
:1017C00038B500254FF47A730446018342832946D5
:1017D0004FF48072C0E901530A4BC0E9045503601D
:1017E00020302EF0E5FEC4F82051C4F82C522046DB
:1017F000C4F82451C4F83052C4F82851C4F8345203
:1018000038BD00BFA06A070810B504460021FFF7E5
:10181000D3FF204610BD10B4D0E90034096862102F
:10182000E4075DF8044B01EB020044BF8A58D3582B
:1018300018470146043008B5FFF7EDFF08BD00006A
:10184000034A0346C26007C983E80700704700BF28
:10185000806A070810B586B004460391684606A959
:1018600080E80C0001E90C00204603A9FFF7E8FF1F
:10187000204606B010BD37B56C46054684E80C001E
:1018800094E80C00FFF7E6FF284603B030BD0000E7
:101890002DE9F0410368054688B00E465B6A98471B
:1018A0009C201AF057FEB5F91A20B5F91810044615
:1018B00015F088FC710020462C6115F09FFCBC20BF
:1018C0001AF048FE04460646234B04F1400746F84A
:1018D000043B3046FFF798FF002138461BF0B6F86E
:1018E00004F1540840461BF04FF81C4B4FF40062C3
:1018F00018212046009300231BF038F9184B294685
:1019000004A8C5F8384202930023039302AB0CCB22
:10191000FFF7B1FF04A920461BF0F2F910E04046A2
:101920001BF072F838461BF0D0F83046FFF71FFB6B
:10193000BC2120461AF042FE2BF0BCFCF2E7F4E793
:1019400004A8FFF714FB08B0BDE8F0819C21F0E784
:1019500004A8FFF70CFBEFE7509E07088C6A070806
:101960000917040808B5FFF764FF08BD08B5FFF7BD
:10197000F9FF08BD10B50B2004F01CFE04460C2036
:1019800004F018FE214602460748FFF719FF162209
:1019900017210648FFF714FF7B227C210448BDE88D
:1019A0001040FFF70DBF00BF202500245C27002456
:1019B000982900240629A8BF062121EAE1710160C7
:1019C000704710B5FFF7F6FF0371826010BD00008D
:1019D00073B505461446002940D0252905D18068F5
:1019E00002B0BDE8704004F004BC732909D113684B
:1019F00080681A1D1968226002B0BDE8704004F0CA
:101A0000F4BB532909D1136880681A1D1968226034
:101A100002B0BDE8704004F0E4BB642901D069293C
:101A20000AD12368A8681A1D22600A22196802B028
:101A3000BDE8704004F035BC01F0FD02442A0FD12E
:101A400023688068073323F0070303F1080222604C
:101A500002220092D3E9002304F0C6FC02B070BD5C
:101A6000782905D1236880681A1D22601022DDE7DD
:101A7000582920D14849806804F0B7FB23681A1D13
:101A80001E6840F6FE732260B4B29C420FD830212B
:101A9000A86804F0AEFBFE2C09D83021A86804F039
:101AA000A8FB0E2C03D83021A86804F0A2FB10225A
:101AB000B1B2A868BBE7702909D1236880681A1DF4
:101AC0001968226002B0BDE8704004F095BB62293D
:101AD00005D12368A8681A1D22600222A6E74229C0
:101AE00004D12E49806804F080FBF2E76C290AD10A
:101AF000236880681A1D196822600A2202B0BDE8B6
:101B0000704004F0ACBB75290AD1236880681A1DA7
:101B1000196822600A2202B0BDE8704004F0C3BB1D
:101B2000632905D1236880681A1D1978226057E758
:101B3000432916D1236880681A1D22601C78A4F1FD
:101B400020035E2B01D821464AE7134904F04DFBE0
:101B50000E2C03D83021A86804F04BFB102221463C
:101B6000A7E774290AD1236880681A1D1B68012B16
:101B7000226001D10A493FE70A493DE754297FF431
:101B80006DAF236880681A1D1B68012B22600CBF93
:101B9000054906493CE700BFF06A0708F36A0708F1
:101BA000F66A07085C9E07080C8207082B82070864
:101BB000F7B54C1C02AD0646097845F8042D79B1FD
:101BC000252909D1671C21782A4630463C46FFF773
:101BD000FFFE21780134F2E7B06804F00AFBF8E771
:101BE00003B0F0BDF7B5064602AD0C4645F8042D2E
:101BF000217871B1252908D1671C61782A463046C1
:101C00003C46FFF7E5FE0134F2E7B06804F0F1FA74
:101C1000F9E703B0F0BD0000044B002201211A6077
:101C200019711A61C3E90222704700BFD42B002446
:101C300070B5044690F82C600025EBB29E420DD999
:101C4000636A53F82500836903B9846143699B067D
:101C500002D50368DB6898470135EEE72368204624
:101C60009B689847D4F80C1119B10B6808469B691A
:101C70009847002070BDF8B506460D4690F82C70C8
:101C80000024E3B29F420CD9736A53F824305B6995
:101C9000DB0604D42B68294628469B699847013403
:101CA000EFE70020F8BD0123C9B2002203FA01F1D9
:101CB000134630B590F82C40D5B2AC4209D9456AEC
:101CC00055F8225001326D6929421CBF0133DBB245
:101CD000F2E7184630BD70B5054690F82C60002438
:101CE000E3B29E420AD96B6A53F8240043695B074A
:101CF00002D503689B6898470134F1E7002070BD66
:101D00002DE9F843044604F06FFC236BC01AD4F8A5
:101D10000831984224D9002694F82C70DFF84880C6
:101D20003546DFF84890F3B29F4211D9636A53F801
:101D3000260043699B0709D503685B68984728B16B
:101D4000013541464846EDB204F062FA0136EAE751
:101D50001DB10549054804F05BFA04F045FC206319
:101D60000020BDE8F88300BF73970708B83300244C
:101D70002DE9F8430546002604F036FC4FF0010932
:101D800007462C4605F1C808226C62B1A36CE16CD1
:101D9000FB1A8B4207D3606C9047E8B1236DDBB12F
:101DA000C4F85090A76414344445EDD104F01CFCF1
:101DB000002495F82C60E861E3B29E4212D96B6A68
:101DC00053F8240043691B0704D5EB69C36103681A
:101DD0001B6998470134EFE7C4E91066C4E912664D
:101DE0002665E0E72B6828465B6898470020BDE839
:101DF000F883000030B585B00446134901A804F00B
:101E00006AFB2046114B01A940F8043B04F084FB17
:101E100004E001A804F014FB2BF04CFA00252C235D
:101E200001A86361258204F00BFB094B2046E562A3
:101E300023604FF47A732563C4F80831054B63625D
:101E40000A23A36205B030BDF86A070818680708BE
:101E5000046B0708E82B0024024B0022C3E9002290
:101E60009A607047102C00240020704700207047B3
:101E700000207047002070470020704770470368BB
:101E800053F8683C184470477047036853F8743C33
:101E900018447047D0F8140118B1036853F8843C13
:101EA0001844704738B50D460431044612F0F0FA74
:101EB000EB682046C4F8843053F8843C2A692344F4
:101EC000C3F884202B68236053F8843C6A69E2508D
:101ED000AB69C4F8843038BD0B4B10B503601346B2
:101EE0000A460A49044612F0D3FA04E0204612F0EA
:101EF00035FF2BF0DFF9064B2046236003F5807396
:101F0000C4F8843010BD00BF248A0708346E070867
:101F1000D06E070870B5074B044605460E4644F8D8
:101F2000043B0B1D0FCB84E80F00337D28462B7537
:101F300070BD00BF7C7C0708D0F8140108B50368A9
:101F40009B6D984701280CBF0120022008BD70B589
:101F50000446164629B1D0F81431586803685B6905
:101F6000984704F041FB0546D4F8140100210368AA
:101F7000DB6D9847D4F8140103689B6C984704F014
:101F800033FB401BB04208D22046FFF7D5FF0128A3
:101F900003D00A2004F046FBF1E72046FFF7CCFF10
:101FA000431E5842584170BD70B59AB01D46044654
:101FB0000E4602A81146FFF7ADFF294608A814AD4A
:101FC000FFF7A8FF1E990EA8FFF7A4FF1F99284648
:101FD000FFF7A0FF08AA00950EAB02A9204600F06B
:101FE00057FFD4F81401002103685B6C9847D4F8BC
:101FF000140104F13402211D03681D6C04F11C035B
:10200000A847D4F8143104F14C011A6852F8840C32
:102010001A58184455690022A84731462046DDE980
:102020002023FFF794FF1AB070BDF0B51C46A3B093
:102030000023154606460F460093FF2304A81A46C0
:10204000194604F067F829460AA81CADFFF762FF9D
:10205000214616AC10A8FFF75DFF28992046FFF730
:1020600059FF04A92846FFF755FF4EF660234FF4A9
:102070007A6239463046CDE9023210AB0AAACDE980
:102080000045FFF791FF23B0F0BDF0B59BB00546CA
:102090000E46114602A814461F46FFF73BFF0321D8
:1020A00002A804F05AF80123214614AC037008A8D2
:1020B000FFF730FF39460EA8FFF72CFF02A9204694
:1020C000FFF728FF0EAB08AA314600942846FFF719
:1020D000ACFF1BB0F0BD70B592B005460E46114680
:1020E00068461446FFF716FF0321684604F035F8EA
:1020F00001232146037006A8FFF70CFF69460CA8D0
:10210000FFF708FF0CAB06AA31462846FFF7BDFFD4
:1021100012B070BD0620704710B50446006808B1C3
:102120001AF05FFA204610BD0B4B10B5044640F87C
:10213000643BFFF7F1FF04F14C00FFF7EDFF04F102
:102140003400FFF7E9FF04F11C00FFF7E5FF201D55
:10215000FFF7E2FF204610BD306B07082DE9F04184
:10216000002205461E4B0446114645F8043B28460E
:1021700013F014F804F11C0600223046114613F047
:102180000DF804F1340700223846114613F006F822
:1021900004F14C0800224046114612F0FFFF0022D5
:1021A00004F16400114612F0F9FF10E04046FFF719
:1021B000B3FF3846FFF7B0FF3046FFF7ADFF2846C4
:1021C000FFF7AAFF2BF076F8F3E7F5E7F7E7002330
:1021D000204684F87C30C4F88030BDE8F08100BF30
:1021E000306B070810B50446FEF7BCFE204610BD54
:1021F00038B504460D4689B91368236085B952681D
:1022000053F8843CE25004F17400FFF7EBFFAB0796
:1022100002D5204612F0A2FD204638BD024BECE765
:10222000014A0023EEE700BFE48807080A460021C0
:10223000FFF7DEBF00220221FFF7DABFD0F800C0AF
:10224000ACF1240CDCF800C06044F3E710B50446A0
:10225000FFF7F0FF842120461AF0B0F9204610BDA8
:10226000D0F800C0ACF1240CDCF800C06044EDE70D
:1022700070B504460D4609BB1368236005BB516960
:1022800053F8843CE150F5B99169234643F8841F23
:10229000DDB902F10C010868C4F884004E6850F8FA
:1022A000841C5E509DB9111D2046FFF7BFFFAB0790
:1022B00002D5204612F052FD204670BD054BDCE7EA
:1022C00004490023DEE70449DFE70449E3E7044962
:1022D000EAE700BFD06E0708D06F07083C6E07081A
:1022E000346E070800220221FFF7C2BFA0F184006C
:1022F000F8E7D0F800C0ACF1240CDCF800C0604472
:10230000F0E70000054B10B5044640F88C3BFFF7A2
:10231000E9FF2046FFF708FF204610BD547007086C
:1023200010B50446FFF7DEFF882120461AF046F973
:10233000204610BDA0F18400F2E7D0F800C0ACF157
:10234000240CDCF800C06044EAE70A460021FFF7ED
:102350008FBF000038B5124C2046FFF7FFFE114B2F
:102360002360002384F8883007F00AFC054611F04A
:10237000F9FD0246294604F18C00FFF7ADFD04F19A
:102380008C00094A0949C4F814012046BDE83840C8
:1023900019F08EBE0248FFF7C7FE2AF08BFF00BF80
:1023A0001C2C002454700708000000240523040896
:1023B00037B5002315464FF47A720446C0E901325E
:1023C000C0E90433164B0360886828B3036801A989
:1023D0001B6C98470146019A1DB1B2FA82F35B0962
:1023E0002B70CAB9204600F09FF815E00D4B236012
:1023F00064697CB16368013B63605BB92368204614
:102400009B689847A368013BA3601BB923682046DB
:10241000DB6898472AF04EFF204603B030BD00BF6E
:1024200060700708C0700708006918B18068003044
:1024300018BF01207047000003692DE9F0410446F0
:1024400086B00E46904613B903689B6B9847256982
:1024500001AC2B689F68084B0093331D0FCB84E8B9
:102460000F00337D4246694628468DF81430B84740
:1024700006B0BDE8F08100BF7C7C0708036970B539
:1024800004460D46164613B903689B6B98472069AE
:10249000324629460368BDE87040DB68184770473C
:1024A000C06810B103685B68184770470020704728
:1024B00010B5044610211AF081F8204610BD08B569
:1024C000FFF7F6FF08BD006908B100F0A5B9704735
:1024D000006908B100F0E5B97047006908B100F083
:1024E000F9BB7047006908B100F0C6BB70470069CE
:1024F00008B100F090B97047006908B100F01AB94E
:102500007047006908B100F018B94FF0FF3070470C
:10251000006908B100F03CB97047006908B100F0EB
:102520006FB94FF0FF30704738B5036904460D4668
:1025300013B903689B6B984729462069BDE838406A
:1025400000F0F0BA38B5046805467CB16368013B19
:1025500063605BB9236820469B689847A368013B8A
:10256000A3601BB923682046DB689847284638BD1E
:1025700037B504464FF4AA7019F0ECFF054600F099
:10258000A3F9002310200095019319F0E3FF012324
:102590002269C560C0E90133124B0360009B0092C1
:1025A00023616369606102A840F8043DFFF7CAFF38
:1025B0002368256920465B6B9847686003B030BD8F
:1025C0002AF0B0FD2B6828465B6898472AF0A4FFE4
:1025D0002AF0E8FD2AF06EFE4FF4AA71284619F0A1
:1025E000EDFFF7E7A47007080121D0F848011AF0C1
:1025F00067B900002DE9F0410446C0B04FF0010872
:102600002B4F2B4D01236422FF21D4F848011AF0EF
:1026100078F9D4F81431B3F5807F06D104F014F8BA
:10262000BD42F6D0002DF4DCEBE7D4F84C011AF0F3
:10263000B3F9A06858B1D4F8142169460368C2F50B
:1026400080725B699847061E07DABE4206D00023F7
:1026500084F8183140B0BDE8F08107D103F0F4FFF1
:10266000D4F84C011AF0B6F93546D9E70025D4F86C
:102670001431B3F5807F10D0D4F80C311DF805204B
:1026800023441A73D4F80C310133DBB2C4F80C3193
:10269000D4F814310133C4F814310135AE42E6D117
:1026A000D4F84C011AF096F984F81881B1E700BF0C
:1026B00047F4FFFF0C30704738B50025044611225F
:1026C00040F8045B29462DF073FFE582204638BDB3
:1026D0002DE9F0470646DFF858A0124D89463446EA
:1026E000114F12490F4803F080FDA31B994513DDDC
:1026F0002378A0460F2B03D85146284603F075FDDA
:1027000098F8001010222846013403F0D9FD39460C
:10271000284603F06AFDE8E70248BDE8F04703F009
:1027200071BD00BFB8330024E4930708087107089F
:10273000E9CB0708D0F81401704738B50446D0F843
:102740004C011AF029F9D4F814313BB94FF0FF3598
:10275000D4F84C011AF03EF9284638BDD4F81431AB
:102760009BB1D4F8103123441D7BD4F810310133D0
:10277000DBB2C4F81031D4F81431013BC4F8143181
:10278000D4F84C011AF026F9E6E74FF0FF35F7E7E9
:1027900070B50446D0F84C010E4615461AF0FCF808
:1027A000D4F8143133B9D4F84C011AF013F94FF0BE
:1027B000FF3070BD9D423146A8BF1D467019814251
:1027C00018D0D4F8143193B1D4F8103123441A7BC3
:1027D000D4F810310133DBB2C4F81031D4F814311D
:1027E000013BC4F81431134601F8013BE7E74FF011
:1027F000FF33F9E7D4F84C011AF0ECF82846D8E793
:10280000D0F8143123B1D0F810311844007B704750
:102810004FF0FF307047704738B50446D0F84C0190
:1028200008B11AF0B9F8A06838B194F81921036812
:10283000A2B35B6898470023A360D4F84C0108B1A9
:102840001AF0C8F8D4F8440150B11AF0BBF9D4F822
:10285000440110B103685B6898470023C4F8443111
:10286000D4F848514DB128461AF030F814212846C2
:1028700019F0A4FE0023C4F84831D4F84C514DB1EE
:1028800028461AF0C1F82421284619F097FE0023A3
:10289000C4F84C31002384F8183138BD9B68984740
:1028A000C9E790F818312BB9D0F81431002BD4BFF8
:1028B000002301231846704710B504460021FEF797
:1028C0007BFF204610BD000038B50025134B0446A1
:1028D0004FF4807203602946C0E901550C302DF099
:1028E00067FEC4F80C5184F8185104F58E70C4F8D2
:1028F000105184F81951C4F81451FFF7DDFF04F5A5
:102900009670FFF7D9FEC4F84451C4F848512046E8
:10291000C4F84C51C4F8505138BD00BF20710708AD
:1029200010B50446FEF71EFB204610BD074B10B540
:1029300004460360FFF770FF04F59670FFF7ECFBA9
:1029400004F58E70FFF7ECFF204610BD20710708DC
:1029500010B50446FFF7EAFF4FF4AA71204619F0BC
:102960002DFE204610BD10B4D0E900340968621075
:10297000E4075DF8044B01EB020044BF8A58D358CA
:1029800018470146043008B5FFF7EDFF08BD000009
:10299000034A0346C26007C983E80700704700BFC7
:1029A000FC70070810B586B004460391684606A976
:1029B00080E80C0001E90C00204603A9FFF7E8FFBE
:1029C000204606B010BD37B56C46054684E80C00BD
:1029D00094E80C00FFF7E6FF284603B030BD000086
:1029E0002DE9F0470B680D468AB00446D0F8501127
:1029F00028461B6B98472B6800212846DB6A9847BE
:102A00002B6804F5967128469B6C9847D4F848319A
:102A10003BB9142019F09EFD064619F041FFC4F899
:102A20004861D4F84C313BB9242019F093FD064697
:102A300019F0AAFFC4F84C61D4F84C0119F0ACFFAE
:102A4000D4F84471002F42D1BC2019F083FD064612
:102A50008046314B06F1400948F8043B4046FEF7FA
:102A6000D3FE3946484619F0F1FF06F1540A5046A4
:102A700019F08AFF4FF48053182216213046CDE911
:102A800000771AF03BF8254B214606A8C4F84461AC
:102A9000CDE9023702AB0CCBFFF795FF06A9304614
:102AA0001AF02EF910E0504619F0AEFF48461AF021
:102AB0000CF84046FEF75BFABC21304619F07EFD6B
:102AC0002AF0F8FBF2E7F4E706A8FEF750FAD4F88C
:102AD0004C0119F07FFF2B68214606A85E6B104B56
:102AE00004930023059304AB0CCBFFF76CFF06A9FE
:102AF0002846B04706A8FEF73AFA012384F81831B1
:102B00000AB0BDE8F0871421D7E72421D5E706A84D
:102B1000FEF72DFAD4E7FAE7509E0708F5250408DA
:102B2000E92504088160FFF75BBF000073B5044628
:102B300080680E4668B1D4F8443153B1036801226D
:102B40000DF107015B699847002802DA2046FFF77C
:102B500063FEA3684BB9902019F0FCFC054612F007
:102B600041FD0123A56084F81931A5681DB9002530
:102B7000284602B070BD606803685B6F98470146E5
:102B8000284611F0E3FF05460028F0D1A068314641
:102B90000368DB689847094B984203D010B184F86A
:102BA0001851E5E7A1682046FFF71AFF0125F6E76F
:102BB0009021284619F002FD2AF07CFB39F4FFFF32
:102BC000F0B5124B8DB006460D4600930B1D17460F
:102BD00001AC0FCB84E80F002B7D694606A83A466E
:102BE0008DF8143000F0E6F806A93046FFF79EFF96
:102BF00004E006A8FFF790FA2AF05CFB044606A85A
:102C0000FFF78AFA20460DB0F0BD00BF7C7C0708B4
:102C100070B58EB01546044618220E4602A8002153
:102C20002DF0C6FC02A8FFF747FD60680023ADF851
:102C30001E50026831460093156802AAA84702A9EF
:102C400008A812F06EFA08A92046FFF76FFF08E007
:102C500008A8FFF761FA02A8FFF75EFA2AF02AFB3C
:102C6000F9E7044608A8FFF757FA02A8FFF754FA55
:102C700020460EB070BD0000F8B5044680680E46D0
:102C8000154618B303680121114FDB6A9847A06805
:102C900040F2DC5103681B6B984729463046FFF72A
:102CA00017FDA0682A46314603681B69984785428C
:102CB00006D0B84204D12046FFF7F3FD0028F0D13A
:102CC000A1682046FFF78CFE2846F8BD0546FBE7C5
:102CD00047F4FFFF07B502AB012203F8011D1946B7
:102CE000FFF7CAFF03B05DF804FB08B5FFF749FE24
:102CF00008BD08B5FFF7F9FF08BDCB68C3600BB18D
:102D00005B681847704707B580688DF8071030B1C9
:102D1000036801220DF107011B699847012003B0E8
:102D20005DF804FB806810B5144620B103681B6988
:102D30009847204610BD0446FBE7000038B583687D
:102D40000446ABB9902019F005FC054612F04AFC88
:102D500023682046A5605B69984703685B6F9847C6
:102D60000146284611F0F2FE0F49104803F050FAD0
:102D7000A068C0B1A18911F00BFEA068052103680D
:102D80005B6C9847A06800210368DB6A9847084994
:102D90000648BDE8384003F03BBA9021284619F0B8
:102DA0000DFC2AF087FA38BD30710708B8330024CB
:102DB00046710708F0B587B00C4605461746012650
:102DC0001122002101A82DF0F3FB002120468DF8EF
:102DD000046003F0C2F90378314620468DF80530CF
:102DE00003F0BBF90378022120468DF8063003F08A
:102DF000B4F90378032120468DF8073003F0ADF9CC
:102E000003783A4601A928468DF8083012F072F985
:102E1000284607B0F0BD70B58CB00C4611220646AE
:102E20000021012501A82DF0C3FB002120468DF8CB
:102E3000045003F092F90378294620468DF80530B6
:102E400003F08BF90378022120468DF8063003F059
:102E500084F90378032120468DF8073003F07DF9CB
:102E6000037801A9002206A88DF8083012F042F973
:102E700006A906F14C0012F0F4F906A8FFF74CF988
:102E80000CB070BD06A8FFF747F92AF013FA00004E
:102E90002DE9F0410D46044696B05849284617469C
:102EA0001E4603F049F980F00100C0B284F87C00AE
:102EB000002800F09980112200214FF0010801A89C
:102EC0002DF076FB002128468DF8048003F045F9AB
:102ED0000378414628468DF8053003F03EF9037823
:102EE000022128468DF8063003F037F903780321D4
:102EF00028468DF8073003F030F9037801A9002245
:102F000010A88DF8083012F0F5F810A9201D12F065
:102F1000A8F910A8FFF700F91122002106A82DF04A
:102F200047FB002130468DF8188003F016F903782E
:102F3000414630468DF8193003F00FF9037802212D
:102F400030468DF81A3003F008F903780321304633
:102F50008DF81B3003F001F9037806A9002210A8B0
:102F60008DF81C3012F0C6F810A904F11C0012F004
:102F700078F910A8FFF7D0F8112200210BA82DF046
:102F800017FB00211C988DF82C8003F0E6F80378DD
:102F900041461C988DF82D3003F0DFF803780221AC
:102FA0001C988DF82E3003F0D8F8037803211C9874
:102FB0008DF82F3003F0D1F803780BA9002210A868
:102FC0008DF8303012F096F810A904F1340012F0A8
:102FD00048F910A8FFF7A0F8394610A8FEF79AFFA5
:102FE00010A92046FFF717FF16B0BDE8F08110A822
:102FF000FFF792F82AF05EF9F9E7F8E7EC400024D1
:10300000064B10B504460360406A08B12CF08CFEF4
:10301000606808B101F080F8204610BD987107087B
:1030200010B50446FFF7ECFF3821204619F0C6FA28
:10303000204610BD064A02600022C0E90121C2609C
:1030400002744263C0E90922C0E90B22704700BF45
:1030500098710708034B10B504460360FFF7D0FFD3
:10306000204610BDA871070810B50446FFF7F2FF0F
:103070003C21204619F0A2FA204610BD10B54FF4AD
:103080007A710446FFF7D6FF024B20462360024BBD
:10309000A36310BDA8710708EC24002410B5054CEB
:1030A0002046FFF7EBFF2046034A0449BDE81040E5
:1030B00018F0FEBF382D002400000024553004080D
:1030C000034B10B50446036000F064F8204610BDC1
:1030D000B871070810B50446FFF7F2FF3C212046FF
:1030E00019F06CFA204610BD10B5C0B00446406817
:1030F000694600F0F1FB021E08DD04F10803694691
:10310000606800F07FFC012040B010BD0020FBE7AC
:1031100010B5044600F030F8024B20462360024B05
:10312000A36310BDB8710708EC24002470B50546F0
:103130000E46806B11461A4600F054FA3246044699
:103140000146284600F09AF818B1204600F0F4FB3A
:10315000012070BD10B5054C2046FFF7D9FF204671
:10316000034A0449BDE8104018F0A2BF742D0024A2
:1031700000000024C1300408054B0021302210B5A6
:1031800004460360416008302DF012FA204610BD5D
:10319000CC7107080C4B10B504460360806A08B177
:1031A0002CF0C2FDE06A08B12CF0BEFD206B08B126
:1031B0002CF0BAFD606B08B12CF0B6FD606808B168
:1031C00000F0AAFF204610BDCC71070870B50E1E96
:1031D0000446154601DB002A06DC2BF03DFD1623D4
:1031E00003604FF0FF3070BD1146806A2DF096FAF3
:1031F000A06210B9C4E90200F5E72A4600212DF0CB
:10320000D7F90120C4E90256EDE7000008B5C3680C
:103210008B4203DC82681A448A4206DC2BF01CFDD8
:10322000044B03604FF0FF3008BDC91A836A585C35
:10323000FAE700BF5042B20610B50446806A08B1F2
:103240002CF072FDE06A08B12CF06EFD206B08B125
:103250002CF06AFD606B08B12CF066FD3022002175
:1032600004F108002DF0A4F9606830B100F072FBA1
:10327000606800F051FF0023636010BD70B5064622
:103280000C461546FFF7D8FF74602CB1294620463E
:1032900000F044FB012070BD2046FCE7034B10B555
:1032A00004460360FFF776FF204610BDE071070873
:1032B00010B50446FFF7F2FF3C21204619F07EF9D5
:1032C000204610BD10B5C2B00446406801A900F008
:1032D00003FB021E08DD04F1080301A9606800F089
:1032E00091FB012042B010BD0020FBE7836B0BB1C6
:1032F000FFF7E8BF1846704710B50446FFF73CFFDC
:10330000024B204623600023A36310BDE071070831
:1033100070B5002488B005460E4623462246214655
:10332000009402A802F0F6FE224602A9204600F010
:1033300069FA3246044601462846FFF79FFF28B146
:10334000204600F044FAB0FA80F0400908B070BDA1
:1033500038B5044640680D4600F044FA00B9A5634C
:1033600038BDF0B5441800250A442746211A8A4280
:1033700000D8F0BDE11BC9085E5C2E41013506F0A6
:10338000010605F0070504F8016BEFE703680B7011
:10339000436802204B7070470B680020023B0B60B3
:1033A000704710B5446BA06803681B69984720B14B
:1033B000A06803685B699847F5E710BD10B504463F
:1033C000406B2CF0B1FC2046BDE810402CF0ACBCAA
:1033D00010B5446BA068FEF77FF8A0680368BDE8ED
:1033E0001040DB6A184710B5446BA068A2880368D8
:1033F00021681B6A9847A068FEF766F8002010BD98
:10340000436B986803F007B810B5446BE2682AB1C3
:10341000012200F093FD0020E06010BD00F08EFD61
:103420000028FAD10123E360F7E770B5446B0D463D
:103430001646A068FEF750F8A068FEF71FF8A068CF
:103440002946324603685B6898470546A068FEF740
:1034500026F8A068FEF738F8284670BD2DE9F0413F
:103460001F46466B0AB313684FF47A75926892FB55
:10347000F5F205FB032503F0B7F88046B068036852
:103480001B699847B842044605DA03F0ADF8A0EB93
:103490000800A842F2D32CB92BF0DEFB4FF0FF342A
:1034A000742303602046BDE8F0811546E3E7000081
:1034B00008B508781378834207D028B12BF0CCFBED
:1034C000034B03604FF0FF3008BD0020FCE700BF56
:1034D0005F42B206F8B504680B789C4200D073BB1B
:1034E000971EFF230E46DFF860E011FA87F71C46AF
:1034F000DFF858C0B74208D016F8015B65401EF8E7
:1035000005405C401CF80530F4E7114443EA04230D
:1035100011F8025C1BB211F8011C41EA052109B245
:1035200099420AD0C3685B0701D5FFF73AFF2BF039
:1035300093FB044B4FF0FF3203601046F8BD0022AE
:10354000FBE700BF5A42B206EC710708EC720708AD
:10355000F72908B502D80160002008BD2BF07CFBDC
:10356000162303604FF0FF30F7E700000068B0F16A
:10357000FF3F10B5029C05D1074B9721074A084829
:103580002BF048FB61701112E2701A1220700620B5
:10359000A1702271637110BD387407089F74070809
:1035A00049740708FF2310FA81FCF0B51A46054656
:1035B0000A4F0B4E654506D015F8014B54403A5D55
:1035C0005A40335DF6E743EA02231BB2C3F30722F6
:1035D000425408444370881CF0BD00BFEC710708DA
:1035E000EC720708F8B5074638200E4615462CF051
:1035F00093FB044600F07EF9064B102023632CF069
:103600008BFB00236063876006608580C360204673
:10361000F8BD00BFEC730708F0B5456B4FF6FF77B8
:10362000059C2E88BE4214BF013600262E802E88AF
:10363000361226702D8865700025A570E57000682B
:10364000E171111262721A12A0710C202172A27221
:10365000E372F0BD83681B120B7083684B7000230C
:103660008B70CB7003688B7143680820CB717047F7
:103670000278407800EB022070478B1F1A124371CA
:10368000027108467047436B186A03685B68184705
:10369000436B186A03685B6A18471046704700005E
:1036A000F0B5446B87B0266A01AD3368DF690A4B19
:1036B000009304F10C030FCB85E80F00237F6946CC
:1036C00030468DF81430A288B847B0FA80F040092F
:1036D000404207B0F0BD00BF7C7C0708436B23B1BC
:1036E000186A10B103689B6A1847704710B5446B9D
:1036F000206A03681B69984720B1206A03685B69E8
:103700009847F5E710BD10B50446406B2CF00CFB54
:103710002046BDE810402CF007BB2DE9F0411F46C4
:10372000466B3AB313684FF47A75926892FBF5F2E0
:1037300005FB032502F058FF8046306A03681B69C9
:103740009847B84204460BDA02F04EFFA0EB08009F
:10375000A84205D2306A0368DB6A98470028ECD19A
:103760002CB92BF079FA4FF0FF3474230360204614
:10377000BDE8F0811546DDE7002200F0DFBB000068
:1037800008B513780878984203D14978537899425C
:1037900006D02BF061FA054B03604FF0FF3004E0D8
:1037A000907810B1D0780028F3D108BD5B42B20602
:1037B000F72908B502D80160002008BDFF29FAD01A
:1037C0002BF04AFA162303604FF0FF30F5E708B5F7
:1037D00030B92BF041FA162303604FF0FF3008BDDB
:1037E0000020FCE708B530B92BF036FA1623036049
:1037F0004FF0FF3008BD0029F6D0436B002019625E
:10380000F8E700002DE9F041064638200F469046C3
:103810002CF082FA054600F06DF8FF2324202B607F
:103820000A4B2B632CF078FA3B1D0662044600F12C
:103830000C0668630FCB86E80F003B7D2846C4F872
:103840000480237700232380BDE8F081E874070813
:1038500010B5036904464FF47A70584302F0E2FE53
:10386000A069BDE8104002F0DFBE10B520B1036BC7
:10387000BDE810401B6C18472BF0EEF916230360CF
:103880004FF0FF3010BD00002DE9F3411E46836864
:1038900004460D469046089F3BB10E4B0AAA099973
:1038A0001B680192D86831F0A7FA2FB12046FFF7C4
:1038B000CFFF2046FFF7D9FF6B683146284680339B
:1038C0006B60236B9B69984706F80080013002B05B
:1038D000BDE8F081C00E002410B520B1036BBDE837
:1038E00010409B6A18472BF0B7F9162303604FF07E
:1038F000FF3010BD4FF0FF33C0E90033002330B577
:10390000C0E9023300240025034BC0E9044583616C
:103910008362C0E9084530BD20A1070010B520B181
:10392000036BBDE810401B6918472BF095F916236F
:1039300003604FF0FF3010BD10B520B1036BBDE840
:1039400010409B6B18472BF087F9162303604FF04C
:10395000FF3010BD10B1036BDB6B184770470000E0
:103960002DE9F041036B0F46044611461B6A3846A9
:1039700098470646236B3246394620465B6A98478D
:103980000546013018D1E368990715D52BF064F985
:10399000D0F800802BF060F90368092B1ED1204677
:1039A000FFF7D8FF2046FFF753FF2046FFF7C4FF7D
:1039B0002BF052F9C0F80080E3689A0701D56B1C20
:1039C000D8D0002D07DDAE4205D02BF045F94FF0E1
:1039D000FF350B4B03602846BDE8F0812BF03CF926
:1039E0000368682BDBD02BF037F90368202BD6D087
:1039F0002046FFF72DFF2046FFF737FFD8E700BF2F
:103A00005B42B2062DE9F04FD1B088461E4607460C
:103A10000B9248B92BF020F916234FF0FF3B0360BF
:103A2000584651B0BDE8F08F026B40465368D269EA
:103A3000CD1811F803900693697815F801BCAC789D
:103A4000CDE90CB904EB01240BA9904709F1FF3231
:103A5000A4B20E90069B162A00F25F82DFE812F0F5
:103A60001700170083008300CC00FF00AF015D0248
:103A70005D025D025D025D025D025D0210014701B3
:103A800098015D025D025D025D02B301CE01E9783D
:103A9000B9F1020F95F804A00AEB012AD6E908381B
:103AA0000AF1FF310DBFAD4B9846AD4BD6E9022070
:103AB00018BFD6E90020B1F5FA6F0FAE11D34FF45D
:103AC000FA62CDF808A0CDE90332A64B0193012399
:103AD0000093334603220CA93846FFF7D5FE04466F
:103AE00029E0251A04D40AEB0509914509DD54445F
:103AF000CDE902439C4B01930023009333460222FD
:103B0000A8E03B6B31460CA89B6998471AF0070365
:103B100000F1010418BF012303EBDA0A06F800A044
:103B200008EB050000221146A0EB080399450DDCC7
:103B300009B132550134BBF1000F3FF471AF224699
:103B40000FA93846FFF70CFF834669E710F8013BE1
:103B5000072903FA01F342EA030202D13255013484
:103B6000E0E70131E0E7B9F1040FE8780DF13C0935
:103B7000D6E90A830CBFD6E90412D6E906122E79DB
:103B800014BF9846794B06EB002618BF784B701E81
:103B90007C2809D97D220296CDE90332714B01932D
:103BA000012300934B4695E7A51A04D406EB050ABA
:103BB0008A4508DD3444CDE902436B4B0193002371
:103BC00000934B469BE73B6B49460CA876009B69EC
:103BD0009847441C09F80060AA45ACDD38F8153058
:103BE0001B0A09F80430023438F81520013509EBB6
:103BF000040303F8012CEFE77368E21A02D4336878
:103C000093420BDC5B4B02940193002300930FABB8
:103C100002220CA93846FFF737FE60E7E9782B79D6
:103C200003EB0123B3F57F4F00D05BB90033316A5A
:103C300018BF01238B540B9C41460FA822462CF041
:103C4000B9FB78E7CDE902344B4B01930023009395
:103C50000FAB03220CA93846FFF716FE3FE7F369C6
:103C6000E31A02D4B2699A4202DC0294434BCBE7D6
:103C7000E8782A79F16A02EB002221F81320DAE7CA
:103C8000E9780DF13C092A7902EB0122511EB1F5C8
:103C9000F66F03D26979B2EBC10F09DD4FF4F66319
:103CA000CDE90223364B0193012300934B46D0E725
:103CB0007168611A04D455183068854207DD1444D0
:103CC000304B02940193002300934B46A0E7063348
:103CD000306A4344FFF745FB3B6B49460CA89B69A0
:103CE000984758F8003049F80030041D23E7E97878
:103CF0002A7902EB0122511E7A2903D86979B2EBA5
:103D0000C10F06DD7B23CDE902231F4B0193012365
:103D10009DE7F069201A14D402EB000CB1698C45C0
:103D20000EDCC8EB4002D31A84450DDC0FAC3B6BB4
:103D30000CA89B692146984758F800302350D4E7D7
:103D400014440294114B5FE7AC790130E979F26ACF
:103D500001EB04212A440235D152E5E73E750708FC
:103D600034750708727507089A7507085D750708A6
:103D70004E750708BC750708E57507082376070820
:103D80005176070885760708AF760708E8760708B2
:103D90000FAD3B6B0CA89B6929469847B4222B18A2
:103DA000C11C5A70FF226C189A70604A13686B50DD
:103DB000536863600A2300F10B042B54BBE62AF01E
:103DC0004BFF6D2329E6F169611A3FF54EAFB369E8
:103DD0008B427FF74AAFEA782B796C79F06A03EB74
:103DE0000223AA799BB202EB042230F8114022EAA6
:103DF00003022340134320F811301CE7EA780DF149
:103E00003C0A95F80490287A09EB0229EA7900EB3C
:103E10000220421E782A09D8B9F1000F06D0B9F164
:103E20007D0F03DC6A7AB2EB400F10D079237D223C
:103E30000CA9CDE904323E4B032201930123CDE9C5
:103E40000209009338465346FFF71EFD47E66A799C
:103E5000A446A979D6F81CE001EB02218AB2B4EBA2
:103E60000E010792A2EB0E0206910DD44944D6F83A
:103E700018C06145089105DC002A03DB81188C45D8
:103E800009910FDA04EB090C002AA2BF079B1B184B
:103E90000793079BCDE902C3264B019300230093B0
:103EA00053462CE6396B0CA80A924FEA49098C69F3
:103EB00051460793A0470A9A441C079BC8EB420847
:103EC0000AF80090A8EB03030999914218DC069BBD
:103ED000C0EB43000138089B069A93427FF72BAE54
:103EE0000219F16A8B5A1B0A0AF8043002348A5A02
:103EF0000AEB040303F8012C069B01330693EAE75F
:103F000095F80AE0013295F80BC0F16A0CEB0E2C23
:103F10002944023521F803C0D6E7074B0122CDF82A
:103F2000089001930FAB009273E600BF1777070864
:103F3000207707086C770708BD770708036B2DE922
:103F4000F04F5C6887B005460F460134914692B148
:103F50000DF1080AD0E90423CDE902238369049313
:103F60000026B0462B6B44B91B6B424639462846A7
:103F70009847834623E09246F2E7D3F844B052468E
:103F8000234669462846D847B0F1FF3F834626D1ED
:103F9000EB68980702D44FF0FF3B10E02AF05CFE7C
:103FA00004682AF059FE0368742B0CD12846FFF7E9
:103FB0004FFC2846FFF759FC2AF04EFE0460584695
:103FC00007B0BDE8F08F2AF047FE0368092BF3D154
:103FD0002846FFF7BFFC2846FFF7AEFCECE72B6B4B
:103FE000224607EB08012846DB6A9847C0B92AF049
:103FF00033FE68230360EB689A07CCD52AF02CFEC9
:104000000368682B17D12AF027FE04682846FFF7BB
:10401000A1FC2846FFF790FC2AF01EFE0460BAE7D8
:10402000411CE8D0241A804457D1296B76B1012E67
:104030002CD0022696E72AF00FFE03686F2BE2D001
:104040002AF00AFE0368092BA5D1DCE74B68FB5C6C
:10405000B9F1000F0CD1062B52DDA3F10F02012A9A
:1040600051D9162B52D0172B10D10126092437E035
:10407000053B0126112B07D806FA03F340F603424D
:1040800013423ED19B0341D4344629E04B68FA5C8D
:10409000B9F1000F17D10F2A03D3102A0DD9172A0F
:1040A0000ED08B681C44CB6808EB04029A4213DDE7
:1040B0002AF0D2FD174B03606DE73B445C79F0E7D3
:1040C0003B445C7AEDE7042A03DD112A01D0172A6C
:1040D000E7D13B445C78E4E70226002C7FF742AF4F
:1040E000AB6AD5E90801012871F1000202DA002B60
:1040F0007FF738AF04930DF1080ACDE9020131E7EB
:1041000001260424ECE701260524E9E7012606241C
:10411000E6E700BF5B42B20610B1036B9B6C184729
:104120007047002070470020704730B5A1F110049F
:10413000002500F00F02CD7302390009D3B2092A1D
:10414000CCBF373330330B748C42F2D130BD2DE904
:10415000FF470024061D05468A469046994600946E
:1041600023464FF0FF32B1213046CDE9014413F030
:10417000B9FA29682846DDE90C23CDE90023424637
:104180004F694B465146B847009423464FF0FF32E3
:10419000C1213046CDE9014413F0A4FA204604B011
:1041A000BDE8F0872DE9D04F9B4603689246044650
:1041B0009B6ADDE90889984702460B4650465946F6
:1041C00029F01AFC134302D00020BDE8D08F2368E9
:1041D00020469B6A984702460B464046494629F0CE
:1041E0000BFC1343F0D11AEB0806236820464BEB77
:1041F00009079B6B9847B94208BFB0422CBF01200A
:104200000020E2E701682DE9F04114461D46096BE4
:104210000646884702460B462046294629F0ECFB15
:10422000134302D00020BDE8F081DDE906233046CB
:10423000A71845EB030817F1FF323368196B48F1F3
:10424000FF33884702460B463846414629F0D4FBE7
:104250001343E7D1336830469B6B9847414508BF0D
:10426000B8422CBF01200020DDE72DE9D04F9B464E
:104270000368924604465B6ADDE90889984702466E
:104280000B465046594629F0B7FB134302D0002095
:10429000BDE8D08F236820465B6A984702460B46EC
:1042A0004046494629F0A8FB1343F0D11AEB080613
:1042B000236820464BEB09079B6B9847B94208BF20
:1042C000B0422CBF01200020E2E7C220704700006E
:1042D000244830B5037887B0BFF35B8F13F0010437
:1042E0001CD117F0F5FEC8B11F4B66223B211F48B9
:1042F000CDE903435A23CDE901323D233C2200930B
:10430000572319F0C7FE194C194B1648236017F0B4
:1043100001FF184A2046184917F0CAFE13481AF040
:10432000F3F8164D1A22002329461048CDE9002340
:1043300000230022FFF70BFF2B780446B52B04D196
:104340000F4B01221D600F4B1A70084819F038FFFF
:10435000B4FA84F0400907B030BD024818F0E2F822
:1043600028F0A8FFD42D0024005A6202E02D00247A
:10437000EC7707080000002435450408E82F0024E6
:104380000C000024D82D002410B504461AF058FD66
:104390002146FFF7CAFE1AF059FD04F11001FFF79C
:1043A000C4FE1AF059FD04F12001FFF7BEFE3020D3
:1043B00010BD000008B54DF659720021074820F0E5
:1043C000E0FFBFF34F8F0649064BCA6802F4E06274
:1043D0001343CB60BFF34F8F00BFFDE7B02D002428
:1043E00000ED00E00400FA0510B50446FCF7BAFD44
:1043F000204610BD064B10B504460360806A08B124
:1044000016F07AFC201DFFF7EFFF204610BD00BF1D
:10441000008C070800B5C3B01622172103A812F0BC
:1044200093FE4FF4A17302AA1021ADF808300023C7
:1044300003A80093022312F0B3FD03A8FFF7DAFFED
:1044400043B05DF804FB03A8FFF7D4FF28F032FF68
:104450001D4B01211D4AA62070B51A6002F070F9AB
:104460000121A62002F0ECF9FFF7D4FF184B43F22C
:10447000D2021A60FFF72CFF164B1B7833B1164B94
:104480001B689A8840F209439A421BD8134B9B6DD4
:1044900003F46043B3F5004F14D002F0A5F8104DBB
:1044A000044602F0B3F8064602F0B0F8801BA842BA
:1044B000FAD902F099F8001B642803D0BDE87040D7
:1044C00025F076BE70BD00BFB02D0024004000581E
:1044D00000400052D82D00240C0000240044025853
:1044E0009F86010010B50446FFF784FFFC2120469B
:1044F00018F064F8204610BD38B5074B0546044651
:1045000045F8BC3B19F05CFE284618F07DFA201DEA
:1045100013F028F9204638BD80AA070810B50446D4
:10452000FFF7EAFF4FF40271204618F047F82046E3
:1045300010BD0000034B10B504460360FFF7DCFF1D
:10454000204610BDEC77070810B50446FFF7F2FFD0
:104550004FF40271204618F031F8204610BD036870
:104560000868184708B5011DFFF7F9FF08BD0000EE
:10457000044A0346C260002203C99A6083E803002C
:10458000704700BF3C78070813B50446CDE9001218
:104590006946FFF7EDFF204602B010BD10B5044696
:1045A000FFF7F2FF204610BD08B5FFF7DBFF08BD9F
:1045B00008B5FFF7F9FF08BD70B590F8383105462A
:1045C0001446F3B90368DB69984704F4706304F098
:1045D0000F02B3F5407F04F0F0030CBF0721082160
:1045E000302B0CBF02230123012A08D0901E424227
:1045F0004241A869BDE87040006813F07DBB02220B
:10460000F7E770BD10B590F8383104462BB9A369AF
:10461000186813F0B5FB0028F9D010BD38B590F834
:1046200038510446A5B983695BB1186848B103687D
:10463000DB689847A36904211D60A06917F0BEFFDD
:10464000A5610023C4F82831C4F82C31C4F83031F6
:1046500038BD13B590F8383104466BBBA3691868B0
:1046600013F062FB40B317F043F9A36901220DF187
:104670000701186803685B699847D4F83031B3F5CF
:10468000807F16D0D4F83031B3F5807F11D0D4F8C4
:1046900028319DF80720234483F82820D4F82831B6
:1046A0000133DBB2C4F82831D4F830310133C4F817
:1046B000303117F033F9D1E702B010BD08B590F8EA
:1046C00038313BB1012001F0ADFF0648BDE808409C
:1046D00001F053BA82691AB11368003318BF01237D
:1046E000184608BD883A002470B504460D4601F00E
:1046F00044FA30B12368294620461B6CBDE870405F
:10470000184770BDA0F59860EEE7000013B590F86B
:10471000383104468DF807102BB1C9B20B48FFF7AA
:10472000E3FF02B010BDA369186813F029FB00284D
:10473000F9D0A36901220DF10701186803681B690C
:104740009847013018BF0120EBE700BF883A0024EA
:104750002DE9F04107468846164601F00EFA80B171
:104760000024A6420ED9351B08EB04013846B5F5E6
:10477000007F28BF4FF400752A462C4400F044FF08
:10478000EFE704462046BDE8F081A0F59860DFE73A
:1047900070B590F8383105460E4614462BB10F48D7
:1047A000FFF7D6FF0446204670BDAB69186813F0CA
:1047B000E7FA0028F9D0AB6901211868D0F88830F1
:1047C00088301B6B9847AB692246314618680368EE
:1047D0001B699847013008BF0024E4E7883A0024A9
:1047E00030B50446C3B001F0B3F90546D4F8D83566
:1047F000C3F58073984203DDD4F8D855C5F58075AC
:104800002A4601AB02A9204600F0F5FF019902AB50
:1048100000226D1A1D44D4F8D835B3F5807F19D025
:104820008A4217D0D4F8D835B3F5807F10D0D4F8A9
:10483000D035A85C234483F8D004D4F8D0350133B4
:10484000DBB2C4F8D035D4F8D8350133C4F8D83544
:104850000132E0E743B030BD38B5044600F0BCFBA0
:104860002046FFF7BDFFD4F8D855204600F0BCFB2A
:10487000284638BDA0F59860EEE7000010B590F826
:10488000383104462BB10648FFF7E6FF04462046C0
:1048900010BD17F02DF8D4F8304117F03FF8F6E7C7
:1048A000883A002438B5044600F096FB2046FFF70E
:1048B00097FFD4F8D8354BB1D4F8D435234493F8C6
:1048C000D054204600F090FB284638BD4FF0FF350D
:1048D000F7E7A0F59860E5E710B590F838310446A1
:1048E0002BB10B48FFF7DEFF0446204610BD16F043
:1048F000FFFFD4F830313BB1D4F82C01044494F8D4
:10490000284017F00BF8F0E74FF0FF34F9E700BF4D
:10491000883A002438B5044600F05EFB2046FFF7D5
:104920005FFFD4F8D835A3B1D4F8D435234493F835
:10493000D054D4F8D4350133DBB2C4F8D435D4F82C
:10494000D835013BC4F8D835204600F04DFB284649
:1049500038BD4FF0FF35F7E7A0F59860DAE70000C3
:1049600010B590F8383104462BB11148FFF7D2FF4B
:104970000446204610BD16F0BBFFD4F830319BB181
:10498000D4F82C31234493F82800D4F82C31013387
:10499000DBB2C4F82C31D4F83031013BC4F83031EB
:1049A000044616F0BBFFE4E74FF0FF34F9E700BF21
:1049B000883A002408B54FF4807200212BF0F8FDEE
:1049C0000022C0F80021C0F80421C0F8082108BD69
:1049D00010B4D0E9003409686210E4075DF8044BB4
:1049E00001EB020044BF8A58D358184701460430EF
:1049F00008B5FFF7EDFF08BD034A0346C26007C9CB
:104A000083E80700704700BF4878070810B586B0F4
:104A100004460391684606A980E80C0001E90C00F1
:104A2000204603A9FFF7E8FF204606B010BD37B5C2
:104A30006C46054684E80C0094E80C00FFF7E6FF9E
:104A4000284603B030BD000070B590F8383186B00C
:104A500004460E46002B3BD1856925B9042017F08A
:104A600079FDA0610560A369186850BB8C2017F020
:104A700071FD3346B4F922200546B4F9201013F035
:104A800067FCA3691D60B4F92420531C06D0A069FB
:104A90000321B4F92630006813F06AFCA3691D688D
:104AA000B5B1114B0026214602A800936B46019632
:104AB0000CCBFFF7BCFF324602A9284613F0CEF913
:104AC00003E0314613F005F9DDE702A8FCF74FFAE1
:104AD00006B070BD8C21284617F070FD28F0EAFB67
:104AE00002A8FCF744FAF9E75346040808B5FFF7B3
:104AF0007DFF08BD08B5FFF7F9FF08BD2DE9F843B4
:104B000000242D4D4FF47A782C4F202605F12800F3
:104B10002F60EC61C5E90148C5E90564FFF74AFF6C
:104B200001230E2085F8383101F044FD244D8146E3
:104B30000D2001F03FFDA5F820904FF6FF79688425
:104B400005F128002F60EC61A5F82490A5F82690C7
:104B5000C5E90148C5E90564FFF72CFF85F8384130
:104B60000F23184D2B84562305F128002F606B84EA
:104B70005823EC61AB845923C5E90148EB84C5E9AE
:104B80000564FFF717FF85F8384198230E4D2B84F5
:104B9000992305F128002F60EC616B84A5F824901F
:104BA000A5F82690C5E90148C5E90564FFF702FFAD
:104BB00085F83841BDE8F883B83300245C780708ED
:104BC00004300024403100247C320024002070474F
:104BD0007047704710B5D0F88C452CB1236820463B
:104BE000DB6A9847A468F8E710BD38B50D46D0F8E1
:104BF0008C4534B1236820462946DB689847A46871
:104C0000F7E738BD004870471C790708054B10B519
:104C10000446036014F021FE204614F02FFF2046C6
:104C200010BD00BF9C78070810B50446FFF7EEFFE3
:104C30004FF4B261204617F0C1FC204610BDF7B515
:104C4000002305460E46D0F88C45A4B123683146B2
:104C50000DF1030220461F6901ABB8479DF8031010
:104C60000346042905D0019A284614F005F903B03B
:104C7000F0BDA468E9E7019A9DF80310F4E770B568
:104C800005460E4622B10021BDE8704013F000BF7A
:104C9000D0F88C455CB123680022314620465B6920
:104CA000984710B101212846EEE7A468F2E72146B3
:104CB000F9E770B50E460546D0F88C4500213CB1A9
:104CC0002368314620469B699847A4680146F6E769
:104CD0002846BDE8704013F0CFBFF8B505460E4634
:104CE0001746D0F88C453CB1236820463A463146F9
:104CF000DB699847A468F6E728460121BDE8F8403B
:104D000014F018B870B5002186B0044614F0FFF90D
:104D100000234FF48975A188EF26ADF8063023896A
:104D2000ADF8045002258DF810301B0AE2888DF88A
:104D3000113040F201238DF80750ADF8123040F2E7
:104D400003138DF809500125ADF8143004F10A035E
:104D50008DF8086005AE8DF80A501C468DF80C10D1
:104D600001AD090A8DF80E20120A8DF80B008DF89E
:104D70000D108DF80F202A46083303CAB24243F8BB
:104D8000080C43F8041C1546F5D1128820461A80F9
:104D900006B070BDF8B5002406460D4627463046DD
:104DA0002CF0AEF9A04207D9335D05F8143005EBBD
:104DB000440301345F70F2E7400000F0FE00F8BDEC
:104DC00038B50446D0F88C5535B12B6828465B6A57
:104DD000984710B9AD68F7E7284640F2023304F26D
:104DE0004A51A4F84835FFF7D5FF94F848351844E0
:104DF00084F8480504F5A96038BD000040F202338C
:104E000000F20A5110B50446A0F808350548FFF72E
:104E1000C1FF94F80835184484F8080504F5A1602A
:104E200010BD00BF8878070840F2023310B5044671
:104E3000A0F8C83400F2CA40FFF7A6FA94F8C834C4
:104E4000184484F8C80404F5996010BD2DE9FF41A9
:104E500000231D4A044600F54E788DF80A300925D6
:104E600090F888350192FA228DF8083001238DF8E8
:104E70000C208DF80930C0238DF80B3001AB03CB2B
:104E8000C4F83803C8F8041088F80820D4F88C65F2
:104E90008EB13368002130469B689847478805F5F6
:104EA0004E7300F10901093FE0183A463D442BF0EA
:104EB00081FAB668ECE784F83A5340462D1284F83C
:104EC0003B5304B0BDE8F0810902FFFF73B504460F
:104ED0000D46164623F0D0FB4FF4807301462A4658
:104EE00020460093334614F085FD024B2046236094
:104EF00002B070BD9C78070810B5D0F88C35044618
:104F0000A3B9C0F88C1594F8883508464A790B7116
:104F100094F88835134484F888350B689B6A984761
:104F2000238918442081012010BD13469A68002A65
:104F3000FBD19960E7E71FB5044614F0E3F801469A
:104F4000684613F0DDFA4021684613F04BFBD4F8B5
:104F50008C4534B12368694620461B6A9847A4688B
:104F6000F7E7684613F0D3FA04B010BD684613F0B3
:104F7000CEFA28F09FF910B50446FFF7DCFF204673
:104F8000BDE8104014F0A5B80F4808B50378BFF38A
:104F90005B8FDB0711D417F09BF870B140F25B22F6
:104FA00042F241310948FFF791FF074817F0B2F884
:104FB000074A0849054817F07BF8044808BD02482D
:104FC00017F0B0FA28F076F9F4340024F83400240D
:104FD000000000240D4C040810B5FFF7D5FF03684E
:104FE000BDE810405B6F184710B5FFF7CDFF0368B1
:104FF000BDE810409B6F184710B5FFF7C5FF036869
:10500000BDE81040DB6F184713F022BC13F036BC2C
:1050100013F00EBC704770477047436A93F87800EE
:105020007047D0F8A40470470120704700487047CB
:10503000887A07082DE9F04794B004460F464B22C2
:10504000002101A82BF0B4FA2679D4F8A434751CF9
:1050500094F80E90002B94F80C80EDB294F80DE0CB
:1050600014BF05200020002F40F0938040F2092358
:1050700009218DF81D0042F20540ADF804304FF4CF
:1050800081738DF815100121ADF808308023ADF83B
:105090001E0010208DF80B3032234FF0040A242715
:1050A0008DF80C3008234FF0030C4B228DF80D3097
:1050B0000B238DF819101D348DF80E3040F20223A9
:1050C0008DF81C10ADF8103002238DF8210005205A
:1050D0008DF822108DF825108DF8271006218DF8F7
:1050E00006208DF80F608DF812308DF817608DF85E
:1050F0001A308DF81B308DF823008DF826C08DF8FE
:105100002A308DF82B108DF82C008DF816A08DF814
:1051100024708DF828A08DF829708DF82D708DF8E9
:105120002E1007218DF82F6041F202068DF8311004
:105130008DF8411040F207518DF83050ADF83660CF
:1051400040F209468DF83A5040F602258DF83200BB
:105150008DF842002046ADF848100DEB0A018DF89D
:1051600033908DF834C0ADF83860ADF83C508DF810
:1051700043808DF844308DF846308DF84AE08DF844
:105180004B308DF84D302BF015F9204614B0BDE8AA
:10519000F0870020FAE700000A4B10B504460360D0
:1051A000FFF7F2FE14F059FB04F5247013F0B4FA83
:1051B00004F17C0013F0B0FA04F1700013F0ACFAC3
:1051C000204610BD487A070810B50446FFF7E4FFF3
:1051D0004FF49561204617F0F1F9204610BDFFF716
:1051E0000BBF0000034B10B50446036013F050F9E9
:1051F000204610BD6479070810B50446FFF7F2FF9A
:105200002821204617F0DAF9204610BD034B10B5CF
:105210000446036013F03CF9204610BD34790708BA
:1052200010B50446FFF7F2FF3421204617F0C6F907
:10523000204610BD034B10B50446036013F028F957
:10524000204610BD4C79070810B50446FFF7F2FF61
:105250003821204617F0B2F9204610BD38B51E4B54
:105260000D4604464FF400721968C0F80F10998873
:105270009B79A0F8131002214375284613F0A8F972
:105280004FF4007220730221284613F0A6F94FF460
:10529000007260730321284613F09AF9A073284620
:1052A00013F036F920B9AF220C490D4816F028FA50
:1052B00004F185020023C4F8882204F2992284F8BC
:1052C000783084F88430C4F88C3284F89832C4F88A
:1052D0009C24C4F8A03438BD80790708237A0708D5
:1052E0002E7A07082DE9F34104460E461546FFF7CE
:1052F00083FEF28823799A4237D1002D35D1777811
:10530000012F2ED1F378202B27D13289072A24D1DF
:1053100004F10F0804F11605404629462BF018F851
:10532000D0B1D4F81630C4F80F30638B207CE17B09
:10533000A4F8133001EB0021E57C607C237F01EBB6
:1053400000410095A07C2568637501EB0061237D19
:105350002046627D6D6BA8473D46F378212B08BF40
:105360000125284602B0BDE8F0810025F9E710B517
:105370000446FFF741FEFFF707FE217B14F00AF910
:1053800004F1850304F17C00C4F888320023C4F8DA
:105390008C3284F8843013F074F994F884302BB98B
:1053A00023682046DB6BBDE81040184710BD0000A5
:1053B00070B50446FFF720FED4F8A0542DB140F29A
:1053C000DD120F490F4816F09BF904F29923C4F837
:1053D0009C34FFF7D9FD617B14F03AF884F89852B9
:1053E000C4F8A00404F5247013F04BF994F8983233
:1053F0002BB9236820469B6BBDE87040184770BDF1
:10540000237A07088C79070802232DE9F0414371BC
:1054100000230446054683609046144B04F17C0645
:1054200045F8703B284613F01FF9304613F01CF97D
:1054300004F52477384613F017F9C4F8A484FFF76D
:10544000A3FD2146FFF758FD0CE0384613F064F940
:10545000304613F061F9284613F05EF927F02AFF71
:10546000F6E7F8E72046BDE8F08100BF487A070874
:1054700070B504460D46FFF7BFFD84F87850002D47
:105480003ED194F8843033B1FFF77EFD217B13F0D9
:1054900059FE84F8845004F1850304F17C0600254C
:1054A0003046C4F88832C4F88C5213F0EAF830461B
:1054B00013F0E0F828B94FF4A2721449144816F01A
:1054C0001FF994F8983233B1FFF75EFD217B13F09A
:1054D00039FE84F8985204F2992304F52475C4F82F
:1054E0009C3400232846C4F8A03413F0CAF8284698
:1054F00013F0C0F820B94FF4A77204490548DEE75D
:1055000004F17000BDE8704013F0BBB8237A0708BF
:105510009A790708AB79070810B50446FFF76CFDC8
:1055200000212046BDE81040FFF7A2BF38B50D4668
:105530000446FFF761FD042D05D020460021BDE89B
:105540003840FFF795BF38BDF8B5164604460D46FE
:105550001F46FFF751FD0423EA88337023799A42EE
:1055600025D16978012922D1EA78212A08D0222A76
:105570000BD0202A4FF000001BD13070163401E010
:105580000F34317007203C60F8BDAB88204613F023
:10559000010308BF1946FFF76BFFAB8803F0010357
:1055A000E366AB8803F00203A36602233370002096
:1055B000EAE703233370E7E710B58AB00446FFF744
:1055C0000BFD684612F054FF0D4B694604F1700064
:1055D0000093099413F06DF82046FFF705FD094B81
:1055E000002168461A6812F009FF6846FFF7FAFDC5
:1055F0000AB010BD6846FFF7F5FD27F05BFE00BF5F
:10560000647907088879070870B58EB004460E469D
:105610001546FFF7E1FC01A812F02AFF114B01A982
:1056200004F17C00019300230C958DF83430CDE912
:105630000A4613F03EF82046FFF7D6FC0A4B00213D
:1056400001A81A6812F0DAFE04E001A8FFF7DEFDF7
:1056500027F030FE9DF8344001A8FFF7D7FD204623
:105660000EB070BD347907088879070810B5044674
:10567000FFF7C2FC94F884307BB9D4F88C3263B164
:10568000FFF782FCD4F88C3204F18502217B13F001
:105690001FFF10B1012384F8843010BD2DE9F843B9
:1056A0001E460446894690469DF82070FFF794FCFC
:1056B0000023336094F87830E3B194F88430CBB9A8
:1056C000D4F88C52C5F50075454528BF4546B8F15C
:1056D000000F05D02A464946D4F888022AF06AFE0F
:1056E000D4F88C322B44C4F88C32356017B1204684
:1056F000FFF7BCFF2046BDE8F843FFF775BCF0B5E7
:105700000446406A85B0012690F878502DB984F897
:1057100030503546284605B0F0BD04AB0027D4E92B
:105720000A1243F8047D0096FFF7B8FF0399E36A75
:10573000A26A5B1A0A44E362A26213B984F8306079
:10574000E8E7606A3D46FFF791FFE3E72DE9F043A4
:105750001C4691B0054689469046FFF73DFC002C5B
:105760004FF0000602A806BF01AC01270027266003
:1057700012F07EFE134B02A905F5247002938DF8FA
:105780003C708DF83D60CDE90B59CDE90D8412F0E8
:1057900090FF2846FFF728FC0B4B314602A81A68F9
:1057A00012F02CFE04E002A8FFF744FD27F082FD72
:1057B0009DF83D4002A8FFF73DFD204611B0BDE831
:1057C000F08300BF4C7907088879070810B5D0F836
:1057D000A034044673B990F898325BB9FFF7D4FB54
:1057E0004FF4007304F29922617B13F0D3FD01237F
:1057F00084F8983210BD70B504461E460023084652
:10580000336094F87830EBB194F89832D3B9D4F887
:10581000A054D4F89C14954228BF15462A462AF075
:10582000C9FD3560D4F89C34D4F8A0242B44551B12
:10583000C4F89C34C4F8A05425B92046BDE8704093
:10584000FFF7C4BF70BD37B50446406A90F8785082
:105850002DB984F835500125284603B030BD02AB80
:10586000002243F8042DD4E90A12FFF7C4FF01997E
:10587000A26A0A44A262226B13680B441360019966
:10588000E36A5B1A94F83410E36209B9126802B94A
:105890001BB9012384F83530DEE7606A0025FFF785
:1058A00095FFD9E710B50446FBF7AEFF204610BDC3
:1058B00010B4D0E9003409686210E4075DF8044BC5
:1058C00001EB020044BF8A58D35818470146043000
:1058D00008B5FFF7EDFF08BD034A0346C26007C9DC
:1058E00083E80700704700BF7479070810B586B0D9
:1058F00004460391684606A980E80C0001E90C0003
:10590000204603A9FFF7E8FF204606B010BD37B5D3
:105910006C46054684E80C0094E80C00FFF7E6FFAF
:10592000284603B030BD0000F0B58BB00546FFF748
:1059300063FB06ACFFF728FBAF7B06460021204641
:10594000FFF7B0FF009403234FF40072394630464E
:1059500013F0E6FF2046FBF70AFBFFF715FB234B8E
:1059600006462F7B0293002329462046039302AB71
:105970000CCBFFF7CCFF009402234FF400723946A2
:10598000304613F0CDFF2046FBF7F1FAFFF7FCFAA3
:10599000174B06466F7B0493002329462046059348
:1059A00004AB0CCBFFF7B3FF009402234FF400725B
:1059B0003946304613F0B4FF06E02046FBF7D7FA2D
:1059C00027F078FCF9E7F8E72046FBF7D0FAFFF775
:1059D000DBFA4FF40073D5F89C24697B13F0DAFCF2
:1059E000012085F898020BB0F0BD00BF6F5304088A
:1059F000B153040808B5FFF769FF08BD08B5FFF704
:105A0000F9FF08BD6FF01500704700290CBF6FF05B
:105A1000180000207047012070476FF01500704794
:105A20006FF015007047112070477047704770473E
:105A300003689B6C1847A0F59860F9E770477047BA
:105A40007047704710B50446012000F0EBFD94F854
:105A5000780010BDA0F59860F4E7000038B54FF06D
:105A6000FF320123FF210B4816F04BFF0A4D00F0D7
:105A7000BBFD044695F878301BB1012000F0D2FD43
:105A8000F8E700F0B1FD001BC728F6D9BDE83840A3
:105A9000FEF790BCC0400024883A002407B502AB52
:105AA000012243F8041D1946FFF7AEFD18B1019815
:105AB00003B05DF804FB4FF0FF30F9E7A0F5956007
:105AC000FFF7ECBF07B5002302A9012201F8013D51
:105AD000FFF73CFE20B19DF8070003B05DF804FB22
:105AE0004FF0FF30F9E7A0F59560FFF7EBBF2DE928
:105AF000F8430446884617461E46089DFFF77CFA81
:105B0000D4F8F095B9F1000F04D02B46324639464F
:105B10004046C847C4F8E085C4F8E475C4F8E865B1
:105B2000C4F8EC55BDE8F883B0F5966F03D10121B8
:105B3000014816F0C5BE7047C04000240068704799
:105B40000C30704708B5FFF7FBFF0023036008BD6A
:105B500038B50546FFF740FA95F898325BB9D5F8A5
:105B6000A044B4F5007F28BF4FF400742846FFF727
:105B70003BFA204638BD0024F8E790F878007047DB
:105B8000114B03F1780270B503600446C0F8A824F5
:105B900000F2F45603F1D80200F23465E833C0F89D
:105BA000AC24C0F8C034AE4204D0103D2846FBF708
:105BB000DEF9F8E704F5956015F024FA2046FFF7C2
:105BC000EBFA204670BD00BF607B0708A0F595602A
:105BD000FFF7D6BFA0F2AC40FFF7D2BF10B5044626
:105BE000FFF7CEFF4FF4C761204616F0E7FC2046D2
:105BF00010BDA0F2AC40FFF7F1BFA0F59560FFF734
:105C0000EDBF00002DE9F74304461E4688461546C1
:105C100022F032FDBDF82C3004F595670146019362
:105C20002A46BDF82830204600933346FFF7ECFBA8
:105C30000021384615F0BCF94FF47A73002504F2C0
:105C4000F45904F59A60C4F8C8342946204B4E46EE
:105C5000C4F8C45403F178022360C4F8A82403F103
:105C6000D802E833C4F8AC244FF48072C4F8C034CE
:105C70002AF09EFCC4F8D055C4F8D455C4F8D855C1
:105C800004F2346530461036FBF7BEFDB542F9D15B
:105C90000023C4F83436C4F8F035B8F1000F13D03F
:105CA0002046FFF789FC0FE04D4504D0103D284603
:105CB000FBF75DF9F8E7384615F0A4F92046FFF741
:105CC0006BFA27F0F7FAF9E7204603B0BDE8F08356
:105CD000607B0708884238B5044606D00D46FBF7BE
:105CE00041F920462946FDF708F8204638BD08B599
:105CF000FFF726FF0068003018BF012008BD000034
:105D000010B50446FFF7F3FF28B940F20222064916
:105D1000064815F0F5FCE068FFF710FF0346204643
:105D2000BDE81040184700BF417B07084C7B0708BF
:105D3000F8B506460025FFF75FF906F2F454D6F8E9
:105D40003436AB420AD920462746FFF7D0FF10343D
:105D500020B138460135FFF7D3FFF0E7F8BD00006A
:105D6000044BC36003460A6843F8042B00224260D8
:105D70005A607047AC7A070813B50446019121B9FF
:105D8000FFF7E0FE204602B010BD01A9FFF7E8FFD3
:105D9000F8E710B4D0E9003409686210E4075DF850
:105DA000044B01EB020044BF8A58D3581847014600
:105DB000043008B5FFF7EDFF08BD0000034A0346B5
:105DC000C26007C983E80700704700BFA07A0708D0
:105DD00010B586B004460391684606A980E80C0019
:105DE00001E90C00204603A9FFF7E8FF204606B0B2
:105DF00010BD37B56C46054684E80C0094E80C00ED
:105E0000FFF7E6FF284603B030BD00002DE9F04162
:105E100088B00446FFF7E0F8384B2046C4F8F03568
:105E2000FFF7E2F8364B04A82146029300230393C0
:105E300002AB0CCBFFF7DDFF2046FFF7CDF8D4F81F
:105E40003406032803D92046FFF7CEF80AE0431CA6
:105E500004EB001004A9C4F8343600F2F450FFF744
:105E600039FFF0E704A8FBF782F8BC2016F072FBBC
:105E700005460646234B05F1400746F8043B3046ED
:105E8000FBF7C2FC0021384616F0E0FD05F154088E
:105E9000404616F079FD1C4B4FF4807218212846BD
:105EA0000093002316F062FE184904A8C4F8DC55DC
:105EB000FFF762FF04A9284616F022FF10E04046D3
:105EC00016F0A2FD384616F000FE3046FBF74FF8FC
:105ED000BC21284616F072FB27F0ECF9F2E7F4E754
:105EE00004A8FBF744F82046FEF77AFC08B0BDE8AA
:105EF000F08104A8FBF73BF8EEE7FAE7295B04081A
:105F0000E1470408509E0708B87A07085D5A04085C
:105F1000A0F59860FFF77ABF0368184708B5FFF748
:105F2000FBFF08BD08B5FFF742FF08BD08B5FFF746
:105F3000F9FF08BD37B50F4C0F4D204616F0B0FCE9
:105F40002A460E49204616F0B3F842F21203012207
:105F50000B4CCDE9003200224FF4F8532046114695
:105F6000FFF750FE2A460749204603B0BDE83040FF
:105F700016F09EB8C040002400000024CDC80508DB
:105F8000883A0024815B040808B528F03BFE2DE91F
:105F9000F04F027D85B005460E46012A40F08E8006
:105FA00000214FF0FF3B04460B465F4694F804C0C7
:105FB00048B2BCF1000F73D194F805C0BCF1000FDA
:105FC0006ED1B7F1FF3F17BF0133012338465BB2F3
:105FD000934201DD1A4683460131023408295DD11E
:105FE000002402EB0B03A1460293CB4502DC029B8B
:105FF0004B4558DC95F8058095F804A04FEA281722
:1060000008F00F080AF00F035FEA2A1AFAB20192A9
:106010006FD05FFA8AF1BAF1090F30460393D4BF0B
:106020003031573100F0E5F8039B0444092B30462A
:10603000039394BF03F1300103F1570100F0D9F845
:106040000444BAF1000F02D1039B03B94FB1092FE9
:10605000019F3046D4BF30375737F9B200F0C9F846
:106060000444B8F1090F304694BF08F1300108F13B
:10607000570100F0BEF8B9F1070F044404D03A21EB
:10608000304600F0B6F8044409F101090235B9F1CF
:10609000080FAAD1204605B0BDE8F08F074685E776
:1060A0004FF0FF3098E7CB45EED1BBF1000FE6D1C2
:1060B0003A21304600F09DF80444E0E700F1100773
:1060C00000F11309002417F8011B0A22304600F0E2
:1060D000F7F880462E21304600F08BF8B945404451
:1060E0000444F0D10A22E97C304600F0E9F8044487
:1060F000D0E7002B9AD1A9E7054B102210B5044632
:1061000003600175002104302AF052FA204610BDC8
:106110007C7C070870B5074D8374056000259DF8E9
:106120001030057545608560C56001744274C374A4
:1061300070BD00BF7C7C070808B50B46027D097D59
:10614000914208D1011D1022181D2AF001F9B0FA60
:1061500080F0400908BD0020FCE7037D13B9103131
:10616000084470470431FBE707B501210648FFF7F3
:10617000C3FF002305481A4619460093FFF7CAFFDC
:1061800003B05DF804FB00BFD4400024EC400024C1
:106190002DE9F04106460D4601EB02080C46444548
:1061A000A4EB050707D03368304614F8011B1B68C1
:1061B00098470028F3D13846BDE8F08170B5044611
:1061C00008460D462AF09CFF2368024629462046D1
:1061D0005B68BDE87040184709B1FFF7EFBF08469C
:1061E000704708B5FFF7F8FF08BD08B5FFF7F4FFE3
:1061F00008BD03681B6818470B460A680146126809
:10620000184610470149FFF7D9BF00BF0ED0070855
:1062100038B50546FFF7E0FF04462846FFF7F2FFD2
:10622000204438BD70B58AB00D460023012A98BFBE
:106230000A220AA901F8043DB5FBF2F402FB145648
:106240002546F3B2092E94BF30333733DBB201F861
:10625000013D002CF0D1FFF7BFFF0AB070BD2DE962
:10626000F04107460E4615462AB90368C9B21B68B5
:10627000BDE8F04118470A2A05D1002905DBBDE831
:10628000F041FFF7CFBFD2B2F9E72D21FFF7B1FF01
:1062900004462A4671423846FFF7C4FF2044BDE851
:1062A000F081FFF7DCBF10B42AB90368C9B25DF80A
:1062B000044B1B681847D2B25DF8044BFFF7B2BF1E
:1062C000FFF7F1BF0000000070B52DED068B0A9DB1
:1062D000064643EC182BB4EE488B002DB8BF0225C0
:1062E000F1EE10FA06D73C49BDEC068BBDE87040D4
:1062F000FFF764BFB0EEC87B9FED316BB4EE467B19
:10630000F1EE10FA01DD3549EEE79FED2F7BB4EE9B
:10631000C78BF1EE10FA02DD31493046E4E79FED1C
:106320002C7BB4EEC78BF1EE10FAF5D4B5EEC08B32
:10633000F1EE10FA11D52D21B1EE488BFFF759FF80
:106340000446B6EE007B0023B2EE046BDAB20133F2
:10635000AA4204DA87EE067BF8E70024F1E738EE7C
:10636000078B0A223046BCEEC89B19EE101AFFF7C5
:1063700059FF0444EDB1B8EE499B1A493046B2EEDC
:1063800004ABFFF71BFF044438EE498B15F1FF35D2
:106390000FD328EE0A8B0A223046BCEEC89B19EEBA
:1063A000101AFFF73FFFB8EE499B044438EE498BC3
:1063B000ECE7BDEC068B204670BD00BFAFF300805C
:1063C000FFFFFFFFFFFFEF7F000000E0FFFFEF4157
:1063D000000000E0FFFFEFC1807C0708847C070815
:1063E000887C070864690708FFF76EBF10B504468C
:1063F00000F0FAF8E060236820465B6998470028BF
:1064000008DA00F0F1F8E368C01AA3689842F2D302
:106410004FF0FF3010BD2DE9F04180460D468F183A
:106420000C46BC42A4EB050607D04046FFF7DEFF52
:10643000002802DB04F8010BF3E73046BDE8F081E9
:1064400010B50446006808B129F06EFC204610BD66
:1064500010B50446006808B129F066FC00232360EB
:10646000C4E9013310BD38B504460D46006801315A
:106470002AF054F910B1C4E90005012038BD0368C1
:1064800010B5044623B143688B4201D3012010BDEF
:106490002046FFF7E8FF0028F9D0A368002BF5D1CC
:1064A00022681370F3E770B50E4611460446154690
:1064B000FFF7E5FF20B92046FFF7CAFF204670BD71
:1064C0002A463146A560206829F074FF2268A36837
:1064D0000021D154F2E738B5002304460D4683600D
:1064E000C0E9003339B108462AF00AFE29460246BF
:1064F0002046FFF7D8FF204638BD88420B4610B52E
:10650000044604D0096821B19A68FFF7CCFF204601
:1065100010BDFFF79DFFFAE7002310B50446836026
:10652000C0E90033FFF7E9FF204610BD704713B5FF
:10653000002000900DF0B8FE044610B1009802B0A3
:1065400010BD01AB042269460DF08CFE20460DF013
:10655000ADFEF3E710B500F069F80A4CFDF778FFDF
:10656000FEF712FDFEF707FD4FF4E1310648FFF795
:106570004DFCFAF7CBF9FAF73FF8002CFBD0AFF35C
:106580000080F8E700000000883A002470B5054656
:106590000024074EFDF799FEE3B2984206D918464B
:1065A0001B010134F35EAB42F4D170BDFF20FCE768
:1065B0001000002410B50446FDF787FE84423BBF5F
:1065C0002401024B4FF0FF30185F10BD1000002473
:1065D00010B5044611F068FD204610BD10B5044604
:1065E00011F062FD204610BD07B50749684611F05D
:1065F00098FD4FF47A720023DDE9000127F0ACF931
:1066000003B05DF804FB00BF0841002407B504494E
:10661000684611F086FD009803B05DF804FB00BFEA
:106620002041002416F058BA16F016B908B50448EF
:1066300011F044FD0348BDE8084011F03FBD00BF24
:10664000204100240841002416F056BA38B50A4CFF
:106650000A4D204611F0A2FD2046094C2A46094960
:1066600015F026FD204611F0A4FD2A4620460649D5
:10667000BDE8384015F01CBD204100240000002476
:1066800008410024DD650408D165040870B504469E
:106690000D46164600211C2229F08AFF204632466C
:1066A000294613F0B9FD204670BD00002DE9F041E8
:1066B00004460E46FDF709FE84423CD21F4D2701D9
:1066C000EA19D06810B11C2115F078FF2046FFF7B9
:1066D00071FF80461C2015F03DFF044600211C225E
:1066E00029F066FF4146204613F093FDEB19012E79
:1066F000DC6010D006D3022E12D0204610F0F5FB3D
:10670000022103E0204610F0F0FB00212046BDE806
:10671000F04110F0F7BB2046BDE8F04110F0D8BBC7
:10672000204610F0E2FB0121F0E71C21204615F085
:1067300045FF26F0BFFDBDE8F08100BF100000243A
:1067400030B589B004460D46FFF720FFC0B2FF28E0
:1067500004D02946FFF7AAFF09B030BD012D14D09F
:106760000AD3022D1CD00222214601A8FFF78EFF7A
:1067700001A813F0EDFCEFE70022214601A8FFF786
:1067800085FF01A813F0E4FCE6E71C22002101A824
:1067900029F00EFF0022214601A813F03FFDDBE7A0
:1067A0000122214601A8FFF771FF01A813F0D0FCD8
:1067B000D2E700002DE9F34106460F46FDF785FDBF
:1067C00086422AD21B4D4FEA061805EB0802D46810
:1067D000ACB93046FFF7EEFE06461C2015F0BAFEB7
:1067E00004461C22002129F0E3FE00970023012229
:1067F0003146204613F02BFD05EB0803DC600E4B01
:106800000E491A46D3F894008842FBD123683FB161
:10681000A1680B604FF44073536102B0BDE8F08192
:10682000E1681B04F5E71C21204615F0C7FE26F0A1
:1068300041FD00BF100000240064025800030080E6
:1068400030B589B005460C46FFF7A0FEC0B2FF2860
:1068500004D02146FFF7AEFF09B030BD1C22002155
:1068600001A829F0A5FE294601A813F0EDFC094B6B
:1068700009491A46D3F894008842FBD1019B2CB1F8
:1068800003990B604FF440735361E5E71B040499CF
:10689000F7E700BF00640258000300801EF0040FF9
:1068A0000CBFEFF30880EFF30980816911F8021C37
:1068B000002932D101B590E80F10E047BDE8005043
:1068C0008CE80300244B93E80600914208BF704710
:1068D0001A6041B91EF0100F10D1204B186820F03B
:1068E000010018600AE02CE9F00F1EF0100F08BF3D
:1068F0002CED108A81F822E0C1F838C0906B92F834
:10690000221061F0FF0E1EF0100F08BFB0EC108ACD
:10691000B0E8F00F80F309887047114A1368994274
:10692000FAD801B552F821C00FC8E047BDE80050C1
:10693000CCF80000704701B501F0D4FBBDE8014080
:10694000EFF3098CBEE701B501F090FBBDE8014013
:10695000EFF3098CB6E70000440C002434EF00E0AC
:10696000547D0708014608B530B96FF0030000F008
:106970001DFA6FF0030008BD132001F0ABFF30B922
:106980004FF0FF3000F012FA4FF0FF30F3E7002035
:10699000F1E7000008B5EFF305832BB9EFF310839F
:1069A00013B9EFF3118333B16FF0050000F0FEF976
:1069B0006FF0050008BDDFF808C000DFFAE700BF90
:1069C00065690408EFF310832BB9EFF311800038E9
:1069D00018BF012070470120704710B520B103781F
:1069E000F32B01D1002906DA6FF0030102F05CFA03
:1069F0006FF0030010BD00F10C0353E8000F20EA14
:106A0000010243E8002404B1F7E7F3E738B505468F
:106A1000A0B1846802686CB114F0030302D1C168AC
:106A20000F2926D800246FF00801002002F03CFA5C
:106A3000204638BDC368002BF4D11546104BD3F85F
:106A4000900078B100F087FC0446A0B10123F32246
:106A5000A3700023656022700A4AC4E90233084B20
:106A60005A66E5E701221021D3F8800000F0FAFB16
:106A7000EAE71546EBE76FF0040102F015FAD7E7F5
:106A8000300C0024F16A0408930710B502F00104E9
:106A900022D400F10C0384B153E8000F00EA010294
:106AA0008A4203D0BFF32F8F002005E020EA0102C5
:106AB00043E8002404B1EFE710BD53E8000F08429B
:106AC00003D1BFF32F8F002005E020EA010243E845
:106AD000002404B1F1E7EFE7C06801EA00031CB14C
:106AE000994218BF0020E7E7002B08BF0020E3E72A
:106AF000F8B50546846804B9F8BD94F82320284603
:106B0000616AA768FFF7C0FF064638B1204601F06A
:106B100062FC00223146204601F0F6FD3C46EAE7E1
:106B2000F8B50D4617461E46044620B10378F32BF0
:106B300001D1002907DA20466FF0030102F0B4F911
:106B40006FF00300F8BDFFF79FFF0028FAD186B170
:106B50003146432001F0BEFE40B1074B20465E693E
:106B6000314601F01DFC756286F823706FF001005C
:106B7000E8E76FF00200E5E7300C002470B5054649
:106B800010B10378F32B07D028466FF0030102F011
:106B90008BF96FF0030070BD836863B1284601F084
:106BA00011FC00226FF0020101F0AEFDA868002880
:106BB000F4D101F08FFCAB78002613F001032E70A6
:106BC0000FD0094B2946D3F8904024B1204600F05D
:106BD000DCFB3046DFE7D3F8800000F078FB20468E
:106BE000D9E71846D7E700BF300C00242DE9F04163
:106BF000064620B10378F32B01D1002909DA6FF0A2
:106C000003056FF00301304602F04EF92846BDE857
:106C1000F08100F10C0353E8002F42EA010543E83C
:106C2000005000B1F7E7B4681CB9204601F052FCEF
:106C3000ECE794F823203046616AD4F80880FFF727
:106C400023FF074678B194F823309B0756BF656A47
:106C5000054620EA0505204601F0BDFB0022394625
:106C6000204601F051FD4446DEE70000024608B52B
:106C7000EFF3058333B100206FF0050102F014F942
:106C8000002008BDFFF79EFE0028F4D11046DFF873
:106C900008C000DFF5E700BF0D6A0408024638B5FA
:106CA000EFF305834BB192B96FF003046FF003016A
:106CB000104602F0F9F8204638BDFFF783FE0028A1
:106CC000F1D11046DFF82CC000DF0446F3E713785B
:106CD000F32BE9D10029E7DB02F10C0353E8000FA5
:106CE00040EA010443E8004505B1F7E7104601F02A
:106CF00041FAE0E7ED6B0408024608B5EFF30583BF
:106D000023B11046BDE80840FFF767BEFFF75AFE03
:106D10000028F6D11046DFF808C000DF08BD00BF2C
:106D2000DB69040838B504461D46EFF3058343B11B
:106D30008CB920466FF0030102F0B6F86FF0030043
:106D400038BDFFF73FFE0028F2D120462B46DFF882
:106D500024C000DFF4E72378F32BEAD1002DE8D13B
:106D60000029E6DB2046FFF78FFE002808BF6FF002
:106D70000200E5E7216B0408024608B5EFF305833E
:106D80003BB110466FF0050102F08EF86FF0050080
:106D900008BDFFF717FE0028F3D11046DFF804C046
:106DA00000DFF5E77D6B0408704770477047EFF32D
:106DB00010832BB9EFF31180003818BF0120704702
:106DC00001207047064BDA6A3AB1D0695B6C1BB19F
:106DD0001B69984228BF184670474FF0FF30F5E70F
:106DE000300C0024014BD868704700BF300C0024E1
:106DF00008B5094B1A7A022A08D0032A0AD04FF0A4
:106E0000FF3002F045F84FF0FF3002E0032200208F
:106E10001A7208BD0120FCE7300C002470B5464C06
:106E2000237A012B00F0858033B14FF0FF3002F060
:106E30002FF84FF0FF3070BD404DEB68E3652B8AB3
:106E4000D5E90B61A4F85430AB683046236400F0F8
:106E5000F1F908B1C4F88060D5E90561304600F069
:106E6000E9F908B9D4F880606667D5E9076130466A
:106E700000F0E0F908B9D4F88060A667D5E90961A7
:106E8000304600F0D7F908B9D4F88060E6676E6B39
:106E90003EB131683046D6E9022300F03BFAC4F82F
:106EA0008460AE6B3EB131683046D6E9022300F013
:106EB00031FAC4F88860EE6B3EB131683046D6E9ED
:106EC000022300F027FAC4F88C602E6C3EB13168C2
:106ED0003046D6E9022300F01DFAC4F890606E6CCB
:106EE0003EB131683046D6E9022300F013FAC4F807
:106EF0009460AE6C3EB131683046D6E9022300F0B2
:106F000009FAC4F89860EE6C3EB131683046D6E9B3
:106F1000022300F0FFF9C4F89C602D6D3DB1296893
:106F20002846D5E9022300F0F5F9C4F8A050012362
:106F3000237200207FE700BF300C0024E47C0708A8
:106F400070B5254D2B7A012B07D06FF006004FF05E
:106F5000FF3401F09DFF204670BD01F01FFD10B908
:106F60004FF0FF30F3E71D4AFF231D4E82F8223019
:106F700092F82230D26863F0FF031A49C2F302226A
:106F80007068DB4314BFB3FA83F32023C3F12003FB
:106F9000934298BF531CFE2202FA03F30F4ADBB25E
:106FA000D37701F0D1FF04460028D9D102F024F8AC
:106FB000286102F00DF80C4801F004FA01F082FAA1
:106FC0003368DB074CBF0223032383F31488BFF32A
:106FD0006F8F02232B72BEE7300C002400ED00E01F
:106FE000E47C0708476904084C0C002408B50A4BE8
:106FF0001A7A023A012A02D840B1012809D04FF08A
:10700000FF3001F045FF4FF0FF3001E002221A721D
:1070100008BD0322FBE700BF300C002410B50F4C65
:10702000237A022B13D101F0DBFF01236372BFF33C
:107030004F8F0B4A5168C90003D54FF00061516072
:10704000A37204232372BDE81040FFF7BBBE6FF0AC
:10705000070001F01DFF002010BD00BF300C002410
:1070600000ED00E038B51E4C0546237A042B35D1DF
:10707000FFF7A8FEE26AA842034694BF00F1FF337F
:107080002B4612B1D069C01AD061626C12B110697E
:10709000C01A1061E06803440544E360E368AB4252
:1070A00013D102230020237201F014FA002363722B
:1070B000BFF34F8FA27A22B1A3724FF08052094BD7
:1070C0005A60BDE8384001F083BF0133E36001F04E
:1070D000BFF9236D002BE1D09847DFE738BD00BF33
:1070E000300C002400ED00E0704738B504460D4632
:1070F000FFF75AFE29462046BDE8384001F08ABE17
:1071000008B5FFF7F1FFEFF3058333B16FF005002A
:1071100001F0BEFE6FF0050008BDFFF748FE002835
:10712000F4D1DFF808C000DFF6E700BF1D6E0408E9
:1071300008B5EFF3058333B16FF0050001F0A8FE49
:107140006FF0050008BDFFF732FE0028F4D1DFF82C
:1071500008C000DFF6E700BF416F040808B5EFF391
:10716000058333B16FF0050001F092FE6FF005006A
:1071700008BDFFF71CFE0028F4D1DFF808C000DFCF
:10718000F6E700BFF16D0408024608B5EFF305838A
:1071900033B16FF0050001F07BFE6FF0050008BD14
:1071A000FFF705FE0028F4D11046DFF808C000DF25
:1071B000F5E700BFED6F040808B5EFF305832BB1C9
:1071C0006FF0050001F064FE002008BDFFF7EFFD41
:1071D0000028F5D1DFF804C000DFF6E71D700408D1
:1071E000024608B5EFF305832BB16FF00500BDE84B
:1071F000084001F04DBEFFF7DAFD0028F5D110463A
:10720000DFF804C000DF08BD6570040808B5EFF3BF
:10721000058313B1054BD86808BDFFF7C8FD0028EA
:10722000F8D1DFF80CC000DFF6E700BF300C002417
:10723000E56D040810B598B140EA010313F00703A7
:107240000ED117290AD90160083910220C184260A2
:1072500084600B5081684A60C3600123184610BDEA
:107260000023FBE7F0B580B399B132F003032CD1D2
:107270000F3100F1080521F007072B462D685C68E7
:10728000E91A24F00304091B8F4204D92968002954
:10729000F3D10846F0BD46683A4304683E44466070
:1072A000204450F8041C08388E4288BF4660586855
:1072B00018B903F108015A60EBE720F00300191830
:1072C0001D504A6019600831E3E70021E1E730B55D
:1072D00090B1D9B1A1F1080500F108040022AC4237
:1072E0000BD151F8043C23F0030443681B1B43609B
:1072F00042B941F8042C012030BD236822463BB13D
:107300001C46ECE751F8083C1360F4E70846F3E745
:107310001846F1E730B5C0B189B1C2B1CBB1002494
:107320000160C3604361C0E9014202FB01F41D1921
:1073300005611846013904D1A21A99500121084665
:1073400030BD851805602846F4E70146F7E7114689
:10735000F5E71946F3E7034610B5A8B100F11402AA
:1073600052E8000F10B9BFF32F8F04E0016842E824
:10737000001404B1F4E738B1043353E8002F511C72
:1073800043E8001404B1F8E710BD30B5F0B1C368AC
:107390008B421BD803698B4218D900F114031A6879
:1073A0000A60BFF35F8F53E8002F0C689442F6D158
:1073B00043E8001505B1F2E7043050E8003F5A1EDB
:1073C00040E8002101B1F8E7002030BD6FF0030074
:1073D000FBE7EFF310832BB9EFF31180003818BFF0
:1073E0000120704701207047036B30B5E3B1CD78C1
:1073F0000024DA78AA420FD31A46C1E901248AB1DF
:107400009160A4B16160283050E8003F5A1C40E808
:10741000002101B1F8E730BD5A681C46002AECD0C3
:107420001346E6E7C162ECE7C1E90133C1620163DB
:10743000E9E7D1E9013223B19A608A681AB1536051
:107440007047C262F9E703637047F8B5877804466E
:107450008FB3C5680027014605F10C062846FFF7E3
:10746000E8FF27703046FFF790FFAB68002B48D04D
:107470003046FFF770FF0446002842D0284600F04F
:10748000A1FF06463A46394601F03EF9304601F082
:107490000FF86A6A0646816804F10C0028F08AFF3A
:1074A000F923A7702370F368E37021462846BDE8EE
:1074B000F840FFF799BF8568AB68002BF5D05B7883
:1074C000832BF2D1284600F07DFF06463A46394626
:1074D00001F01AF9304600F0EBFF06466A6A04F143
:1074E0000C01806828F066FFF3680BB1E2781A702F
:1074F0000023214605F10C002370BDE8F840FFF79A
:1075000044BFF8BD2DE9F0410C46174698460546A4
:1075100018B10378FA2B00D141B928466FF0030166
:1075200001F0D8FC6FF00300BDE8F0818368C3B1BF
:107530005B78832B15D100F045FF06460122002120
:1075400001F0E2F8304600F0B3FF06466A6A2146D1
:10755000806828F02FFFF0680028E5D00770002031
:10756000E2E705F10C00FFF7F6FE064670B1214692
:107570006A6A0C30002428F01DFFF92331462846A2
:107580003370B470F770FFF72FFFE8E7B8F1000F22
:1075900010D04146932001F09DF940B1074B284699
:1075A000596900F0FDFEEFF30983C3E902476FF06C
:1075B0000100B9E76FF00200B6E700BF300C00240D
:1075C0002DE9F84F8846074638B131B1B0FA80F35B
:1075D000B1FA81F10B441F2B06DC6FF00301002090
:1075E000002401F077FC70E008F1030626F00306A2
:1075F0000C3606FB00F9F2B194683CB1A30702D146
:10760000D368332B05D86FF00801E8E7D368002B67
:10761000F9D1D2F800A0D2E904533DB115F0030B23
:1076200001D1994554D96FF00901D8E7002BFAD15F
:107630001CB19B460CE092461546274BD3F8A000A0
:10764000D8B1FFF788FE0446A0B14FF0010B35BB5F
:10765000214B00224946D86FFFF704FE0546C0B90A
:10766000BBF1000F06D01C4B2146D3F8A00058B147
:10767000FFF78BFE6FF00401B1E701223421D3F84C
:107680008000FFF7EFFDDEE7D3F88000FFF71FFE75
:10769000F0E74BF0020B4A46002128F089FFFA235D
:1076A0003246394604F10C002370002384F802B0FE
:1076B000A360C4F804A0C4E90983C4E90B332B46D2
:1076C000FFF728FE044B054A1A672046BDE8F88FED
:1076D000002CE4D1B1E700BF300C00244B74040847
:1076E00000F1280310B553E8002F12B9BFF32F8F14
:1076F00004E0511E43E8001404B1F4E70AB9002085
:1077000010BDC06A01230028F9D0821CD2E84F1FA7
:10771000C2E8443F04B1F9E711F0FF0FF0D08068F0
:10772000F1E700002DE9F0410F4615469846044662
:1077300018B10378FA2B00D141B920466FF003014C
:1077400001F0C8FB6FF00300BDE8F081FFF7C8FF50
:10775000064600283AD001462046FFF76AFE626AD4
:1077600006F10C01384628F025FE0DB1F3782B7098
:10777000002504F10C07314638463570FFF705FE49
:10778000A3680BB90020DFE73846FFF7E4FD0646A3
:107790000028F7D0204600F015FE074629460122B2
:1077A00000F0B2FF384600F083FE626A0746816847
:1077B00006F10C0028F0FEFDF923B5703146337058
:1077C0002046FB68F370FFF70FFEDBE7B8F1000F10
:1077D00010D04146832001F07DF840B1074B204690
:1077E000596900F0DDFDEFF30983C3E902756FF01D
:1077F0000100A9E76FF00200A6E700BF300C0024EB
:1078000008B5064B08219A6ED86EFFF7D9FE044BD7
:10781000D864B0FA80F04009404208BDE47C070813
:10782000300C00242DE9F04106460F4690461C46D8
:10783000EFF305834BB196B930466FF0030101F0C9
:1078400049FB6FF00300BDE8F081FFF7C2FD00289F
:10785000F1D130462346DFF848C000DFF3E7337844
:10786000FA2BE9D1002FE7D0002CE5D106F10C006E
:10787000FFF771FD054680B1726A39460C3028F079
:1078800099FDF9232846AC702B7085F80380C5E973
:10789000017600F06FFC2046D5E76FF00200D2E7DA
:1078A00005750408F8B504460F4616461D46EFF365
:1078B000058343B18CB920466FF0030101F00AFB48
:1078C0006FF00300F8BDFFF784FD0028F2D12046D9
:1078D0002B46DFF844C000DFF4E72378FA2BEAD127
:1078E000002FE8D0002DE6D12046FFF7F9FE05462F
:1078F00070B100F10C01626A384628F05BFD0EB1F0
:10790000EB7833702846EC6000F034FC0020D9E7B7
:107910006FF00200D6E700BF25770408EFF310836D
:107920002BB9EFF31180003818BF012070470120F8
:107930007047000070B5A8B38468D0E900566CB1F8
:1079400014F0030302D1C2681B2A1AD800246FF076
:107950000801002001F0AEFA204670BDC368002B7C
:10796000F4D1124BD3F8940030B901221C21D3F882
:107970008000FFF777FC01E0FFF7EDFC044660B103
:107980000123F522A3700023E67022706560237640
:10799000C4E90233C4E90433DEE76FF0040101F007
:1079A00089FAD9E705460646DBE700BF300C00241C
:1079B000284B70B55D6904460E4635B96FF0070176
:1079C00001F078FA4FF0FF3070BD10B10378F52B5D
:1079D00007D020466FF0030101F06CFA6FF003004E
:1079E000F2E7037E53B9C0E90353EB6A436103B185
:1079F00018610123EC6200202376E5E7C278D10705
:107A00000DD5C168A9420AD1FF2B06D16FF00F0135
:107A100001F050FA6FF00200D6E70133EBE7002ED9
:107A2000F8D093070AD5E06895F9203090F9202026
:107A30009A4203DA80F8203000F0D6FC3146532019
:107A400000F048FF18B12946204600F0A9FC6FF06D
:107A50000100B9E7300C00242E4B5A6970B504467A
:107A600032B96FF0070101F025FA4FF0FF3070BD19
:107A700010B10378F52B07D020466FF0030101F019
:107A800019FA6FF00300F2E7037E33B96FF00E01CD
:107A900001F010FA6FF00200E9E7C168914202D0EC
:107AA0006FF00D01F4E7013BDBB2037613BB4369D2
:107AB0000BB1016919612169F1B14B6192F9213072
:107AC000D56ADDB982F82030A36883B1204600F082
:107AD00079FC06462A46294600F016FEF36AC4E9F8
:107AE0000365636103B11C610123F4622376002006
:107AF00000F0F0FC0020BAE7D362DFE7E9788907FD
:107B000006D5A96821B191F920108B42B8BF0B4668
:107B10006D69D6E7300C002470B5044610B10378C7
:107B2000F52B07D020466FF0030101F0C3F96FF089
:107B3000030070BD037EBBB16369C0680BB12269ED
:107B40001A61226902B3536190F92120C36AEBB92B
:107B500090F92030934203D080F8202000F044FCBC
:107B6000A068F8B900F0B6FCA078002610F001007B
:107B70002670DED0134B2146D3F89450DDB1284651
:107B8000FFF703FC3046D4E7C362DDE7D978890705
:107B900006D5996821B191F920108A42B8BF0A46EA
:107BA0005B69D4E7204600F00DFC00226FF0020173
:107BB00000F0AAFDD4E7D3F88000FFF788FB284641
:107BC000B7E700BF300C00242DE9F0410446002641
:107BD00001270CB9BDE8F081E378D4F814801B07C5
:107BE00012D5A36826767BB1204600F0EBFB00227D
:107BF0000546114600F088FDEB6AC4E9035663614F
:107C000003B11C61EC6227764446E2E710B4C37806
:107C10009B071DD5C06890F92120C36ADC78A407B2
:107C200009D59C688C4208BF8C6824B194F9204027
:107C3000A242B8BF22465B69002BEFD190F92030F9
:107C4000934205D080F820205DF8044B00F0CCBBB7
:107C50005DF8044B70470000024608B5EFF305835A
:107C600033B100206FF0050101F024F9002008BDB8
:107C7000FFF754FE0028F4D11046DFF808C000DFFB
:107C8000F5E700BF35790408024608B5EFF3058330
:107C90003BB110466FF0050101F00CF96FF00500E3
:107CA00008BDFFF73BFE0028F3D11046DFF804C003
:107CB00000DFF5E7B1790408024608B5EFF3058364
:107CC0003BB110466FF0050101F0F4F86FF00500CC
:107CD00008BDFFF723FE0028F3D11046DFF804C0EB
:107CE00000DFF5E7597A0408024608B5EFF305838B
:107CF0003BB110466FF0050101F0DCF86FF00500B4
:107D000008BDFFF70BFE0028F3D11046DFF804C0D2
:107D100000DFF5E7197B0408EFF310832BB9EFF3CD
:107D20001180003818BF01207047012070470C30C7
:107D3000D0E85F3F13B9BFF32F8F04E05A1EC0E8AD
:107D4000512F01B1F4E798B2003818BF01207047F5
:107D500030B500F10C02C189D2E85F3F994202D8E8
:107D6000BFF32F8F04E05C1CC2E8554F05B1F3E769
:107D7000C0899BB2984294BF0020012030BD000012
:107D8000F8B515464FF6FE73421E06460F469A4258
:107D900001D8884207D26FF003010024002001F0CF
:107DA0008FF82046F8BD7DB1AC682A6844B114F064
:107DB000030302D1E9680F2922D86FF00801ECE72C
:107DC000EB68002BF9D11546114BD3F8980080B120
:107DD000FFF7C1FA0446A8B10123F622A3700023DD
:107DE00065602270A3600B4A094BA781E6819A6601
:107DF000D7E701221021D3F88000FFF733FAE9E733
:107E00001546EAE76FF0040101F05AF8C9E700BF30
:107E1000300C0024197E0408836810B504465BB159
:107E2000FFF785FF40B1204600F0CCFA0022BDE804
:107E30001040114600F068BC10BD38B5054610B1C1
:107E40000378F62B07D028466FF0030101F038F8CD
:107E50006FF0030038BD84683CB100F0B3FA012232
:107E6000002100F051FC0020F4E7FFF771FF38B962
:107E700028466FF0100101F023F86FF00200E9E7E7
:107E80002046E7E738B50D46044610B10378F62BD7
:107E900007D020466FF0030101F012F86FF00300E5
:107EA00038BDFFF744FF68B975B12946632000F07B
:107EB00011FD20B1064B2046596900F071FA6FF0B0
:107EC0000100EDE70020EBE76FF00200E8E700BFFC
:107ED000300C002470B5054610B10378F62B07D09E
:107EE00028466FF0030100F0EBFF6FF0030070BD58
:107EF000836863B1284600F065FA00226FF0020142
:107F000000F002FCA8680028F4D100F0E3FAAB7896
:107F1000002613F001032E700FD0094B2946D3F829
:107F2000984024B12046FFF730FA3046DFE7D3F817
:107F30008000FFF7CCF92046D9E71846D7E700BF05
:107F4000300C002410B50446EFF3058333B1002054
:107F50006FF0050100F0B4FF002010BDFFF7DCFE5C
:107F60000028F4D12046DFF808C000DFF5E700BFA5
:107F7000817D0408024608B5EFF3058343B182B959
:107F800010466FF0030100F09BFF6FF0030008BD87
:107F9000FFF7C2FE0028F2D11046DFF824C000DF50
:107FA000F5E71378F62BEBD10029E9D11046FFF75E
:107FB000BEFE002814BF00206FF00200E7E700BFFC
:107FC000857E040810B50446EFF3058343B184B9F8
:107FD00020466FF0030100F073FF6FF0030010BD47
:107FE000FFF79AFE0028F2D12046DFF830C000DF0C
:107FF000F5E72378F62BEBD12046FFF7A9FE20B159
:10800000204600F0B7F80020E9E720466FF01001A5
:1080100000F056FF6FF00200E1E700BF3B7E04086E
:10802000024608B5EFF305833BB110466FF005013A
:1080300000F046FF6FF0050008BDFFF76DFE002859
:10804000F3D11046DFF804C000DFF5E7D57E040861
:1080500010B5D0E85F3F5A1C914200D80022C0E81A
:10806000542F04B1F5E798B210BD000038B51C4C90
:1080700000F0BCFFE3680133E36000F0E9F90020A1
:1080800000F028FA236D03B19847226C32B3A3693C
:10809000E16B994203D0D969E36301B9DA61DA6926
:1080A000C2B9237A022B19D1656ABDB1E36B95F988
:1080B000202093F920309A4210D1284600F08BF905
:1080C000E06B00F0A3F9284600F0FCF9236CE563AF
:1080D000EB6103E0013ADA61002AE2D038BD00BF6B
:1080E000300C002470B5224C04F1560504F15A06F8
:1080F000B4F85410D5E85F3F13B9BFF32F8F04E0F5
:108100005A1EC5E8502F00B1F4E79BB25BB330466E
:10811000FFF79EFFE36D53F8200020B30378F13B97
:10812000082BE5D801A252F823F000BF51810408C2
:10813000F180040857810408F1800408F1800408E4
:108140005B8104085F810408F180040863810408EE
:10815000236E9847CCE7636EFBE7A36EF9E7E36E07
:10816000F7E7236FF5E70020BDE8704000F0B2B9F3
:10817000300C002470B5164C0546B4F8541004F1C8
:108180005602D2E85F3F994202D8BFF32F8F04E036
:10819000581CC2E8560F06B1F3E79BB2994205D8C6
:1081A00029460220BDE87040FEF79FBF04F1580049
:1081B000FFF74EFFE36D43F82050637A23B9054B78
:1081C0004FF080525A6070BD0123A372FBE700BFDD
:1081D000300C002400ED00E0EFF310832BB9EFF337
:1081E0001180003818BF01207047012070470378C4
:1081F000F12B00D07047C068F9E7000010B5C469E2
:10820000621CD0E904310CD103B1596142691AB141
:1082100013610023436101E0074A13630023C36134
:1082200010BD1BB1DA6959612244DA614269002A42
:10823000EED1014AD362F1E7300C002401230A4A4F
:1082400090F9201043701C32936810B51BB193F95C
:1082500020408C4205DCC0E90232906003B1D86056
:1082600010BD1A469B68F1E7300C0024014B586999
:10827000704700BF300C002408B500F031FEDFF875
:1082800010C000DF4FF0FF31002000F007FEFEE7D6
:1082900071870408930710B502F0010422D400F19D
:1082A000280384B153E8000F00EA01028A4203D098
:1082B000BFF32F8F002005E020EA010243E80024ED
:1082C00004B1EFE710BD53E8000F084203D1BFF33C
:1082D0002F8F002005E020EA010243E8002404B1CA
:1082E000F1E7EFE7806A01EA00031CB1994218BF89
:1082F0000020E7E7002B08BF0020E3E7084A002141
:10830000136B10B53BB94FF0FF34C0E90431C461C1
:1083100021B1086110BD19461B69F3E71063F9E745
:10832000300C0024002310B50380044683789A079C
:1083300008D513F0100F016B0E4B0FD0D3F884004B
:10834000FFF723F8A378DB0712D50A4B2146D3F8B1
:10835000880038B1BDE81040FFF717B8586FFEF736
:10836000B6FFEFE7D3F88000BDE81040FEF7AFBFDF
:1083700010BD00BF300C0024C2780346D20701D4E0
:10838000FFF7D0BF042242700022C260034A516B43
:10839000816001B1C8605363704700BF300C002496
:1083A00091F92020836810B51BB193F920409442C5
:1083B00005DAC1E90230816003B1D96010BD184609
:1083C0009B68F1E783689A68826002B1D0600022FE
:1083D0001846DA607047C2682AB18368936003B1B7
:1083E000DA600023C360704710B50146044664B1EB
:1083F0002378F12B07D00846FFF7EDFF2046BDE8B4
:108400001040FFF7CDBFE468F1E710BD012301463E
:1084100043700148FFF7C4BF4C0C002470B50B4DEE
:108420002E7A022E10D16C6A74B1696994F92020F9
:1084300091F920309A4207D12046FFF7CCFF084639
:10844000FFF7E4FF6670AC61002070BD300C0024C3
:1084500038B5164DEC6A44B3E369013BE36123BBD5
:108460006378732B06D009D8532B0BD003F0DF03AE
:10847000432B0DD12046FFF7BAFE09E003F0EF03CE
:10848000832BF6E72046FFF7B2FE2146FFF7BEFB3F
:108490002046FFF7A0FFFFF7B9FF246924B1E36985
:1084A000002BDDD000236361EC6238BD300C00246A
:1084B00090F82230826B13F0100F0CBF6020202048
:1084C0001044704702234370014B9861704700BF0E
:1084D000300C002470B5124D04462E7A696990B9AB
:1084E000022E0FD16C6A6CB194F9202091F92030E2
:1084F0009A4207DD2046FFF76EFF0846FFF79EFE13
:108500006670AC6170BD022E05D190F9202091F902
:1085100020309A42F1DC2046BDE87040FFF776BF7C
:10852000300C00242DE9F04F85B08146029128B926
:108530006FF00301002400F0B1FCBCE0002A45D03C
:10854000966846B1B40702D1D368432B06D86FF0C2
:1085500008010020EEE7D368002BF8D19769D2E933
:1085600004453CB1600702D1002D40F0B2806FF0AD
:108570000A01EEE72FB17B1E372B03D96FF00B01F9
:10858000E7E71827002D40F0A880D2E900A3019367
:108590004EBB574BD3F88800F0B1FEF7DCFE064621
:1085A00000283AD04FF00108002C44D1DFF840B148
:1085B000E5B9504ADBF88400556DB8B1FEF7CBFE43
:1085C0000246E0B148F01008344623E092461446D3
:1085D000182715460192DCE701224421D3F88000D8
:1085E000FEF740FEDBE74FF00008DDE722462946B4
:1085F000DBF87400FEF736FE02460028E4D1B8F13D
:10860000000F16D0DBF8882052B110463146FEF735
:10861000BCFE002248F002087CB96FF0040198E724
:108620003146DBF880000392FEF751FE039A1446B0
:10863000F0E74246EEE72246344640F2F1137FB2BD
:10864000FD2184F802802380019BC4F804A0E3701C
:10865000002384F8207084F8217061846563C4E984
:108660000233C4E90433C4E90633C4E90933C4E975
:108670000B32A5F140031344C4E90E391E4B1360BD
:108680001C4B1B685B071AD4A36B00201A4603F12E
:10869000340143F8040B9942FBD1184B2046C2E940
:1086A0000D394FF08073D363029B1362104B144A51
:1086B0001A66FFF70FFF204605B0BDE8F08FAD0842
:1086C0004FF0CC33113D002DDED0013D42F8043F88
:1086D000F9E7002F7FF44FAF182769077FF447AF02
:1086E000A5F14801074B99427FF64FAF3FE700BF26
:1086F000300C0024E47C0708A52E5AE27982040895
:108700002D870408B7FFFF7F38B504461546FFF7ED
:10871000CFFE01602046FFF771FD1DB1BDE8384076
:10872000FFF7D8BEBDE83840FFF770BE10B54378FC
:108730000446332B0CD1416A90F82320FFF7AAFDA1
:10874000014628B120460022BDE81040FFF7DCBFFB
:1087500010BD10B50446806918B100221146FFF71C
:10876000D3FF6378232B02BFA36800229A6110BD58
:1087700070B50F4C267A022E18D1636AB3B16569C1
:10878000E86AFFF721FA2846FFF7E3FF04F11C002F
:10879000FFF718FE4670A061EFF30983AB63002377
:1087A00028466361BDE87040FFF7E6BD70BD00BFBD
:1087B000300C002410B5044610B10378F12B07D01B
:1087C00020466FF0030100F069FB6FF0030010BD5D
:1087D000437803F00F03022B1ED0032B2BD0012B69
:1087E0002ED1FFF7F8FDE06AFFF7EEF92046FFF71C
:1087F000B0FF6178022926D11548FFF7E3FD154B3C
:1088000041709861EFF30982A26300225A61204609
:10881000FFF7B2FD0020DAE70E4B1A7A022A02D1E6
:108820005B6A002BDFD16FF00201204600F036FBBF
:108830006FF00200CBE7FFF7CEFDFFF7DFFCD2E7DA
:108840006FF00201F2E70020FFF744FEDFE700BF10
:108850004C0C0024300C002470B5044620B1037881
:10886000F12B01D1002908DA6FF003056FF0030145
:108870002046FEF79AFA284670BD4378042B06D1AD
:108880006FF002016FF00205FEF78FFAF3E700F1D7
:10889000280353E8002F42EA010543E8005606B1D9
:1088A000F7E74378332BE6D1416A90F82320FFF7AE
:1088B000F1FC01460028DED094F8233001229B070A
:1088C00056BF656A054620EA05052046FFF71CFFEE
:1088D000D1E7000038B5174C0246237A022B27D186
:1088E000606A60B160694B1C427009D1FFF706FDF8
:1088F0001148FFF767FD02234370A061012038BDD6
:10890000E36A002213B1DD69A9420BD2C161C0E95B
:1089100004325AB11061002BEAD0DA695861511A59
:10892000D961E5E71A46491B1B69EBE7E062F2E70C
:108930000020E4E7300C00244C0C0024F8B5164B62
:1089400005460F4616465C693CB920466FF00701A4
:10895000FEF72BFA4FF0FF30F8BD002807DA20466B
:108960006FF00301FEF721FA6FF00300F4E70A4607
:1089700001462046FFF78EFC0028EDD14EB131466E
:108980003320656284F82370FFF7A4FF6FF00100C5
:10899000E2E76FF00200DFE7300C002438B50D4C41
:1089A00000210D48A26DFFF7BDFD0C4D636EA8625E
:1089B0005BB1984758B9E26DE96C206EFFF7B2FDE4
:1089C000A864003818BF012038BD0120FCE7002052
:1089D000FAE700BFE47C07080D8E0408300C002481
:1089E00010B50446EFF3058333B100206FF00501A5
:1089F00000F054FA002010BDFFF7EEFB0028F4D180
:108A00002046DFF808C000DFF5E700BF2585040831
:108A100008B5EFF3058313B1054B586908BDFFF79F
:108A2000DBFB0028F8D1DFF80CC000DFF6E700BF61
:108A3000300C00246D82040808B5EFF305833BB1C8
:108A400000206FF0050100F029FA6FF0050008BD65
:108A5000FFF7C2FB0028F3D1DFF804C000DFF6E720
:108A60001D84040810B5044600F046FAEFF30583B0
:108A70003BB120466FF0050100F010FA6FF00500E1
:108A800010BDFFF7A9FB0028F3D12046DFF804C092
:108A900000DFF5E7B5870408024638B5EFF3058334
:108AA0004BB192B96FF003046FF003011046FEF76B
:108AB0007CF9204638BDFFF78FFB0028F1D1104626
:108AC000DFF844C000DF0446F3E71378F12BE9D167
:108AD0000029E7DB5378042B07D16FF00201104621
:108AE0006FF00204FEF761F9E3E702F1280353E8AF
:108AF000000F40EA010443E8004505B1F7E71046DE
:108B0000FFF738FBD5E700BF5988040810B50446C5
:108B1000EFF305833BB100206FF00501FEF745F947
:108B20006FF0050010BDFFF757FB0028F3D120467A
:108B3000DFF804C000DFF5E73D8904080C4A30B5D2
:108B4000536C002413B11D698D420AD90161C0E93B
:108B500002431BB11D699860691A19612CB1E0606C
:108B600030BD1C46491BDB68ECE75064F8E700BFEA
:108B7000300C00242DE9F041184D6C6C54B323697E
:108B800001276E69013B2361236913BBE3680BB1C5
:108B9000A2689A606B64002304F11801E86C1A461D
:108BA000FEF740FE58B121460320D5E905836B61ED
:108BB000FEF79BFA6B6913B9B04508BF0026E3784E
:108BC000012B09D161692046FFF7B8FF6C6C002CBE
:108BD000DAD16E61BDE8F0816770F7E7300C0024F0
:108BE00008B5FEF70DFE18B9034B044A1A6508BD17
:108BF0004FF0FF30FBE700BF300C0024758B0408FA
:108C0000044607B54FF0FF33002269462046FEF7C1
:108C100049FE0028F6D1DDE900309847F2E7000070
:108C200008B5094A094B1A60094B9B1A094A136097
:108C3000094A0A4B1A600A4B9B1A0A4A136000F051
:108C400051F800F083F800BF00FC07246C490024B1
:108C50000000082468490024981E0124F4690024B7
:108C600000FC0724F069002438B50E480B250E4B94
:108C70001C24456003600D4BC4608360FEF7ECFF6D
:108C80000B4B18600B480C4BC460C0E900350B4B14
:108C90008360FEF7E1FF0A4B1860BDE8384026F01C
:108CA00085BF00BF38490024B87D07084C4900241F
:108CB0004849002408490024C57D07081C490024B0
:108CC00018490024FDF746BC024B4FF0FF311868ED
:108CD000FEF7DABF48490024014B1868FEF7ECBFE5
:108CE0004849002408B511F08DFD0C4B0C499868DB
:108CF0004FF00053C21802F16042126843F8042B8F
:108D00008B42F7D1054B4FF000529A6021F048FB9F
:108D100023F0C2FDBDE8084000F015B800ED00E00A
:108D2000980200207047704708B500F043F8FFF73D
:108D3000F9FFFFF799FFFFF7F6FF12F069FFBDE8B3
:108D40000840FFF7BFBFFEF7DBB90000114C124B24
:108D500023614FF4004363614423E3600F4BA3603E
:108D60001823A3610E4B07B5224600210D4823604E
:108D7000FFF736FE034628B922460B4900900B4800
:108D800012F056FFFEF7D4F9002309491A46009362
:108D9000F5E700BFB0FC0024B07C0024704900243B
:108DA000DF7D0708298D0408E47D07081D01018087
:108DB000007E07081FB5064B6C460FCB84E80F00FA
:108DC0002046FEF749FF034B186004B010BD00BFFA
:108DD000187E0708A87C002473B506460C46154685
:108DE00012F018FF58B90634324628462ABF054B00
:108DF000054953F824100023009312F019FF02B024
:108E000070BD00BFDC7F0708307F070808B500F0A1
:108E1000F7F80000002307B5421E00930023042A40
:108E200019D8DFE802F003080C10140001220C49E5
:108E30000C4812F0FDFE02220B490C48F9E7032210
:108E40000B490C48F5E704220B490C48F1E70522D1
:108E50000B490C48EDE702460B490C48E9E700BF17
:108E6000287E070825010280497E07082601028026
:108E70006E7E070827010280A37E07082801028072
:108E8000DE7E07082A0102801E7F0708000102809B
:108E90000146014AFFF7A0BF31010180014AFFF7F7
:108EA0009BBF00BF32010180014AFFF795BF00BFA1
:108EB00037010180014AFFF78FBF00BF33010180F6
:108EC00011F1110F02D0024AFFF786BF704700BFB1
:108ED00034010180014AFFF77FBF00BF38010180E4
:108EE00010B5FFF795FD034B1B6813B1BDE81040AB
:108EF000184710BDB4490024024B1B6803B1184742
:108F0000704700BFB4490024024B987A003818BF5C
:108F100001207047300C002408B5FEF74DF90022FF
:108F2000064912F093FFC31C04D98B22044905485B
:108F300012F0E6FBBDE80840FEF752B9098F0408BD
:108F40001780070829800708B0F57A7F10B50C460E
:108F500004D0322219491A4812F0D2FB12F086F8D6
:108F60000028184A16DB00F16043F02103F5614345
:108F700083F80013916800F1100341F82340BFF318
:108F80004F8F926852F823309C420AD03F220B49FF
:108F90000D48E1E700F00F03F021043B134419767C
:108FA000E8E7002808DB0123420900F01F0003FA6C
:108FB00000F0064B43F82200002010BD1780070880
:108FC0005680070800ED00E06380070800E100E03C
:108FD00008B512F0C3FEBDE8084012F072B90000F7
:108FE000014B186812F0A2B920690024014B1868DF
:108FF00012F05EB92069002408B512F037F808BDF8
:10900000024C08B523689847FCE700BFD40C002445
:1090100003680BB108461847704710B50446F9F7C6
:109020006CFE204610BD08B5FCF76AFE08BD0000C6
:10903000044B0022C3E901221A611A60024ADA6075
:10904000704700BFB84900241190040810B50022F1
:10905000034600F1110403F8012B03F8012B9C4295
:10906000FBD1418210BD000042F60211024808B552
:10907000FFF7ECFF08BD00BFCC4900240068704733
:1090800008B5F7F774FF08BD10B50446F9F735FECB
:10909000204610BD884238B5044606D00D46F7F785
:1090A00061FF20462946F9F728FE204638BD08B55D
:1090B000F9F700FB0068003818BF012008BD000068
:1090C00070B504460D461646FFF7F1FF28B940F289
:1090D00002220749074812F013FBE068FFF7CEFFB2
:1090E0003246034629462046BDE87040184700BF77
:1090F000B48007084C7B070808B5FFF7E1FF08BDFF
:1091000008B5FFF790FF08BD10B504460021F8F739
:1091100053FB204610BD884238B5044606D00D46A4
:10912000F7F720FF20462946F9F7E7FD204638BD2E
:10913000D0E90032096812F0010F01EB620005D09E
:1091400010B454100A595DF8044BD358184701461F
:10915000043008B5FFF7ECFF08BD0000034A0346E2
:10916000C26007C983E80700704700BFC0800708D6
:1091700010B588B0059108A902AC019001E90C0076
:1091800005A984E80C00FFF7E9FF019808B010BDBD
:1091900037B56C46054684E80C0094E80C00FFF7F0
:1091A000E7FF284603B030BD08B5FFF7D0FF08BD84
:1091B00008B5FFF7F9FF08BD10B504460021F8F720
:1091C000FBFA204610BD10B50446F7F7CBFE20464B
:1091D00010BD08B5F9F76EFA0068003818BF012015
:1091E00008BD00687047884238B5044606D00D4671
:1091F000F7F7B8FE20462946F9F77FFD204638BD2F
:1092000070B504460D461646FFF7E3FF28B940F255
:1092100002220749074812F073FAE068FFF7E1FFFE
:109220003246034629462046BDE87040184700BF35
:10923000B48007084C7B070808B5FFF7E1FF08BDBD
:1092400010B50446F9F759FD204610BD0068704777
:1092500010B50446F7F786FE204610BD10B504464B
:10926000F7F780FE204610BD10B504460021F8F740
:10927000A3FA204610BD08B5F9F71CFA00680038BB
:1092800018BF012008BD884238B5044606D00D46F7
:10929000F7F768FE20462946F9F72FFD204638BD2E
:1092A000884238B5044606D00D46F7F75BFE2046E7
:1092B0002946F9F722FD204638BD08B5F9F7FAF935
:1092C0000068003818BF012008BD10B50446002111
:1092D000F8F772FA204610BD70B504460D46FFF748
:1092E000CAFF28B940F202220649074812F008FADC
:1092F000E068FFF7ABFF294603462046BDE8704013
:10930000184700BFB48007084C7B070808B5FFF773
:10931000E3FF08BD70B504460D46FFF7CEFF28B940
:1093200040F202220649074812F0EAF9E068FFF726
:109330008DFF294603462046BDE87040184700BF10
:10934000B48007084C7B070808B5FFF7E3FF08BDAA
:1093500010B5044613F058FB204610BD10B5084C5C
:10936000204613F011FB00232046064A84F82430DF
:1093700023630549C4E90A33BDE8104012F098BEE2
:10938000E049002400000024519304080268814B46
:109390009A422DE9F04393B040F0F9801EF04AF96B
:1093A00012F0A6FA7C4A0023C2F88430BFF34F8F34
:1093B000536923F480335361BFF34F8FD2F8803069
:1093C00043F6E074C3F3C900C3F34E335B0103EA11
:1093D0000406014646EA81750139C2F87452F9D291
:1093E000203B13F1200FF2D1BFF34F8FBFF36F8FEC
:1093F00012F094FA694B01260025D3F8E0204FF4CF
:1094000000470DA9664842F001024FF030090224DE
:109410004FF00308C3F8E020D3F8E02002F0010287
:109420000192019AD3F8E02042F00402C3F8E02050
:10943000D3F8E02002F004020292029AD3F8E0206E
:1094400042F04002C3F8E020D3F8E02002F04002EE
:109450000392039AD3F8D82042F40042C3F8D820EC
:10946000D3F8D82002F400420492049AD3F8D8200A
:1094700042F48032C3F8D820D3F8D82002F48032E6
:109480000592059AD3F8D82042F40032C3F8D820C8
:10949000D3F8D82002F400320692069AD3F8E020DE
:1094A00042F40072C3F8E020D3F8E03003F4007314
:1094B0000793079BCDE90D76CDE90F5517F012FC08
:1094C0000DA93848CDF8349017F00CFC3246102125
:1094D000344817F0EDFC32462021324817F0E8FC02
:1094E0000DA931480E960D940F9517F0FBFB3246EF
:1094F00021462D4817F0DCFC192015F089FC39466F
:109500002A46274817F0D4FC642015F081FC324627
:109510003946234817F0CCFC0B274FF4605308A9B9
:1095200022480A95CDE90834CDE90B8717F0DAFB1C
:1095300008A91C480C97CDE90844CDE90A5817F052
:10954000D1FB08A917480C97CDE90894CDE90A4842
:1095500017F0C8FB802308A913480C97CDE90834FD
:10956000CDE90A6817F0BEFB042308A90E480C9742
:10957000CDE90834CDE90A4817F0B4FB08A90A4838
:109580000C97CDE90844CDE90A5817F0ABFB13B0AE
:10959000BDE8F0830080024000ED00E00044025886
:1095A000002402580008025800000258001802580F
:1095B00030B570B1CC6864B18A6852B10B6943B1FF
:1095C0000D6849688560C1608361C0E9042400209A
:1095D00030BD4FF0FF30FBE773B50023466804460B
:1095E000019366B1A36998470546A3699847431B51
:1095F000B3F5FA6FF9D901230025636027E083688A
:1096000003B19847202300252360636901AA122132
:109610003046984700281DDB019B03F01F03B3422F
:109620001AD10025266020681F2833D87DB9236908
:109630004FF400422946984700282EDB636901AAAF
:1096400029462068984700280ADA6FF00405284662
:1096500002B070BD6FF004050136202ED5D1E2E7CF
:10966000A36998470646019B1B0402D4002DB9D07C
:10967000EDE7A3699847801BB0F5FA7F07D86369C7
:1096800001AA0021206898470028ECDADDE76FF096
:109690000105E8E76FF00205D9E76FF00305D6E7AB
:1096A00037B500254369044601AA012100680195E8
:1096B0009847A84203DA6FF0040003B030BD636935
:1096C00001AA0121206898470028F4DB019B5B0771
:1096D0002CD5636901AA2946206898470028EADB4F
:1096E000019BDD040ED403F40452B2F5045F01D1F2
:1096F0000220E2E7980401D50320DEE7D90513D55F
:109700000420DAE7636901AA1F212068984700282E
:10971000D1DB019BDA040BD503F01C03182BE7D037
:10972000082BE9D0142BEBD00520C6E70120C4E7B5
:109730000620C2E740F2DC50704700207047062048
:10974000704770477047C0F86C1170470020704731
:109750001FF060BDF0B500F582779FB006460D465C
:10976000384613F019F978220021684626F020FFC8
:1097700000226B462C4611460CB30A2911D1002455
:10978000184A1949022011F0BBF9AB7B012B02D911
:10979000284605F0E0FE384613F01CF920461FB0BD
:1097A000F0BD6068186060890244586009B143F8F0
:1097B000043C246804B99C6001310C33DCE70B499C
:1097C000301D4A603222C1F808D016F009FB03466A
:1097D00028B1074A0220044911F092F9D5E7012483
:1097E000D3E700BFCC800708F38007083C4A002479
:1097F000F8800708032A0846024928BF032226F0FA
:10980000D9BD00BF8B8F070808B5044A082004495A
:1098100011F076F9BDE8084012F05EBB2081070820
:10982000F380070810B5064C06492046FFF7C0FE36
:109830002046FFF7D1FEB0FA80F0400910BD00BF0E
:109840001C4A0024D80C00240148FFF729BF00BFA0
:109850001C4A00240238032815D8DFE800F0020A69
:109860000C114FF400530B604FF480430120136040
:1098700070470023F7E74FF400530B600023F5E730
:1098800000230B60F2E70020704708B500F0F6FAFD
:1098900008BD000030B5051D85B000230C462846E4
:1098A00001A9009316F074FB48B96946284616F0E2
:1098B000BAFB38B1184A0220184911F021F94FF0CB
:1098C000FF3026E0284616F0CBFB0099002911DD79
:1098D000019B03F01F020A44BFF34F8F10481A4444
:1098E000C0F85C322033D11A0029F9DCBFF34F8F66
:1098F000BFF36F8F4FF4C172BDF80010002005F068
:109900005DFE206028B1BDF80020019905F0A3FF9D
:10991000002005B030BD00BF2B810708F380070889
:1099200000ED00E03D200022072108B515F0C4FD40
:109930003D20BDE8084015F0F1BD00207047000053
:109940000022064B1B680270802243714270E122A4
:1099500082701A0CC2701A0A0271704700E8F11F77
:1099600010B50446FFF7E9FF20B92046BDE81040D6
:10997000FFF7E6BF10BD000070B586B0044615F0D5
:10998000EFFD2F492F4B02AD012604342846ADF8D8
:109990000860CDE903134FF08073059315F002FEC4
:1099A00040F201132848ADF80830284BCDE90303F5
:1099B0004FF480332846059315F0F4FD042015F08C
:1099C000DFFD234B28462360FFF7CAFF214B65606C
:1099D00008202361204B2672E36040F2F4531F4AB3
:1099E00063610A231E490093042311F089F820467D
:1099F00016F08EFD054600BB1A4E01463022301D82
:109A000026F0D6FD212333604FF44033C6E90453DA
:109A1000154E2946013532460023204606F5BF661D
:109A200016F04CF9042DF4D1104A08200C4911F01D
:109A300067F8FFF7F7FE06B070BD0020FBE700BF38
:109A40000000043009000003004004300D00000352
:109A500000800240000004300001043056810708F5
:109A6000F38007083C4A0024000404307081070892
:109A7000084608B5FFF774FF012008BD002307B5AD
:109A80001A4602490248009312F0D2F88A81070868
:109A900005001180002307B51A46024902480093C9
:109AA00012F0C6F8BE8107080500118038B50D4BCD
:109AB00000250446036000F5827040F8485C12F00F
:109AC00063FF04F5947012F05FFF04F5A670FFF7D2
:109AD000FCFB04F5AE70FFF7C7FB2046C4F87051DD
:109AE00038BD00BF5882070810B50B4C2378BFF370
:109AF0005B8FDB070ED4204612F0EAFA50B107481C
:109B0000FFF7D4FF204612F005FB054A054903483C
:109B100012F0CEFA014810BD144A0024704A002405
:109B200000000024899B040837B50D4604460192C5
:109B3000FFF7DAFF019B2A462146043016F07AFB34
:109B4000003818BF0120404203B030BD37B50D4684
:109B500004460192FFF7C8FF019B2A4621460430C4
:109B600016F096FB003818BF0120404203B030BD0C
:109B700008B5FFF7B9FF043016F08EFC002008BDD1
:109B800008B5FFF7B1FF08BD0A4B10B504460360E6
:109B900000F5AE70FFF762FB04F5A670FFF758FB07
:109BA00004F5947012F030FF04F5827012F02CFF6F
:109BB000204610BD5882070808B500F5A670FFF7CB
:109BC00062FB08BD08B500F5AE70FFF769FB08BD84
:109BD000F0B59DB00446FFF737FE01280546D4F8DE
:109BE000707139DD012F18DC01AA02A9FFF732FEDE
:109BF00018B94FF40053CDE90130261D03A93046B2
:109C000016F078FB019B03A930460993029B089349
:109C100016F036FC304616F06FF804F5AE76304696
:109C2000FFF729FB60B1012D0EDD012F08DC0121BA
:109C30003046FFF76BFB114A1149082010F060FF16
:109C4000C4F870511DB0F0BD012FF9DD0021304680
:109C5000FFF75CFB0B4AEFE7012FDEDD0A4B4FF00D
:109C60000052C3F88420BFF34F8FBFF36F8F201DC6
:109C700016F08CF82046FFF755FECEE7F281070874
:109C8000F38007081182070800E100E073B504467D
:109C9000002600F594752846019612F07DFE01A974
:109CA0002046FFF7F7FD002804DA284612F092FE5E
:109CB00002B070BD019919B104F5A670FFF744FB1D
:109CC000284612F087FEE6E738B50E4C05462378A5
:109CD000BFF35B8FDA0708D4204612F0F9F920B100
:109CE000094B20461D6012F015FA074C4FF0FF3269
:109CF00000210120FEF70AFFC307F7D52068FFF710
:109D0000C5FFF3E7184A0024E84B0024D0E90032ED
:109D1000096812F0010F01EB620005D010B4541075
:109D20000A595DF8044BD35818470146043008B56A
:109D3000FFF7ECFF08BD0000034A0346C26007C9F5
:109D400083E80700704700BF4482070810B588B059
:109D5000059108A902AC019001E90C0005A984E86D
:109D60000C00FFF7E9FF019808B010BD37B56C464D
:109D7000054684E80C0094E80C00FFF7E7FF28464E
:109D800003B030BDF0B505468DB012F08FF828460F
:109D9000FFF7F2FD064600284ED02022002104A83D
:109DA00026F006FC264B4FF40060039325F0B4FF29
:109DB00005F1C00303AA2946079005934FF40063F9
:109DC000204808934423069328230993FEF708FEAE
:109DD000C5F8BC0010F0B4F91B4B07461A4A0193B2
:109DE0000023294603A80293FFF7C0FF102138463D
:109DF0000FF052FF0446A0B103A9FFF745F9204632
:109E0000C82110F0ECF82046C82110F0EBF82046ED
:109E10000E4910F0EAF822460D4938460FF0FCFFD3
:109E2000044603A8C5F87441F7F7A1F80A20FCF727
:109E3000B1FD2846FFF776FD30460DB0F0BD00BFFE
:109E400031820708C99C0408D19B0408819004084A
:109E50000191040808B5FFF768FF08BD08B5FFF7D2
:109E6000F9FF08BD08B5FFF73FFED0F8BC0020B1F0
:109E70000121BDE80840FEF70FBE08BD08B5FFF799
:109E800033FE0430BDE8084016F030B910B5044682
:109E9000FBF772FF204610BD0858704730B55518C3
:109EA00054586B6804B1601843601C60014B5350F8
:109EB0006B6030BDEFBEADDE00224FF00A0C2DE925
:109EC000F0430746964610464FF02E080B18BE5C2E
:109ED0001D462C46B6FBFCF90CFB1960303005F82A
:109EE000010B30465FFA89F60928F2D885F800E0C0
:109EF0001D46AC4210D81C46581A01332578002D57
:109F0000F9D1032A02F101021CBF013084F800805C
:109F1000042ADBD1BDE8F08320782E7804F80169AB
:109F200005F8010BE5E71029F0B501D90020F0BDD7
:109F3000561E002403320A278C42F7D0035D303BC3
:109F4000092BF3D8234600248B420BD306F8014F8C
:109F5000964214D18B4217BFC05C0120B0FA80F04A
:109F60004009E4E7C55C303D5FFA85FCBCF1090FB0
:109F7000ECD807FB04540133FF2CE5D9D6E78B421C
:109F8000D4D05C1CC35C2E2BD6D0CFE72DE9F84F84
:109F90000F460546014600234FF001084FF0FF0928
:109FA00031F8022B5ABB5A1C072A21D9D01A404536
:109FB00001D980469946531C072BF1D94FEA480B2B
:109FC0003C46002618494FF03A0AB14519D1B9F17B
:109FD000000F01D104F801AB464423465D44072E2F
:109FE00003F801AB1DD90022D81B1A70BDE8F88F09
:109FF00031F8024B501C002CD8D10246D4E71A4647
:10A00000D9E72A880136204652BA92B226F090FD4E
:10A01000082E04EB0003E6D002350133024904F8B0
:10A0200000A01C46D1E700BF589F070827292DE94B
:10A03000F0410646104656D91022002126F0B8FA03
:10A040000020BDE8F08124F0200E3A46AEF1410E2A
:10A05000BEF1050F02D9303C092CEDD8013905D0ED
:10A060003A4617F8014B0CB13A2CECD1941B042C56
:10A07000E2DC082BE0D0002716F8014BA4F1300EEB
:10A080005FFA8EF8B8F1090F03D84EEA0714A7B2A9
:10A09000F2E7A4F1410EBEF1050F03D8373C44EAC4
:10A0A0000714F4E7A4F1610EBEF1050F01D8573C87
:10A0B000F5E73C0A00F813400CF81370013351B176
:10A0C00014783A2C0DD154783A2C0AD10135B3D1F9
:10A0D000013202391D46561C59B132784AB1374611
:10A0E000BEE70139F7E74FF0FF35002302F1010C1D
:10A0F000F2E76A1C13D0C3F108035C0004EB4503CC
:10A1000000EB4505C3F110021844294626F0ECF98E
:10A1100022460021284626F04BFA012091E7082B21
:10A120008AD1FAE72DE9F04F8DB04B68D74A0193F9
:10A130008B68D1F800A00293CB68D1F814E00393A8
:10A140000B69D1F81C9004938B69D1F830C005934A
:10A150000B6AD1F8388006934B6AC66807938B6AFE
:10A16000CB4D0893CB6A3544DFF8ACB309934B6B06
:10A17000E3440A93CB6B0B9383681A44D0E9043110
:10A1800052444B4033404B401344C24A0A44019965
:10A1900006EB736304690A440169049F7140194026
:10A1A00061401144BC4A2244029C03EB31512244D9
:10A1B00086EA03040C4074401444039A01EBF4341F
:10A1C000154483EA010222405A402A44B34D3D44DB
:10A1D00004EBB222059F1D4481EA040313404B4067
:10A1E0002B44AF4D754402EB73630D4484EA0201C6
:10A1F000194061402944AB4D3D4403EB3151069F6A
:10A20000254482EA03040C4054402C44A64D4D449E
:10A2100001EBF434154483EA010222405A402A44F7
:10A22000A24D3D4404EBB222079F1D4481EA040382
:10A2300013404B402B449E4D3D4402EB7363099FFA
:10A240000D4484EA0201194061402944089DA5F5A6
:10A25000244503EB31514F3D254482EA03040C4071
:10A2600054402C44934D3D4401EBF4340A9F154473
:10A2700083EA010222405A402A448F4D654404EB90
:10A28000B2221D4481EA040313404B402B448B4D02
:10A290003D4402EB73630B9F0D4484EA02011940B5
:10A2A00061402944864D454403EB3151254482EAFF
:10A2B00003040C4054402C44824D3D4401EBF434E3
:10A2C000019F154483EA010222405A402A447E4DF0
:10A2D00004EBB2223D44059F1D4484EA02030B4077
:10A2E00063402B44794D02EBF3633D44099F0D44D9
:10A2F00082EA0301214051402944754D03EBF1519D
:10A300003D44089F254483EA010414405C402C44EA
:10A31000704D01EBB4445544154481EA04021A40DF
:10A320004A402A446C4D04EB323275441D4484EAA1
:10A3300002030B4063402B44684D02EBF3633D4442
:10A340000B9F0D4482EA0301214051402944644D92
:10A3500003EBF1513D44049F254483EA010414407A
:10A360005C402C445F4D01EBB4443D44079F1544D1
:10A3700081EA04021A404A402A445B4D04EB32321F
:10A380003D44039F1D4484EA02030B4063402B4479
:10A39000564D02EBF36345440D4482EA030121402C
:10A3A00051402944524D03EBF1513D44069F2C444A
:10A3B00083EA010515405D402C444E4D01EBB44449
:10A3C0003D440A9F2A4481EA04051D404D402A4429
:10A3D000494D04EB32323D44029F2B4484EA02058E
:10A3E00093440D4065402B44444D02EBF3633D44E0
:10A3F000069F294482EA0305254055402944404DE3
:10A4000003EBF1514D442C4483EA010515405D40B6
:10A41000254401EBB54581EA050404EA03024A40FC
:10A420005A44AEF5B82B05EB3232ABF2BE6B54405A
:10A430005B442344334C3C4402EB3373099F0C448C
:10A4400085EA0201594021442F4C3C4403EB7151F1
:10A45000019F254482EA03044C4025442B4C44448C
:10A4600001EB3545144483EA01026A402244284C3A
:10A470003C4405EB7222049F1C4481EA05035340CF
:10A480002344244C3C4402EB337347E078A46AD75E
:10A49000EECEBDC156B7C7E8DB702024AF0F7CF508
:10A4A0002AC68747134630A8019546FDD89880698B
:10A4B000AFF7448BBED75C892211906B937198FDE6
:10A4C0008E4379A62108B44962251EF640B340C0E8
:10A4D000515A5E26AAC7B6E95D102FD6531444021E
:10A4E00081E6A1D8C8FBD3E7E6CDE121D60737C383
:10A4F000870DD5F4ED145A4505E9E3A9F8A3EFFC5F
:10A50000D9026F6781F6718722619D6D0C38E5FD78
:10A5100044EABEA4A9CFDE4B8A4C2A8D089F0C4486
:10A5200085EA020159402144894C4C4403EB7151A6
:10A53000254482EA03044C402C44864D3D4401EB03
:10A5400034440A9F154483EA010262402A44824D42
:10A550003D4404EB7222039F1D4481EA04035340EF
:10A560002B447E4D554402EB3373294484EA0205A3
:10A570005D4029447A4D3D4403EB7151059F2544CC
:10A5800082EA03044C402C44764D3D4401EB3444B4
:10A59000079F2A4483EA010565401544724A3A44FC
:10A5A00004EB75250B9F134481EA04026A401A44A8
:10A5B0006E4B634405EB32720B4484EA0501514053
:10A5C00019446B4B3B4402EB7151029F1C4485EADA
:10A5D00002034B401C44674B3B4401EB3444039F54
:10A5E0001D4482EA010363402B44634D04EB732353
:10A5F000554463EA010A2A44604D8AEA040A4D443C
:10A60000524429445E4D03EBB262454462EA0409B8
:10A610002C445C4D89EA03097544494402EBB1516D
:10A6200061EA03082B44584D88EA02086544444413
:10A6300001EB744464EA020E2A44544D8EEA010E82
:10A640003D44734404EBF32363EA010C2944089D61
:10A650008CEA040CA5F580156244A5F6833503EB5E
:10A66000B262254462EA04075F403944019F02EB6D
:10A67000B15161EA030454402C44454D01EB74444C
:10A680003D4464EA02072B44424D4F403B44069F41
:10A6900004EBF3233D4463EA01072A440B9D674022
:10A6A0003A443D4F03EBB2622F443C4D62EA040C46
:10A6B0003944059F8CEA030C3D4461442C44384DD9
:10A6C00002EBB15161EA030757403C440A9F01EB9A
:10A6D00074443D44049F1D4464EA02034B402B44F0
:10A6E000304D04EBF3233D442F4F154463EA010240
:10A6F00062402A44099D03EBB2622F442B4D0F4464
:10A7000062EA040159403944029F02EBB1513D44D1
:10A71000079F254461EA030454402C44244D3D44E2
:10A7200001EB74442B4485682644154464EA020214
:10A730004A4085601A4403691C44436906EBF226CB
:10A7400019440461C66041610DB0BDE8F08F00BFDF
:10A75000604BBBF670BCBFBEC67E9B28FA27A1EA41
:10A760008530EFD4051D880439D0D4D9E599DBE6CE
:10A77000F87CA21F6556ACC4442229F497FF2A43F3
:10A78000A72394AB39A093FCC3595B6592CC0C8F83
:10A79000D15D84854F7EA86FE0E62CFE144301A3B3
:10A7A000A111084E827E53F735F23ABDBBD2D72AAB
:10A7B00091D386EB0023C0E90033084B836003F19B
:10A7C0008833C36003F12943A3F59613A3F68B6383
:10A7D0000361A3F188334361704700BF01234567DC
:10A7E0002DE9F843141E05460E4630DD036803F0DC
:10A7F0003F071B19036022BF43680133436097B1D1
:10A80000C7F1400844450EDB00F1180942464644B2
:10A81000A4EB080409EB0700002725F0CBFD49460F
:10A820002846FFF77FFC264403E0403C2846FFF71C
:10A8300079FC3F2CA6EB0401F7DC002C07DD05F1C9
:10A84000180022463844BDE8F84325F0B3BDBDE802
:10A85000F883000037B50D460446D0E90021530FB8
:10A8600043EAC103D10002F03F02372ACDE90013C9
:10A8700094BFC2F13802C2F178021749FFF7B0FF66
:10A88000082269462046FFF7ABFFA3682B70A36838
:10A890001B0A6B706389AB70E37AEB70E3682B7112
:10A8A000E3681B0A6B71E389AB71E37BEB7123698E
:10A8B0002B7223691B0A6B72638AAB72E37CEB72A7
:10A8C00063692B7363691B0A6B73E38AAB73E37D64
:10A8D000EB7303B030BD00BF9482070810B50022AF
:10A8E00010F0010304D0A1B310F8012B12020139BA
:10A8F00010F0030405D002291ADB30F8024B1219BC
:10A90000023908290BDB50F8044B121942F10002FE
:10A9100050F8044B121942F100020839F1E70229FC
:10A9200006DB30F8024B121942F100020239F6E759
:10A9300019B10478121942F10002C2F30F44C2F3B4
:10A940000F021219C2F30F44C2F30F02121903B11E
:10A9500052BA104610BD130911D051F804CB40F87B
:10A9600004CB51F804CB40F804CB51F804CB40F8A9
:10A9700004CB51F804CB40F804CB013BEDD112F0ED
:10A980000F0305D011F801CB00F801CB013BF9D141
:10A990007047000008290A4613B5044605DD002368
:10A9A0000F491048009311F043F94822002125F087
:10A9B000FFFD04F11403201DE36010232361FCF765
:10A9C00055F90346206020B9009022460649074801
:10A9D000E9E70221FCF762F9002002B010BD00BFD8
:10A9E000D482070805010380ED8207080F01038068
:10A9F00007B590F8252090F82430934205D0002325
:10AA000003490448009311F013F903B05DF804FB07
:10AA1000088307080401038002224FF0FF3370B55A
:10AA200004460E4600681146FCF77CF9FCF796FBDD
:10AA300094F824300546012103F10A02013303F0A2
:10AA4000070344F82260206884F82430FCF726F9D4
:10AA500094F8243094F82520013303F0070393423F
:10AA600003D102212068FCF747F92846BDE8704071
:10AA7000FCF78ABB0222002373B504460E46006829
:10AA80001146FCF74FF9021E01DB930709D400239E
:10AA900016491748009311F0C3F84FF0FF3002B089
:10AAA00070BDFCF75BFB94F824300546012103F1EF
:10AAB0000A02013303F0070344F82260206884F897
:10AAC0002430FCF7EBF894F8243094F82520013377
:10AAD00003F00703934203D102212068FCF70CF92D
:10AAE0002846FCF751FB0020D9E700BF1D8307086B
:10AAF0000F010380F7B5174604460E46FCF786FBA8
:10AB0000002F4FF0020205464FF0010114BF3B46F3
:10AB10004FF0FF332068FCF705F9021E01DBD30775
:10AB200009D4002317491848009311F079F84FF021
:10AB3000FF3003B0F0BDFCF711FB07462EB194F8CF
:10AB400025300A3354F82330336094F8253002213D
:10AB50002068013303F0070384F82530FCF79EF8E2
:10AB600094F8242094F825309A4203D101212068DA
:10AB7000FCF7C2F83846FCF707FBFCF747FB401B25
:10AB8000D7E700BF358307080D01038073B50222A4
:10AB900004460D46002301210068FCF7C3F8021E9D
:10ABA00001DBD30709D4002316491748009311F09D
:10ABB00037F84FF0FF3002B070BDFCF7CFFA064611
:10ABC0002DB194F825300A3354F823302B6094F8D3
:10ABD000253002212068013303F0070384F8253073
:10ABE000FCF75CF894F8242094F825309A4203D1BD
:10ABF00001212068FCF780F83046FCF7C5FA0020F8
:10AC0000D9E700BF538307080F01038037B5044617
:10AC10000D462422002125F0CBFC04F11403221D53
:10AC20002946E36010234FF6FF702361FDF78AF990
:10AC30000346206028B9009022460349034810F0DB
:10AC4000F7FF002003B030BD718307080F010380B8
:10AC500073B50D460446FCF7D9FA0646002D206868
:10AC600014BF29464FF0FF31FDF784F950B100239E
:10AC7000224606490648009310F0D2FF4FF0FF30FD
:10AC800002B070BDFCF7C2FA801BF9E78B8307089E
:10AC90000D01038013B504460068FDF793F930B148
:10ACA0000023226803490448009310F0C1FF02B05A
:10ACB00010BD00BFA783070816010380704700007E
:10ACC00013B530220021044625F072FC0C4B201DE8
:10ACD000636004F11403E3601C232361FCF7BCFFF1
:10ACE0000346206048B9009022460649064810F005
:10ACF00097FF4FF0FF3002B010BD0020FBE700BF10
:10AD0000BD830708C88307080F01038013B50446F5
:10AD10004FF0FF310068FCF7B7FF30B10023224647
:10AD200003490448009310F083FF02B010BD00BF38
:10AD3000DD8307081501038013B504460068FCF79E
:10AD4000BBFF30B10023224603490448009310F0B2
:10AD50006FFF02B010BD00BFF38307081701038027
:10AD600007B50C4B0C4803600C4B83601C23C3607D
:10AD700003234360FCF770FF094B186030B90346AA
:10AD8000024600900749084810F052FF03B05DF8F2
:10AD900004FB00BF0B84070810FD0024F4FC002412
:10ADA000F0FC00241A8407081D010380094B07B535
:10ADB0004FF0FF311868FCF767FF30B100230649F8
:10ADC00006481A46009310F033FF012003B05DF8E7
:10ADD00004FB00BFF0FC0024478407081501038032
:10ADE000074B07B51868FCF767FF30B1002305492A
:10ADF00005481A46009310F01BFF03B05DF804FBF2
:10AE0000F0FC00245F84070817010380FCF7FEB9FB
:10AE100008B5FDF7FDFD014B186008BDEC4B0024A3
:10AE200008B5FDF7F5FD034B1B681B1A5842584146
:10AE300008BD00BFEC4B00242DE9F34782462348B0
:10AE40009146884602681D46052A04DD00232049F4
:10AE50000093204827E06C211F4F01FB02F60132CE
:10AE6000BC1902600A460021204625F0A1FB1B4BBD
:10AE70002846A561BAF1000F08BF9A460A9BE36114
:10AE80004423C4F804A0236106F128033B44E36093
:10AE900024F042FF00236061236230B90346009032
:10AEA0002A460F490F4810F0C3FE321D494640465E
:10AEB0003A44FDF795FD0346B85118B902460A49D0
:10AEC0000090C6E7204602B0BDE8F087784E002427
:10AED0008D8407082D010380F04B00247984070836
:10AEE000AA8407081F010380CB8407080FF0A4BEC3
:10AEF0000FF014BE0FF0FABE38B5094B0D460446EC
:10AF000040221846002125F053FB10222946243008
:10AF1000FFF721FD034B5C43034B1C6038BD00BFB2
:10AF2000804E002490D003007C4E002470B51C4C51
:10AF30000025FF269CB0256065602581A672E6721B
:10AF400000682561E06006A865612583A676E6763F
:10AF5000126884F82330E2610A0A84F8211084F828
:10AF600020201A0A84F82220FFF724FC40222146E0
:10AF700006A8FFF735FC02A906A8FFF76BFC042220
:10AF800002A90DEB0200FFF7E6FC064B1C68019BD3
:10AF90001C44FFF73BFFFA2303FB00401CB070BDCD
:10AFA000804E00247C4E002438B505460C46FFF741
:10AFB00037FF20B12046A84794F9040007E0226833
:10AFC000214628460C3201F0ABF90028F4D038BDF8
:10AFD00000B589B060B1292300908DF8081069464A
:10AFE00005488DF80930FFF7DFFF09B05DF804FB75
:10AFF0006FF00F00F9E700BFC5C0040830B50D467B
:10B0000089B0114600F0A0FD0446A0B10090694649
:10B010000A488DF80850FFF7C7FF60B104F10C0033
:10B02000FFF74CFE04F13000FFF7E2FC214600245C
:10B03000072004F053F8204609B030BDE9BA0408EF
:10B0400000B589B038B129230090694603488DF8CE
:10B050000930FFF7A9FF09B05DF804FB2DBD040816
:10B0600038B5054640B1FFF7EBFF044610B9284656
:10B0700000F09AFD204638BD0446FBE700B589B0D4
:10B0800068B161B15AB1009006488DF81030CDE931
:10B0900002126946FFF788FF09B05DF804FB6FF004
:10B0A0000F00F9E76DC0040800B589B070B1094B15
:10B0B0000090002908BF19460748ADF80C200291FE
:10B0C0006946FFF771FF09B05DF804FB6FF00F00F0
:10B0D000F9E700BF08850708CDBD040800B589B0B1
:10B0E00048B100908DF80E1069460448FFF75CFFE8
:10B0F00009B05DF804FB6FF00F00F9E701BE04082A
:10B1000000B589B070B1094B0090002908BF1946FD
:10B110000748ADF80C2002916946FFF745FF09B0DA
:10B120005DF804FB6FF00F00F9E700BF0885070822
:10B1300039BE040800B589B038B1009069460448AA
:10B14000FFF732FF09B05DF804FB6FF00F00F9E77D
:10B15000EDBE040800B589B040B100900291694687
:10B160000448FFF721FF09B05DF804FB6FF00F0002
:10B17000F9E700BF91BF040829B102B112688A60E3
:10B180008B81FFF7E7BF6FF005007047F0B589B01E
:10B190000E9E002837D0047804F0F004102C35D12E
:10B1A00090F8C04003F0040504F002042C4301D0E1
:10B1B00066B30024254601F1040C04E05CF8347009
:10B1C0007D1923D20134A242F8DC002D02D10020E7
:10B1D00009B0F0BD02DACEB16FF00045ADF80C2039
:10B1E00000220090029169460A4804928DF81C30B2
:10B1F000CDE90552FFF7D8FE0028E9D1002EE6D0B0
:10B20000069B3360E4E76FF00F00E1E76FF00500A5
:10B21000DEE700BF05C004081FB5CDE90212069A9B
:10B2200002A900920122FFF7B1FF05B05DF804FB0F
:10B2300038B5044648B1FFF7B9FD002394F908502A
:10B240002372FFF7CDFD284638BD0546FBE773B5F1
:10B2500005460E4621B96FF00F04204602B070BDBE
:10B2600000230B600028F6D0FFF7E2FF04468DF8BC
:10B2700003000028F1D1AB6F13B96FF00E04ECE7B7
:10B2800095F8C030DA07F8D49B0705F1780007D5A8
:10B2900001A9FFF77BFC013006D16FF00604DCE763
:10B2A000224601A9FFF726FCD5F8C8301BB10022C1
:10B2B0000121284698470DF10301019800F0FAFB9F
:10B2C00010B19DF90340C8E7019B002BD5D0336036
:10B2D000C3E7002337B504460D46019319B96FF053
:10B2E0000F0003B030BD0B600028F8D0036B33B9FA
:10B2F000FFF79EFF0028F4D16FF00A00F1E794F801
:10B30000C03002F00402303001A903F003031343FC
:10B3100002D194F908207AB1FFF738FC01300DD141
:10B320002046FFF785FF0028DBD194F8C030DB070B
:10B33000E2D46FF00600D4E7FFF7DCFB2378019836
:10B3400003F0F003102B17D10DF1030100F0B2FB55
:10B3500030B19DF9030010F10F0F08BF0020C0E7C6
:10B36000019B1A89D4F8C83013B1012120469847AF
:10B37000019B00202B60B4E70368F2E7036BF0B594
:10B38000044689B00F461646002B45D090F9C050B0
:10B3900090F8C030002D14DA03F07F0380F8C0303D
:10B3A000D4F8C8301BB100220121204698476368B9
:10B3B0005BBB2046FFF73CFF051E08BF6FF00D0585
:10B3C0001EE0FFF786FF0546D0B932073F680CD470
:10B3D000CFB13A89237803F0F003102B05D16946E9
:10B3E0000F4800940292FFF7DFFD4FB9F306D7D55F
:10B3F00094F8C0306FF0060563F07F0384F8C03026
:10B40000284609B0F0BD0122E4E7012120466FF093
:10B410000E05FFF7DDFDF3E76FF00A05F0E700BF6B
:10B42000CDBF040838B1037803F0F003102B02D12C
:10B430000022FFF7A3BF6FF00F007047F7B5044677
:10B440000E4621B96FF00F04204603B0F0BD00276F
:10B450000F600028F6D0037803F0F003102B1BD107
:10B460000620019703F02EFE054690B120463A468D
:10B4700001A9FFF783FF044620B12946062003F007
:10B480002DFEE1E7019BA881A860C5E90033356086
:10B49000DAE74FF0FF34D7E73A46FFF71AFF0446E2
:10B4A000D2E7002A14BF0223002300290CBF19464B
:10B4B00043F00101FFF78CBD2DE9F34117461D460E
:10B4C000BDF82080064628B9384602B0BDE8F041F4
:10B4D00004F041B8036B002BF6D0062003F0F2FD18
:10B4E00004460028F0D0C0E9007705B12D683A89FC
:10B4F000214606F13000A560A4F80C800192FFF708
:10B50000B9FA019A014628B1204602B0BDE8F041DF
:10B5100000F01ABED6F8C83023B1304602B0BDE8FC
:10B52000F041184702B0BDE8F081000007B50146C0
:10B530004068019004F041FB0198094904F040FB88
:10B540000198084904F040FB01980222064904F0E2
:10B5500049FB0649019803B05DF804EB04F038BBE1
:10B5600055BA040803BA0408A1B9040871B504085F
:10B57000F7B504460D46FFF719FC002794F8C030D4
:10B58000667843F001036760257284F8C030677005
:10B59000FFF726FCD4F8C8301BB13A4604212046F8
:10B5A0009847D4F8C8301BB100222046114698476E
:10B5B000D4F8C8301BB1002202212046984705F17B
:10B5C0000F03DBB2022B96BF1A4A002152F8231058
:10B5D000236B2BB104F130000191FFF74BFA019975
:10B5E000A36F1BB104F17800FFF744FA012E02D0DB
:10B5F000F31E012B1BD894F8C03023F0040213F083
:10B60000040384F8C02012D1D4F8C420042E10689A
:10B6100008BF13714FF0000300F10C0018BF157143
:10B62000C4F8C43003B0BDE8F040FFF733BB03B04B
:10B63000F0BD00BFE884070870B5054638B3D0F800
:10B64000C44014B1227124680C342B7803F0F00349
:10B65000102B03D112B92846FFF768FF95F8C030C8
:10B66000002203F0040623F00403C5F8C42085F883
:10B67000C030D5F8C8306A7013B102212846984707
:10B680001EB920462CB1FFF705FB002001E06FF04A
:10B69000050070BDD0F8C4302DE9F74F1B7F04467C
:10B6A00090F8C060884603F004024FF6FF7B06F076
:10B6B00002061643D4F8C450AA6828691168526873
:10B6C0000144121A6068B2F5803FB0F864702ABF76
:10B6D0004FF6FF791FFA82F943F00203B94542D9C8
:10B6E000002E3CD0002F3CD1AB69002B0CBF6FF07B
:10B6F00006050025D4F8C430D3E905329A426CD24D
:10B70000D4F8C8301BB1002203212046984794F892
:10B71000C03043F0100384F8C030002D72D1D4F84B
:10B72000C430D3E905329A426AD0003E18BF0126E0
:10B73000606806F055FC043077D16FF00305D4F84B
:10B74000C4301D7100251868C4F8C4506570B8F184
:10B75000000F70D00C30FFF79DFA28465CE043F0F4
:10B760000203B94604E0D94502D1B2F5803F05D2C3
:10B7700092B24A4526D1AA89012A23D943F002036D
:10B780004FF0010A4A46019306F011F90546E0B967
:10B79000D4F8C470019BBA69B9684A444868BA6170
:10B7A0003A694A4482423A6107D1BA89013A92B26F
:10B7B000BA8112B108313D61B960BAF1000F7FF46E
:10B7C00079AF08E04FF0000ADCE7431CDBB2012B45
:10B7D000B5D84FF0FF35002E8CD16368B3F86420E4
:10B7E000B2F5866F03D3B3F86630042B95D9D4F83D
:10B7F000C830002B91D000220321204698478CE7C7
:10B80000012695E76B1C9AD1606806F0E9FB0430CD
:10B8100093D026B94FF0FF3003B0BDE8F08FD4F8D5
:10B82000C4309B6923B1002589E7002EFBD1F1E7E5
:10B830006FF0060583E74046EEE700002DE9F84F7C
:10B84000D0F8C4300546894644681B7A032B03F0C0
:10B85000010A03F002080FD0BAF1000F05D0237DD2
:10B860005A1F012A08D9082B06D0B8F1000F16D0AC
:10B87000678B17F0100704D001270021204604F041
:10B880009CF9237D012B0CD10021204604F0A4F962
:10B8900027BB42465146204604F04AFD21E0474678
:10B8A000EFE7BAF1000F07D00021204604F088F935
:10B8B0000021204604F090F9B8F1000F03D00021D8
:10B8C000204604F081F9002FE3D0002220461146E3
:10B8D00004F088F90021204604F07AF9204604F0AB
:10B8E0008BFC064668B1431C0BD1D5F8C43093F8E5
:10B8F00009B0BBF1000F35D11FB15E46204604F000
:10B90000F1FAD5F8C4301C681E710023C5F8C430A4
:10B910006B70E6B93FB1D5F8C8306E601BB13246E6
:10B92000042128469847BAF1000F06D0D5F8C83050
:10B930001BB10022284611469847B8F1000F06D0E7
:10B94000D5F8C8301BB10022022128469847B9F12A
:10B95000000F1CD0002604F10C00FFF79BF93046C5
:10B96000BDE8F88FB8F1000F03D00A49204604F073
:10B970002BF901222046084904F034F920460749F2
:10B9800004F026F92946204604F017F9E7E74E4669
:10B99000E5E700BF03BA0408A1B9040871B50408BB
:10B9A00010B54178044601291DD1FFF773FE94F8C4
:10B9B000C030DA0615D562689AB1B2F86410B1F5F4
:10B9C000866F0ED3B2F86620042A0AD823F010033B
:10B9D00084F8C030D4F8C8301BB1002202212046C0
:10B9E0009847002010BD0429E1D1D0F8C4201AB135
:10B9F000537A0BB1013B537201212046FFF71EFF22
:10BA0000D5E738B515460446E0B1417801291BD188
:10BA1000FFF740FE6368ABB1B3F86420B2F5866F00
:10BA200010D3B3F86630042B0CD894F8C03023F050
:10BA3000100384F8C030D4F8C8301BB12A46022164
:10BA400020469847002038BD0429E3D10121FFF7A3
:10BA5000F5FEDFE7F8B50646154608460EB3346B2B
:10BA600054B912B900242046F8BD118904F058F8E1
:10BA7000284603F070FDF6E782B11789294606F1E2
:10BA80003000FEF7F7FF044670B9D6F8C830002B37
:10BA9000E8D001463A4630469847E4E7044D174659
:10BAA000ECE76FF00504DEE74FF0FF34DBE700BFA3
:10BAB000F5840708094B984203D1F32301200B704A
:10BAC0007047074B984201D1F223F7E7054B9842A4
:10BAD00001D1F123F2E70020704700BFF48407088A
:10BAE000F6840708F584070838B50023056804467E
:10BAF0000371686828BB2B7803F0F003102B14D077
:10BB0000202B1CD106F04BFF22686860506850B1B2
:10BB100013780C49222B04BF0123037406F012FF93
:10BB200023685B686BB9FF230AE004F0D5FA68600C
:10BB300020684368002BF6D0FFF7F8FCF0E7FA2303
:10BB4000237138BDB9B4040870B5054607200E4608
:10BB500003F0B8FA044628B3057005F0F005002399
:10BB6000102D0372436001D0202D0FD104F1300558
:10BB700000212846FEF70EFF014638B904F10C00FB
:10BB8000FFF744F840B12846FEF732FF2146072070
:10BB9000002403F0A3FA05E0A067607084F8C000F9
:10BBA000C4E93106204670BD10B504460C30FFF7DD
:10BBB00085F8002321460720E360BDE8104003F02C
:10BBC0008DBA036BF7B5044663B100F1300501A9E6
:10BBD0002846FEF7DBFF013015D12846FEF708FFA7
:10BBE00000232363A36F63B104F1780701A93846EA
:10BBF000FEF7CCFF013019D13846FEF7F9FE0023DD
:10BC0000A36703B0F0BD2378019803F0F003102B75
:10BC100009D10DF10301FFF74DFF0028D7D101989D
:10BC200003F099FCD3E700F08FFAD0E70DF10301A0
:10BC30000198FFF73FFF06460028D7D1019D28460F
:10BC4000FFF7BFFF686810B104F04CF96E6028463A
:10BC5000FFF7AAFFCAE70000F7B50D46044620B972
:10BC60006FF00505284603B0F0BD836F002BF7D0B9
:10BC700000F1780771B92C493846FEF7FBFE024601
:10BC80000028EDD1D4F8C830002BE9D00146204679
:10BC90009847E5E7D0F8C8100078FFF755FF06464B
:10BCA00070B921493846FEF7E5FE024628B9D4F8B6
:10BCB000C83013B10146204698474FF0FF35D1E711
:10BCC0004560FFF733FC31463846FEF7D3FE0546A4
:10BCD00000B3706800210024019003F06EFF01980A
:10BCE000002103F06DFF0198002103F06DFF002299
:10BCF0000198114603F076FF0021019803F068FFD8
:10BD000006F130007460FEF773FE30463463FFF7CF
:10BD10004BFFD2E7D4F8C830002BA3D0024601462F
:10BD2000204698479EE700BFF484070870B5044694
:10BD30000068437813F0FD0F08D0032B03D190F86F
:10BD4000C0305B0702D4FB23237170BD0025257131
:10BD5000FFF737FF2368586860B11A7802F0F002E5
:10BD6000102A18D0202A02D1456206F0EFFD236880
:10BD700000225A602068D0F8C83013B10022114662
:10BD800098472068D0F8C830002BDED0002202216E
:10BD9000BDE8704018470422294618465A7003220D
:10BDA0002272C3F8C440FFF749FD0028CDD00648F1
:10BDB000FEF7C2FF206829460C30FEF749FF024813
:10BDC000BDE87040FEF7A2BF20FD0024036810B557
:10BDD0000446586888B11B7803F0F003102B07D095
:10BDE000202B0AD1A289A16806F032FC207110BD77
:10BDF000A289A16803F0BAFDF8E76FF00500F5E746
:10BE000010B50446807B03F0E1FA014688B123684F
:10BE1000586870B11B7803F0F003102B06D0202B6C
:10BE200007D106F05FFD0023237110BD03F0EEFD86
:10BE3000F9E76FF00503F7E7036813B504465868A0
:10BE4000002842D01A7802F0F002102A08D0202AE6
:10BE50003ED1A289A16806F04DFD207102B010BD4F
:10BE60005A78032A37D0002A38D11846FFF75EFBEC
:10BE700020681C4BA289A168406803F0C9FE002815
:10BE8000EBD12268032192F8C030517013F0020107
:10BE900006D043F004036FF0040082F8C030DCE702
:10BEA00023F00403C2F8C4400F4882F8C030019167
:10BEB000FEF742FF206801990C30FEF7C9FE0A48E0
:10BEC00002B0BDE81040FEF721BF6FF00E00C4E7DE
:10BED0006FF00500C1E76FF00800BEE76FF00900E2
:10BEE000BBE700BF39B6040820FD0024036873B522
:10BEF00004465868002845D01A7802F0F002102A4B
:10BF000042D15B78002B39D1067D1EB1FA238DF822
:10BF1000073020E00DF10702FF2103F07FFD054609
:10BF2000C8B12068036B23B13030FEF761FD236890
:10BF30001E6320680023866F8DF8073086B1216864
:10BF4000022328464B704D6003F037FE23680F49EB
:10BF5000586803F041FE9DF80730237102B070BDB0
:10BF600031467830FEF716FD8DF807000028E6D040
:10BF7000284604F041F923685E60ECE7022B01D10A
:10BF80000023C4E7F523C2E7F023C0E759BC040847
:10BF900010B504460068FFF74BF968B92368586884
:10BFA00088B11B7803F0F003202B0CD1A2689368B2
:10BFB00011681BB906F08CFC207110BD9389083202
:10BFC00006F04CFCF8E76FF00A00F5E7F8B500233F
:10BFD0000446037103685A6892B11B7803F0F003BA
:10BFE000102B0DD185684FF6FF77BD422E46236892
:10BFF00028BF3E465868B1B203F092FDAD1BF4D1A4
:10C00000F8BD000013B504460068FFF711F908BB3E
:10C010002068037803F0F003102B19D14178E1B9BF
:10C020004368EBB10123C0F8C44001914370FFF7AE
:10C0300031FB80B10C48FEF77FFE206801990C307F
:10C04000FEF706FE084802B0BDE81040FEF75EBEEF
:10C050006FF00500207102B010BD6FF00400F9E729
:10C060006FF00A00F6E700BF20FD00240268536865
:10C0700030B5BBB1017C846879B11D6825600024AE
:10C080000471127802F0F002102A11D0202A0BD18C
:10C0900029B1C2685B8A138006E05D68EEE71A7C0E
:10C0A000520702D4F523037130BDC2689B8AF2E7C0
:10C0B00021B91A7D012AF5D91B8B00E0DB8AC26801
:10C0C000E9E7000010B504460068436863B10378EF
:10C0D00003F0F003102B07D1227A4378032A01D012
:10C0E000022B01D0032B02D1F523237110BD012BAC
:10C0F00001D1FB23F9E7D30701D5FFF762FD2068E3
:10C10000042300214370C0F8C440FFF797FB0028C8
:10C11000ECD00648FEF710FE206800210C30FEF738
:10C1200097FD0248BDE81040FEF7F0BD20FD002459
:10C1300010B5062002F0C6FF044618B110220021F7
:10C1400024F036FA204610BD10B5044660B10068F0
:10C1500020B103F000FA0023C4E900332146062091
:10C16000BDE8104002F0BABF10BD10B5044630B1B2
:10C17000006808B103F0EFF90023C4E9003310BDF3
:10C1800070B50E4615460446A0B1006808B103F02C
:10C19000E2F941220021362003F010FA206018B99C
:10C1A00060604FF0FF3070BD466005814581606082
:10C1B0000020F8E76FF00F00F5E7000007B527480B
:10C1C000FEF7A4FD264B1B6813B1264A106898475A
:10C1D000224D254E06F068F9431C044621D128461D
:10C1E000FEF7AAFD002201A93046FEF783FC28468F
:10C1F000FEF78CFD019C002CECD02378012B23D082
:10C20000022B27D0002BE5D16068D4E902139847B0
:10C2100010B1606803F09FF92146092002F05EFF2B
:10C22000D8E710B906F01EF9D4E72846FEF784FDDA
:10C23000224601A93046FEF75DFC04462846FEF77B
:10C2400065FD0134EED0D5E7D4E9013098472146A9
:10C250000820E3E7D4E901309847BBE720FD00243C
:10C26000C04E0024C44E0024C84E0024F8B5074632
:10C2700009200E46154602F025FF044668B100234A
:10C280000146C5600370C0E901760548FEF7F2FB80
:10C2900028B12146092002F021FF4FF0FF30F8BD00
:10C2A000C84E002491F83D3013F0180F14BF024A15
:10C2B000024AFFF7DBBF00BFD1290508DDDF040814
:10C2C00038B5054608200C4602F0FCFE014640B198
:10C2D0000123C0E9015403700348FEF79DFB0020D1
:10C2E00038BD4FF0FF30FBE7C84E002470B506465E
:10C2F00008200D4602F0E6FE044660B10123014627
:10C300000370C0E901650548FEF7B4FB28B121467A
:10C31000082002F0E3FE4FF0FF3070BDC84E00244D
:10C3200070B5064E0D4604463046FEF7EFFC284633
:10C33000A0473046FEF700FD002070BD20FD002420
:10C3400037B505460C4602F0F7FC0B4B00210B48B5
:10C350001D600B4B1C60FEF71DFB0A48FEF7B0FC8E
:10C3600018230022084900934FF496630748FEF70C
:10C3700063FD03B030BD00BFC04E0024C84E002492
:10C38000C44E002420FD0024BDC10408F784070822
:10C3900043798B421FBF0023417183710381704732
:10C3A000130A0B54431C02309BB280B2CA5470472C
:10C3B000130E0B54431C10B59BB2140CCC54831CAD
:10C3C000140A9BB2CC54C31C04309BB280B2CA5432
:10C3D00010BD00002DE9F8430E4617469946054664
:10C3E00020B94FF000084046BDE8F8830029F8D096
:10C3F0004FF420724FF49A71362003F0DFF8804634
:10C400000028EED0032F02D17379032B07D1B37923
:10C41000234C13B9FEF76EFD206023683360D8F813
:10C4200004404FF49A720021204624F0C1F8012301
:10C43000042F2370637095F83C30A37033681BBAE7
:10C44000636008D0FB1F012B05D9032F05D1737939
:10C45000043B012B01D86B68E36005F1360304F15E
:10C460001C023C3513F8011BAB4202F8011BF9D149
:10C4700063236FF07D0284F8F27084F8EC3084F866
:10C48000EF30352384F8ED20532284F8F030012377
:10C4900084F8EE2084F8F1300323A9F80030A2E7F5
:10C4A000184F00240346104630B45C1CFF25A2B28E
:10C4B000CD5411FA84F100251446432C0BD9442A9B
:10C4C000C3F1430103F1F10388BF0021194430BCDB
:10C4D00089B203F0F9B8013401F8015BA4B2ECE7CA
:10C4E000F0B50023846A85B0064606212046E36144
:10C4F000FFF74EFF0DF10E03012221463046FFF7F4
:10C5000069FF0546002838D041683922BDF80E3051
:10C51000F031294F981CCA540133022280B29BB2D9
:10C52000CA54B28EADF80E00FFF73AFF3723421C13
:10C530000B5492B2042302308B54ADF80E00BDF8B8
:10C540000E20013B17F801CB501C13F0FF0301F83C
:10C5500002C080B2ADF80E00F1D12A46FFF7A2FF6B
:10C56000164B17482946174ACDE900634323006854
:10C5700006F0D0F8284602F0EEFFA3790020FF2B4A
:10C580001CBF0133A371A279052A97BF01234EF680
:10C5900060239340C3EB431298BF03EB82034FF435
:10C5A000FA729CBFDB009BB203F2F313B3FBF2F30E
:10C5B000238105B0F0BD00BF028507080885070884
:10C5C000104F00240C85070838B5846A05460821F9
:10C5D0002046FFF7DDFE002204F11C01284601F091
:10C5E000B5F8A379FF2B1CBF0133A371012323816D
:10C5F00038BD23B50546002855D0806A002852D0A2
:10C6000000234382836A5A1C0CD01E33B3F5701F7B
:10C6100036BF3C224FF6FF73B3FBF2F39AB2002B06
:10C6200043D08282C36A591C0ED01E33B3F5701FEB
:10C6300036BF3C224FF6FF73B3FBF2F39AB2002BE6
:10C6400036D042814389C381036B5A1C0DD01E33FF
:10C65000B3F5701F36BF3C224FF6FF73B3FBF2F306
:10C660009AB243B3828183890382838942899A4241
:10C6700002D30BB100234381C379FBB1036A00935A
:10C68000436A01932BB9C369009A134043F0807346
:10C6900001930A21FFF77CFE01AB00F11C016A4601
:10C6A000284602F073FD02B020BD01238382B9E762
:10C6B00001234381C6E701238381D4E790F91C203D
:10C6C000037F002A01DBFF23D9E7BF2B8CBF6FF06C
:10C6D0007F434FF6FF73D2E770B5114C2678B6B999
:10C6E000104D06F04DF92860B0B1427A0E4942F083
:10C6F00020024272442205F0ABFF43220A49286817
:10C7000006F0F8F832460949286806F01BF9237844
:10C7100000200133237070BD4FF0FF30FBE700BFF6
:10C72000144F0024104F00240885070895CA0408F8
:10C7300030B5836A0246224C002085B0C3E9080068
:10C74000E07810B11F48C0689862207900282FD087
:10C750001C480069D862607900282CD019484569C6
:10C760001D630969D961A17921B11649896909BA9D
:10C7700019620121D971E17919B11249C96909BA5E
:10C780005962237A93B10F4D03A9002001922B6ABD
:10C790001BBA039302F00AFA637A3BB16B6A03A9EE
:10C7A000019A01201BBA039302F000FA05B030BDD4
:10C7B000986A4008CEE79D6AC5EBC505ED08CFE74E
:10C7C00050FD00245CFD0024F8B504460D461646D5
:10C7D000AAB1104624F094FC88B1C4F141039842F8
:10C7E00028BF18460C232B55A31C013432189BB2CA
:10C7F000A4B228551C46964203D11C18A4B2204668
:10C80000F8BD16F8017B611C2F558CB2F3E70000D0
:10C810002DE9FF41856A804603212846FFF7B8FDD0
:10C820000DF10E03032229464046FFF7D3FD0746CC
:10C8300000286BD044683922BDF80E300426F0344D
:10C84000981CE2540133022280B29BB22146E2548A
:10C850004FF41072ADF80E00FFF7A2FD034632222E
:10C860000133225402309BB280B2E654EA69ADF83B
:10C870000E0012BAFFF79CFD3723264A2354431CAF
:10C8800002309BB2E654ADF80E00BDF80E30013E0A
:10C8900012F8011B581C16F0FF06E15480B2ADF8E7
:10C8A0000E00F2D12146D8F83020FFF78DFF214647
:10C8B0003A46ADF80E00FFF7F5FD1748CDF80080B9
:10C8C0004323164A3946006805F0AAFF0446384655
:10C8D00002F041FEAB792046FF2B1CBF0133AB7148
:10C8E000AB79092B96BFC3EB431242F2107303EBF3
:10C8F00082034FF4FA729CBFDB009BB203F2F31386
:10C90000B3FBF2F32B8104B0BDE8F0814FF0FF34AC
:10C91000E0E700BF02850708104F00240C850708D8
:10C920002DE9FF410746002800F09380846A002C1F
:10C9300000F0928001212046FFF72AFD0DF10E0341
:10C94000032221463846FFF745FD804600287DD06A
:10C9500045683922BDF80E300426F035981CEA549B
:10C960000133022280B29BB22946EA54BA8EADF856
:10C970000E00FFF715FD322300F1020C2B54431C6F
:10C980001FFA8CFC9BB26046EE54E269ADF80EC013
:10C9900012BAFFF70DFD0346362201332A54023046
:10C9A0009BB280B2EE54A269ADF80E0012BAFFF746
:10C9B000FFFC37232A4A2B54431C02309BB2EE540F
:10C9C000ADF80E00BDF80E30013E12F8011B581CE8
:10C9D00016F0FF06E95480B2ADF80E00F2D12946F8
:10C9E0003A6BFFF7F1FE29464246ADF80E00FFF71D
:10C9F00059FD1C4B1C4841461C4ACDE9007343239A
:10CA0000006805F087FE0546404602F0A4FDA379C4
:10CA1000FF2B1CBF0133A371A279052A97BF012305
:10CA20004EF660239340C3EB431298BF03EB82039F
:10CA30004FF4FA729CBFDB009BB203F2F313B3FB1B
:10CA4000F2F32381284604B0BDE8F0814FF0FF35B2
:10CA5000DDE76FF00F05F5E76FF00505F2E700BFC2
:10CA60000285070808850708104F00240C85070871
:10CA700038B5064B1C78013CE4B21C7024B9044D57
:10CA8000286805F063FF2C6038BD00BF144F0024F8
:10CA9000104F0024AE4B2DE9F04F5F6889B09346EC
:10CAA000BB6A0093ABB31B799BB353892B2B30D953
:10CAB00052681378022B2CD197F83C4007F13600CE
:10CAC00002F11C010023DDB2AC4201D9062B19D1C1
:10CAD0005368009A1BBA12689A421AD100239D4AE1
:10CAE0004FF0F009136053601381BBF808A0019365
:10CAF000D846B8F80A304B4511D9D8F804304D461D
:10CB00000293DCE010F8016B013311F8015BAE42D7
:10CB1000D9D0584602F01FFD09B0BDE8F08FA9EB4F
:10CB20000309AAEB030AD8F800801FFA89F91FFA53
:10CB30008AFAB8F1000FDCD1EBE7AB1C9BB2AB4239
:10CB4000E7D36C1CB8F80A2094420DDA029A2A4402
:10CB5000527806291AD8062900F29880DFE801F0F9
:10CB6000981F965E96966500D8F80020002A00F07F
:10CB7000398152681278ECE7082800F28780DFE8F4
:10CB800000F0606670768585857C7E00A1F13300BB
:10CB9000C6B2082EF0D94FF0FF36002403E0042A75
:10CBA000B7D11446062615444FF6FD718D42B0DC10
:10CBB0009D18ADB2002C6CD000220792654AB218C5
:10CBC0000392039911F8012B0391002A61D1042CDF
:10CBD000224607A9404628BF0422CDE9042302F0DB
:10CBE0000BFE049A824294D1042C40F28F80A2075B
:10CBF0008FD1039B4FF00102043C03F8012C079AEC
:10CC0000E4B2554B12BA43F82620059B1A1D92B286
:10CC100093423FF67EAF01361346D2E7032A7FF6F2
:10CC200078AF07260424BEE7002291077FF471AF96
:10CC3000082A144628BF082494423FF66AAF082603
:10CC4000B1E7042A7FF465AF14460326ABE7012A57
:10CC50007FF45FAFB9F1F00F7FF45BAF14460026AD
:10CC6000A1E7012A7FF455AF144616469BE7042A34
:10CC70007FF44FAF1446022695E7042AF2E7042A10
:10CC80007FF447AF144605268DE70022002982D1A4
:10CC9000A5B2B8F80A30AB4211D8ED1AAAEB030AD4
:10CCA000ADB21FFA8AFA5545BFF433AFD8F8008009
:10CCB000B8F1000F3FF42DAFD8F80430029355457A
:10CCC00004D2029B595DFF297FF437AF214A1378C4
:10CCD00010466BBB019B002B32D14378002B3FF4F5
:10CCE00018AF1D4ADBF804101379052B4AD1009BBD
:10CCF0005B79012B3BD13846FFF71AFD97F83D30A1
:10CD000038461B073BD5FFF75FFC02E70AD1079BBC
:10CD10001BBA104A079301239355079B0E4A42F80A
:10CD20002630B6E7012C7FF4F4AE9DF81C30F0E716
:10CD3000094B00211B681170012B13D0022B0DD160
:10CD400000234FF06C0A4FF02C090193D0E600BF8E
:10CD500088FD002450FD00245CFD0024032BB9D184
:10CD6000012301934FF0EC0A4FF06C09C0E6033B3E
:10CD7000022B3FF6CEAE3846FFF7DAFC3846FFF717
:10CD800038FCC6E6062B15D1009B5B79DA1E022A19
:10CD900002D9012B7FF4BDAEB86A0C21FFF7F8FA77
:10CDA0002A4B38461A46194602F0F0F93846FFF782
:10CDB00097FBAEE6022B7FF4ACAE009B5B79062BB3
:10CDC0007FF4A7AE8378002B3FF4A3AE9268BB6AD2
:10CDD000019812BA188138469A610A69DA61FFF738
:10CDE0009FFD96E6062913D806293FF64EAF01A20D
:10CDF00052F821F091CC040813CB04088BCC040822
:10CE000013CB04088BCC04088BCC040829CC040871
:10CE1000A1F13300C6B2082E3FF6BDAE08283FF69A
:10CE200034AF01A252F820F013CB040813CB04084E
:10CE300013CB040813CB04088BCC04088BCC040858
:10CE40008BCC040813CB040813CB0408088507080F
:10CE5000836A7BB15A79052A06D8022A06D84AB1D4
:10CE600000229A71FFF73CBB0A2AF9D100229A717D
:10CE7000FFF7CEBC704700007FB50646002841D0C2
:10CE8000846A002C3ED06379082B3BD10A68E369A1
:10CE90009A4237D10C212046FFF77AFA0DF10E03A2
:10CEA000042221463046FFF795FA054618B341683B
:10CEB0003222BDF80E30F031981CCA5401330422DE
:10CEC00080B29BB2CA54E269ADF80E0012BAFFF705
:10CED0006FFA2A46ADF80E00FFF7E4FA0A4B29462E
:10CEE0000A480B4ACDE900634323006805F012FCB1
:10CEF000284602F030FBA379FF2B1CBF0133A3713E
:10CF00001423238104B070BD08850708104F002446
:10CF10000C850708F0B5856A85B0074605212846C7
:10CF2000FFF736FA0DF10E03032229463846FFF7C4
:10CF300051FA064600285BD044683922BDF80E300D
:10CF4000F034981CE2540133022280B29BB2214695
:10CF5000E254BA8EADF80E00FFF722FA3723421CD6
:10CF60002549235492B204230230A354ADF80E0095
:10CF7000BDF80E20013B11F801CB501C13F0FF034C
:10CF800004F802C080B2ADF80E00F1D121463A6B30
:10CF9000FFF71AFC21463246ADF80E00FFF782FA81
:10CFA00016480097432305F118023146006805F042
:10CFB00037FC0446304602F0CEFAAB792046FF2B10
:10CFC0001CBF0133AB71AB79092B96BFC3EB431286
:10CFD00044F6206303EB82034FF4FA729CBF1B01FB
:10CFE0009BB203F2F313B3FBF2F32B8105B0F0BD58
:10CFF0004FF0FF34E1E700BF02850708104F00241F
:10D0000050B1806A40B140790A2806D0043801281E
:10D010008CBF00200120C0B270470120FBE7000058
:10D020007FB5846A0646002C4DD06379002B4AD028
:10D03000A36903930023C4E90633C4E90833C4E9B0
:10D040000B33A362E3812361A382FFF7D9FF50B3BF
:10D050000DF10A03072221463046FFF7BBF90546CA
:10D0600008B341683622BDF80A30F031981CCA5422
:10D070000133042280B29BB2CA54039AADF80A006D
:10D0800012BAFFF795F92A46ADF80A00FFF70AFA37
:10D090000E484323009603AA2946006805F0C0FB0A
:10D0A000284602F058FA0A4B304619461A4602F052
:10D0B0006DF800212046FFF76BF923791BB1FFF7CC
:10D0C000D7FC0023237104B070BD00BF104F0024B3
:10D0D0000885070838B50446002839D090F83D3057
:10D0E000DA0735D5838E856AB3F5107F02D24FF00B
:10D0F000FF321BE0E5B9342001F04EFF0546002861
:10D10000F5D0A06234220021284623F051FAFFF71F
:10D11000E3FA02460028EAD101232B7194F83D304E
:10D120005B070BD402212846FFF732F9104638BDC1
:10D130002B79002BE6D0FFF79BFCE3E72046FFF7B7
:10D14000CFF902460028F1D02046FFF769FFCEE76D
:10D150006FF00F02EAE700005E4B2DE9F0431D6817
:10D1600085B004265C4F15B905B0BDE8F083AC6A04
:10D170007CB163796BB1A18A69B1628A013292B2E2
:10D180009142628207D12846FFF74AFF2846FFF7FF
:10D19000A1FF2D68E7E7228A002A7FD0511E012ACD
:10D1A00021827BD1013BDBB2092BF2D840F219225C
:10D1B00022FA03F3DB07ECD504212046FFF7E8F859
:10D1C0000DF10E03032221462846FFF703F981469D
:10D1D000002842D041683922BDF80E3001F1F00834
:10D1E000981C08F803200133022280B29BB241460A
:10D1F00008F80320AA8EADF80E00FFF7D1F8372308
:10D20000364908F80030431C02309BB208F803602E
:10D210000423ADF80E00BDF80E20013B11F801CB40
:10D22000501C13F0FF0308F802C080B2ADF80E00E6
:10D23000F1D12A6B4146FFF7C7FA4A464146ADF89D
:10D240000E00FFF72FF94323254A49463868009519
:10D2500005F0E6FA484602F07EF9A379FF2B1CBFE1
:10D260000133A371A379092B96BFC3EB431242F29A
:10D27000107303EB82034FF4FA729CBFDB009BB286
:10D2800003F2F313B3FBF2F3628A2381A38A9B1A9E
:10D29000012B7FF77EAF5B1023827AE7E289002AB9
:10D2A0003FF477AF511E012AE1817FF472AF03F0A2
:10D2B000FB02012A02D00A2B7FF46BAF2846FFF74E
:10D2C00029FEA389628A9B1A012BC4BF5B10E381EC
:10D2D0005FE700BF04170124104F002402850708F0
:10D2E0000C85070838B51E4B00251C6804B938BDED
:10D2F000A36A23B11A89012A03D9013A1A81246841
:10D30000F4E7FCD15A791D810C2A01D0062A03D1F9
:10D310002046FFF7E5F8F2E7012A0CD19B79204679
:10D32000052B02D8FFF7FCFAE9E7FFF779FE204664
:10D33000FFF7D0FEE3E7082A09D19B792046012BAD
:10D3400002D8FFF741F9DAE7FFF753F9D7E7032AE5
:10D35000D5D19B792046012BDBD8FFF759FACEE7D0
:10D360000417012408B5FFF75BFE002008BDFFF796
:10D3700057BE000070B51826074D04464643A8590D
:10D3800018B102F0E8F80023AB511820002300FB8D
:10D390000454237570BD00BF1C4F00242DE9F74FC6
:10D3A0004FF00A0C0024019106469046314DA146EB
:10D3B000A34661466746E64600940A2923B295F8DB
:10D3C00014A019D1BAF1000F4CD04EB16868326880
:10D3D000824205D1B8F1000F36D0A868404533D05D
:10D3E000BAF1010F688A38D12A688AB3009A90424C
:10D3F00005D39C46009002E0BAF1000FE5D101345C
:10D4000018350A2CD9D1019B012B2FD10A290CD117
:10D410000A2F06D1BEF10A0F26D1BCF10A0F25D082
:10D4200067463846FFF7A6FF3946124826B118224C
:10D43000336802FB010253601823002203FB01033F
:10D440005A82C3F808800B46184603B0BDE8F08F37
:10D450005845D4D383469E46D1E74845CFD381462D
:10D460001F46CCE71946CAE77746DAE74FF0FF33A5
:10D47000EAE700BF1C4F00242DE9F3470746884622
:10D4800091461C214FF420720E201D46DDF82CA081
:10D4900002F094F8064688B344680146BDF834307B
:10D4A00042465BBAE38038462B68A360AB88002510
:10D4B000A381DAF80030C4F81230BAF80430E382FD
:10D4C0000A9B1B68C4F80E300C9B1B682570A36177
:10D4D0000123E57063700823A370062323710423DE
:10D4E000637140F6060300934B4605F0C1FA3046DF
:10D4F00002F031F8284602B0BDE8F0874FF0FF3067
:10D50000F9E7000070B50646074D00242B7D2BB1CE
:10D51000AB68B34202D12046FFF72CFF0134183527
:10D520000A2CF3D170BD00BF1C4F00242DE9F04739
:10D53000074688B00C4681B145682B88B3F5807FDB
:10D5400008D12B79062B05D16B79042B02D16B887E
:10D55000082B05D0384601F0FEFF08B0BDE8F08783
:10D56000D5F80E0005F108084E68AB690790002E4B
:10D5700053D0F31A5E425E41C6F1020A5FFA8AFA9C
:10D5800000283ED0214600F0F6FE8146002838D122
:10D59000079B03F0F003E02B33D02246514607A847
:10D5A000FFF7FCFE031E2CDB1820264A4FF0020E6C
:10D5B00000FB03FC02EB0C0181F814E04FF00C0EB1
:10D5C0008C6013FB00E3D8F8000002EB030ED05090
:10D5D000B8F80430AEF80430A1F8129052F80C10EC
:10D5E00079B14FF4006342F80C90204604F1360202
:10D5F00000934346059105F03BFA0599084601F072
:10D60000AAFFEB88B3F5807F0AD0B3F5007FA1D1E4
:10D6100007A92046FFF730FC9CE74FF0020AAFE76E
:10D62000002E97D0022204F136032046039207AA67
:10D630001946CDE90182221D00924246FFF71CFFE8
:10D6400088E700BF1C4F00241FB50246012400F1EB
:10D6500036030432CDE902140449009201911946BF
:10D66000034AFFF709FF04B010BD00BF5E8607083C
:10D6700058860708F8B5134C002502260427227D9A
:10D680006AB1638A01339BB2B3F5967F638203D29A
:10D69000012A09D1042B0FD92846FFF76BFE01356B
:10D6A00018340A2DEBD1F8BD032A01D12775F6E70E
:10D6B000042AF4D12675F2E7211DA068FFF7C4FF04
:10D6C000EDE700BF1C4F00242DE9B0478846182421
:10D6D0001C4902EB420585B0074604FB0214ED002D
:10D6E00000F13609237D05F10C0A022B8A440AD188
:10D6F000638AB3F58E7F12D904352944FFF7A4FF5E
:10D7000008B9032323754FF400634A46414638465F
:10D710000093534605F0ACF905B0BDE8B087B3F50A
:10D72000877FF0D301230435524603930D44064B03
:10D73000494602950193031D00934B46FFF79CFE5B
:10D74000DEE700BF1C4F00245E8607082DE9F34189
:10D750008846054601461446D8F8000000F00BFE46
:10D76000002853D1D8F8003003F0F002E02A4DD061
:10D77000002B4BD02A4601214046FFF70FFE031E27
:10D7800003DA58B202B0BDE8F081DFB2274E1822AA
:10D7900002FB0762137DBBB1CCB14FF0FF30182301
:10D7A00003FB0762127D012A18D9214A03FB076394
:10D7B0002146284617704FF400620C33009205F1A1
:10D7C000360205F055F9DDE70123956013754146F2
:10D7D0002846FFF739FF002CE1D1D3E7D2D1234609
:10D7E0001A7B520615D41B68002BF9D1204601F094
:10D7F0009DFF182303FB07F21D46B05808B101F046
:10D80000AAFE05FB07F30020F450BBE76FF00F0002
:10D81000B8E722464FF420710E2002F040F804468B
:10D820000028E6D14FF0FF30ACE700BF1C4F0024CA
:10D830000C500024F0B5044685B00E460146106831
:10D84000154600F098FD002860D12B6803F0F00227
:10D85000E02A1BD10123ADF808305E238DF80A3091
:10D860006B7803F07F038DF80B30AB788DF80C30BC
:10D87000EB788DF80D3002AB4FF400623146204654
:10D88000009204F1360205F0F3F823E06268A16823
:10D890005A400A4209D09BB24FF6A962934204D083
:10D8A000E368002B34D004F10C051B4918231B48F6
:10D8B0000A788C4603FB0203187D01280CD999686D
:10D8C000A14209D129685B68994205D131462046B9
:10D8D000FFF7FAFE05B0F0BD104B0021187DCAB26B
:10D8E000012809D99868A04206D12F685868874254
:10D8F00002D18CF80020E9E7013118330A29EDD173
:10D90000324629462046FFF721FFE3E7044BB3E701
:10D910006FF00300DEE700BF0C5000241C4F002412
:10D9200058860708F0B5044687B00F4616462421EE
:10D930004FF42072222001F041FE054678B32068A2
:10D9400000236C6800F11C01237104F1080263716B
:10D95000A371E37103462770667053F8046B8B4222
:10D9600042F8046BF9D1C36805A8059300F000FBE9
:10D97000074688B1002669892046A670E67001F046
:10D98000B3F90123608005AA314628460297CDE904
:10D990000063FF2300F0CDFC284601F0DCFD07B05A
:10D9A000F0BD0000524B2DE9F04FD3F808B087B01E
:10D9B00004460E469BF800509A4605F00F05AD0050
:10D9C000132D19D94389032B16D943681B78082BCB
:10D9D00012D1DAF8140000F0F003E02B0CD0DAF8E2
:10D9E000001000F0C8FC68B1371D2389072B03D94C
:10D9F000204601F07FF940B1204607B0BDE8F04F66
:10DA000001F0A9BD0AF11407EFE705F10E01204668
:10DA10001FFA85F8059101F07DFD0599002860D079
:10DA2000238903EB080189B28B42E5D84FF42072B9
:10DA30000E2001F0C3FD81460028DDD0428905F1AA
:10DA400008039A4202D201F086FDD5E759462A46DC
:10DA50004068FCF780FF2946484601F05EFD08B1AA
:10DA60004846F0E72146484601F084FE0028F7D1F9
:10DA700020464C4601F06FFD29462046D4F804901C
:10DA800001F048FD0028B7D165684FF6F7723B6892
:10DA90004146EB60DAF810304FF0FF0A2B61B9F81D
:10DAA000023089F80000284693428CBF09330833BE
:10DAB0009BB2A9F802304FF0000985F808A085F85C
:10DAC0000A9085F80B9001F00FF9012368814A460E
:10DAD000394620460296CDE90093534600F029FCD2
:10DAE0008AE7204601F019FD0028C5D084E700BF71
:10DAF00088FD00240A4604300321FFF713BF0A46BD
:10DB000004300B21FFF70EBF224B2DE9F0431B68B9
:10DB100089B007460E46904608214FF42072362001
:10DB2000069301F04BFD054680B37B68B8F1160FF4
:10DB300044684FF00801069308BF06F104097368B2
:10DB4000204613BFDFF8509063600123636008BF75
:10DB50003372002684F800806670A670E67001F0CB
:10DB6000C3F840F2944360804A460793042306A911
:10DB70002846049307ABCDE902730223CDE9006385
:10DB8000012300F0BDFB284601F0E5FC09B0BDE82B
:10DB9000F08300BF088507081050002438B5437A89
:10DBA00005460C46022B05D0012B09D143890BB148
:10DBB0008B4205D9022C04D801236B8101236B729F
:10DBC00038BDFDF797F9B0FBF4F101FB14046C814B
:10DBD000002CF1D0F2E70000034B044A1A6002F176
:10DBE0008072034B1A60704714500024E00000015B
:10DBF0001050002470B500230546C46AC3620CB9F6
:10DC0000204670BD6B6C26681BB10022211D284682
:10DC1000984721460A20344601F060FAEFE7C36ACC
:10DC200010B50BB11C6804B910BD20460521FFF7E3
:10DC3000B5FF2468F7E7C06A00B9704742680B680F
:10DC40009A42FAD00068F7E770B505460E46FFF72E
:10DC5000F2FF68B90A20EC6A01F034FA40B10023FF
:10DC60003EB132680373C0E9012324B90460E8625D
:10DC700070BD1A46F6E7236803602060F8E70000ED
:10DC800010B50B490446FFF7DFFF60B10223437272
:10DC9000037B01330373636C43B1012204492046C3
:10DCA0009847002010BD4FF0FF30FBE71846F9E71A
:10DCB00014500024F7B50E4641890546174607293A
:10DCC00004D8284601F047FC03B0F0BD4468204664
:10DCD00001F00AF80028F4D139463046FFF7ABFFCF
:10DCE0000028EED02378112B08D0162BE9D1437AE7
:10DCF000012B04BF4FF400738360E2E7124A3968D6
:10DD00001268636891421BD17BB963780BB90A230F
:10DD10006370F36A002BD4D01E68002ED1D0304639
:10DD20006178FFF73BFF3668F7E701A930460193BA
:10DD3000FFF781FF0028C4D06178FFF72FFFC0E70D
:10DD4000002BBED0F8E700BF145000240B6803F08E
:10DD5000F002E02A70B505460E462DD1194A126828
:10DD6000934229D090F83D309B0625D5FFF76CFFF4
:10DD7000044620B3437AD3B9037B2BB96B6C1BB138
:10DD80000122314628469847162221462846FFF7A9
:10DD9000BBFEFDF7AFF80523B0FBF3F303EB830302
:10DDA000C01A01230128637238BF01206081237BE0
:10DDB00000200133237370BD6FF00500FBE74FF0C7
:10DDC000FF30F8E7145000240B6803F0F002E02A5B
:10DDD00070B505460E461BD10F4A1268934217D004
:10DDE0000E4B6FF005001C6804B970BD94F83D300F
:10DDF0009B060BD525B12B6813B16268934205D100
:10DE000031462046FFF7A2FF0028EED12468EBE759
:10DE10006FF00500E9E700BF145000240417012447
:10DE20000B6803F0F002E02A70B505460E462DD1CE
:10DE3000184A1268934229D090F83D309B0625D5A8
:10DE4000FFF7F9FE044608B3037B012B1BD8EB6AEE
:10DE500023B11A68944214D122681A60237A23B13C
:10DE6000172221462846FFF74FFE6B6C1BB100229C
:10DE700031462846984721460A2001F02FF9002014
:10DE800070BD1346E4E7013B0373F8E76FF005004C
:10DE9000F6E700BF14500024F8B50B6806460F469D
:10DEA00003F0F002E02A1DD1104A1268934219D003
:10DEB0000F4B6FF005041D680DB92046F8BD95F8AD
:10DEC0003D309B060CD526B1336813B16A68934286
:10DED00006D139462846FFF7A3FF002C18BF044699
:10DEE0002D68E9E76FF00504E7E700BF1450002450
:10DEF00004170124F8B50F4B02270F4E1D6805B912
:10DF0000F8BDEC6A0CB92D68F9E7638983B1013B70
:10DF10009BB2638163B9637A012B09D1626833686C
:10DF20009A4205D01622214628466772FFF7ECFD7B
:10DF30002468E7E7041701241450002408B590F87A
:10DF40003D30014613F001030BD043684BB1074A43
:10DF50005069834207D000F00EFA003818BF012044
:10DF600008BD1846FCE70120FAE700BF88FD002441
:10DF7000036803F0F002E02A10B502D1144A1068D9
:10DF800088B9144A106878B9134A12685AB192F8DD
:10DF90003D1001F00501052905D1516819B1DBB229
:10DFA0007F2B18BF104610BD90F83D10CA070CD546
:10DFB0004C070AD5426842B15A4084682242F2D0E6
:10DFC0008A0702D4C2689342EDD00068DBE700BF45
:10DFD0001850002404170124081701242DE9F843E0
:10DFE000D0F8048005460E4698F800402309042B1B
:10DFF00005D0284601F0AFFA0020BDE8F88304F010
:10E000000F04B8F8027003897FBABFB24FEA8409DF
:10E01000BB424C4602D9394601F056FB6B89A342FC
:10E02000E7D32B89BB42E4D3132CE2D921464046E7
:10E0300000F05AFE0028DCD1D8F81030544C63614F
:10E0400003F0F003D8F80C20E02B226161D196F8A0
:10E050003D309B0605D498F80930112B71D000276C
:10E060000CE004F114013046FFF7E5FD0028F2D082
:10E07000484AD4E9043191420ED03746206948B16C
:10E08000314600F078F90028B3D1236903F0F0039A
:10E09000E02BAED01FB9ACE7002BEED13746B8F875
:10E0A000063023F0C0033BB1284600F003FB0546D1
:10E0B0000028A1D0D0F80480C4F80880494628463A
:10E0C000C4E9007698F8003003F00F039B00A381A9
:10E0D00001F023FA98F80930062B48D039D8012BE3
:10E0E0004AD0022B4DD03946606900F044F960B93E
:10E0F000636903F0F003E02B07D04946284601F09E
:10E1000022FA02212846FFF7F5FC284601F023FAFF
:10E1100025E03046FFF712FF80B9237D7F2B9AD090
:10E120001D4B1F68002F96D0B74201D13F68F9E719
:10E130003846FFF703FF0028F8D09FE7002E9CD158
:10E1400089E708EB09035B88B3F5884F87D1374629
:10E15000A0E7112BC7D13146284604F0C3F90023AC
:10E16000C4E90033A360A381C4E9043344E7314622
:10E17000284602F0C1FEF2E731462846FFF712FCBE
:10E18000EDE7064A31462846FFF794FDE7E700BF72
:10E1900088FD0024E0000001041701249CFD0024F8
:10E1A0002DE9F04F87B09B46044690469DF84030DD
:10E1B0009DF84490DDF848A0BDF8505001910293BD
:10E1C000002A00F08680002D7FD0282D00F291805B
:10E1D000EE1C26F00306B6B206F114073146BFB2B4
:10E1E00001F098F920B16FF0010007B0BDE8F08FA1
:10E1F00003902A4613996068FCF7ADFBB542039B78
:10E2000005D26068721B1946284422F0D1F9002318
:10E21000616876081D4631F8132001339E4215448B
:10E22000F9DC1421204601F075F90028DBD1626881
:10E23000C7F3870782F8099049EA0B2982F808B0EA
:10E2400047F04007D8F800104FEA2923177043EA37
:10E25000092311614FEA114919FA81F111FA83F387
:10E260001D44029B43EA072753703B1243EA0723EE
:10E2700015FA83F523899071D0711F485BBA018824
:10E2800015FA83F553804BBA0131938015FA83F365
:10E2900001800199D9B91949096813FA81F3D1604C
:10E2A00003EB114399B201EB134303EB1343DB433D
:10E2B0005381BAF83430ABB122899A4212D942461E
:10E2C0005146204600F070FB8FE71427A9E701991B
:10E2D000E2E74389132B86D943680DF114081B69C3
:10E2E0000593E6E7DAF8143042462146504698474F
:10E2F0007BE76FF0050078E71C50002408850708CD
:10E30000F0B59C469DF814509DF81860BDF824E0C7
:10E31000DDE907471AB109B10B6803B9211D05955D
:10E320006346CDE9087ECDE90664BDE8F040FFF71D
:10E3300037BF10B5002486B0CDE903440A9C02948F
:10E340009DF8244001949DF820400094FFF7D8FFE9
:10E3500006B010BD10B5002486B0CDE903440A9C78
:10E3600002949DF8244001949DF820400094FFF70A
:10E3700017FF06B010BD431E0246033312D891F8B2
:10E380003D3013F0020010D04B6893420CD08868E7
:10E390005340034208D1C34322EA0000C31A584243
:10E3A0005841704701207047002070472DE9F04325
:10E3B00085B0434F027804236E46BE46B446D45D12
:10E3C00014F0040477D0302A1BD1427802F0DF0425
:10E3D000582C0DBF827801304FF00809023008BF79
:10E3E0004FF01009804600241EF8025015F0040F6B
:10E3F0000AD004FB0924303C98F8012008F10108F8
:10E40000F2E74FF00A09EDE7B9F1100F0DD115F061
:10E41000440F0AD005F003050A32022D0CBF61201B
:10E420004120121A42EA0414E6E72E2A08D1013BE1
:10E4300041D008F1010098F8012046F8044BBEE7EE
:10E4400012B115F0080037D0A6EB0C008010013097
:10E4500004280CD8DFE800F0300B03101E00B4F1E4
:10E46000807F28D2009BFF2B25D844EA036409B1A2
:10E4700024BA0C6001201FE0B4F5803F1BD2009A43
:10E48000FF2A18D8019BFF2B15D81B0443EA02630F
:10E490001C43ECE7FF2C0ED80098FF280BD8019BFB
:10E4A000FF2B08D8029AFF2A05D81B0443EA006311
:10E4B00043EA0223ECE7002005B0BDE8F08300BF8B
:10E4C00005D307082DE9F74F03680DF1040C0D463D
:10E4D000042000264FF00A0E4FF02E0801931CF87E
:10E4E000014B0027A2460DF1080BB4FBFEF30EFB17
:10E4F0001349DCB23B46BAF1090F07F1010709F1F4
:10E5000030099B44FFB20BF8089CEBD80CF8014C87
:10E5100037462C46FF2B06F101060DD1974218DA3B
:10E520000138254610F0FF0005F8018BD7D1207087
:10E53000084603B0BDE8F08F5D1E9742EDB208DAE1
:10E5400002AF3B44374613F8083C04F8013B2B4626
:10E55000E0E70020EDE70000074A036810B4146804
:10E5600084425DF8044B18BF0B6001464FF0040075
:10E5700008BF136000F0B2BD205000242DE9F04127
:10E58000466804460F4673689A881ABB1A6800F1F9
:10E590001C01426000F1080252F8040B8A4243F861
:10E5A000040BF9D101213046FFF7A9FA304601F0FA
:10E5B000B5F80546304600F0CEFF666866B92046DD
:10E5C0003946FFF7C9FF0B4A284613885B1B1380A7
:10E5D000BDE8F0810025F0E773683046D3F800808D
:10E5E00001F09CF8284485B2304600F0B4FF46465E
:10E5F000E4E700BF1E5000242DE9F04105460F4618
:10E600000026DFF868800024D8F800302146A446B0
:10E61000204653B910B1FFF7B1FF0644BE4201DAFC
:10E62000012CF0DC3046BDE8F081D5F80CE05A69E9
:10E63000724509D1D5F810E09A69724504D1B3F852
:10E640000CE0AA88964508D0013460B1C27F93F8E7
:10E650001FE096459CBF614618461A68002A18BFFD
:10E660009C461346D5E761461846F6E7205000243D
:10E6700010B50446406908B100F06DFF2146052041
:10E68000BDE8104000F02ABD38B5094B00241868D9
:10E6900000B938BDC37F056823B1013BC377044689
:10E6A0002846F5E72146FFF769FF2046F7E700BF58
:10E6B000205000242DE9F74FD0F80490064699F831
:10E6C000003003F00F03052B40F08F80B9F80230C3
:10E6D0005BBA9BB2B9F806506DBA132B40F2858035
:10E6E000143B9BB2019301F019F8AD4A0746138819
:10E6F000904603440A2B6EDCAA4B1C689A46002CF9
:10E7000078D1042000F0DEFC044658B9394648466A
:10E71000FFF772FF874268DC042000F0D3FC044658
:10E72000002862D01C220021201D21F041FF0F2370
:10E7300004F1080209F11401E377DAF80030CAF8AD
:10E74000004023604B4653F8040B8B4242F8040B05
:10E75000F9D1B9F806C0C5F30C051CF0200C4FEA3E
:10E76000C5050AD1019BEB189BB29D4200F2EF80D8
:10E770004FF6EB72934200F2EA8071680B7848889A
:10E7800003F00F0340BA80B24FEA8309B0EB830F66
:10E79000C0F0DD80CA88A0EB090052BAC2F30C02B7
:10E7A0000023D4F804E0D2000B704B7010448B703F
:10E7B000CB701FFA80FB8A80C8805A4500F2C78060
:10E7C0000120BEF1000F27D1002B00F08F801E60CA
:10E7D000DB88934234E001464846FFF70DFF20B145
:10E7E000B8F800303B440A2B86DD304600F0B3FE1B
:10E7F000002675E0D9F80C3062699A420AD1D9F83E
:10E800001030A2699A4205D1A289B9F804309A421F
:10E8100000F0A580246872E7DEF80490B9F804A03F
:10E82000524565D2C1F800E0002B5DD0B3F806E098
:10E830007245C0F08C80D34500F2898072451E601D
:10E8400040F0A880BCF1000F03D0A37F13F00103B8
:10E850006ED000285AD10020B8F800301F44A8F824
:10E860000070BCF1000F06D1019B1D44A37F43F053
:10E870000103A583A3770128BAD1626804F11C00C3
:10E88000A38B566804F108021433356831469BB2F5
:10E8900052F8047B824241F8047BF9D15BBA738061
:10E8A000002330461421B371F371B372F37200F098
:10E8B0001BFA70816668002D3CD13A4B1B68A3425D
:10E8C00002D01D46002B40D129462046FFF744FECA
:10E8D000304600F023FFB8F80030181AA8F80000FE
:10E8E000304603B0BDE8F08FD34530D86660A9E765
:10E8F0002DD0B9F806E0964529D81BB1DB885345E1
:10E9000018BF0020D9F800E04B465AE76368002B97
:10E91000A1D05B689B88002B9DD10B68002B9BD0FE
:10E920005A68C9889388994295D113681146F5E7CA
:10E93000184691E76F681421284600F0EEFD29463D
:10E94000304600F000FF3D68B5E72B68B7E7616827
:10E9500000297FF44AAF2046FFF7FEFD45E7B9F8EE
:10E9600006305BBAC3F30C03002B7FF4F2AEE389ED
:10E970005BBAC3F30C03002B3FF4EBAE4B4604F140
:10E98000080209F1140153F8040B8B4242F8040BFE
:10E99000F9D1DEE6BCF1000F3FF45DAF002054E793
:10E9A0001E500024205000248B8E2DE9F04F2DEDB9
:10E9B000028B08EE102AB3F114028BB0064648BF52
:10E9C000A3F10D028A46C2F3CF0305934368029375
:10E9D0001B7803F00F03052B4FEA830740F0A98053
:10E9E0004389132B40F2A580029B00250489DB8814
:10E9F0005BBAC3F30C0203F40053143C0793059B6A
:10EA0000A4B20392DB009BB206932CB920460BB054
:10EA1000BDEC028BBDE8F08F069B4FF420721421F1
:10EA20000E20A34228BF2346049300F0C7FD804672
:10EA300010B3029B42681946143153F8040B8B4201
:10EA400042F8040BF9D1D8F804B0DDF81090B9F110
:10EA5000000F39D07589ED1BADB24D4528BF4D462D
:10EA600015B936680027F2E7052000F02BFB0346B6
:10EA700028B9404600F06FFD4FF0FF30C7E7019521
:10EA800029467268089000203A440092412200F022
:10EA900027FD089B20B91946052000F01FFBE8E779
:10EAA000CDE90803A9EB0509304600F03FFE099BBC
:10EAB000214A1FFA89F9089940465E611A6100F0FF
:10EAC00042FEB9F1000FCCD1BAF834202F44039B99
:10EAD000133ABFB2C3F30C03A24201DD079A0AB195
:10EAE00043F400535BBAABF806301421049B58463C
:10EAF00014339BB25BBAABF8023000238BF80A30B8
:10EB00008BF80B3000F0F0F8DAF8143018EE102A19
:10EB10004146ABF80A0050469847404600F01BFDBE
:10EB2000049B059AE41A039B1344A4B29BB203937B
:10EB30006BE76FF005006AE771E6040870470000B4
:10EB400001282DE9F0410446884617460BD8154E9A
:10EB5000356865B12946404622F0D6F828B9023416
:10EB60003B6845F82430BDE8F0812D69F1E71420B9
:10EB7000023400F011FA43460B4A0621054621F003
:10EB80008FFF0023C5E902333A6845F824202B6142
:10EB900033680BB93560E6E71A461B69002BFBD1D9
:10EBA0001561E0E784FD0024F069070830B50446EC
:10EBB00085B00D465AB9012804D80D4B21B10A6819
:10EBC00043F8242005B030BD0A4A1268F8E792F8ED
:10EBD000403002A80849009392F83F3092F83E2056
:10EBE00021F0A6FF2A4602A92046FFF7A9FFE9E780
:10EBF000245000240885070810850708012870B5EF
:10EC000005460E4603D811B1074B1C680CB90748DE
:10EC100007E02146304622F077F818B9A81C04EB2B
:10EC2000800070BD2469F1E784FD00240885070891
:10EC3000012838B50446064D07D8FFF7DFFFA84284
:10EC400002D1044800EB840038BD2846FCE700BF31
:10EC5000088507082450002470472DE9F0411C68FE
:10EC60008046069B0E4617461D682B0C13FA85F34B
:10EC7000002513FA84F303EB14439CB204EB134313
:10EC80009CB204EB1344B8F1000F13D125B1230259
:10EC9000C4F307249BB21C4376BA34447FBA3C4485
:10ECA000A0B200EB1444A0B200EB1440C04380B209
:10ECB000BDE8F081B8F80A10D8F80400FBF70EFEA2
:10ECC000B8F80A302044DB0784B204EB104406D5C0
:10ECD0002302C4F3072485F001059BB21C43D8F836
:10ECE0000080D0E7FFF7B9BF08B5FBF7F7FDC043D9
:10ECF00080B208BD70B500260546344645B926B138
:10ED00002302C4F307249BB21C43E04380B270BDCE
:10ED100069896868FBF7E2FD6B890444DB07A0B2F0
:10ED200000EB144406D52302C4F3072486F0010641
:10ED30009BB21C432D68E1E708B5FCF711F800F021
:10ED400011F800F0B1F900F01FFA03F0BFFB00F07A
:10ED5000FDFDFEF741FFFFF7F1FEBDE8084003F0BF
:10ED60006FBB00000B4B0C4A23F003030B490C480C
:10ED700013604FF47A521A6000221A7103F57A5226
:10ED80000A600849116001211171074A1360FBF7FD
:10ED900097BF00BF0340043060500024645000243B
:10EDA00030500024803E803E2C500024F8B50446AC
:10EDB00000286ED0830705D0FBF7F8FFBDE8F840C8
:10EDC000FCF70EB8334EA0F108053368AB42F3D818
:10EDD000314F00F10C0339689942EDD32F48FBF70E
:10EDE00095FF14F8043C1BB92C48FBF7A5FFE3E79B
:10EDF00034F8080CB0F57A5FF6D834F8062CB2F582
:10EE00007A5FF1D83368A5EB030C1FFA8CFC9445AC
:10EE100002D09A5A6245E7D119183E68B14202D031
:10EE20004A886245E0D1002204F8042C1C4A176885
:10EE3000AF4288BF15608D4211D00F797FB9B142C2
:10EE40000DD01668B142195A24F8081C195A08BF87
:10EE50001560B1F57A5F1CBFC918A1F802C034F87B
:10EE6000061C581885420FD006796EB91668B5424F
:10EE700008BF106034F8082C5A5234F8082CB2F548
:10EE80007A5F1CBF9B1859800448BDE8F840FBF727
:10EE900053BFF8BD6050002464500024305000245B
:10EEA0002C5000242DE9F041CC1C054624F003042D
:10EEB000A4B20B2C04D9B4F57A5F02D9002510E076
:10EEC0000C24A142FAD8DFF8CC80D8F80030AB424D
:10EED00003D82D4A1268AA4206D8FBF767FFFBF752
:10EEE0007FFF2846BDE8F081A5F1080635F8087CCB
:10EEF000F61A083FB6B2BF1BBFB2A742DED3F0D0AE
:10EF00002248FBF703FF35F8081CD8F800305818E2
:10EF10000279EAB906F1080233F801C014441C4A28
:10EF20001768A1B213FA84F4874208BF1460002264
:10EF3000227123F801C0668025F8081C5A5AB2F5E0
:10EF40007A5F01D0134459801048FBF7F5FEC8E7FB
:10EF500004F11402BA42F7D806F108020C4814442E
:10EF60000768A2B213FA84F4A74288BF04600020A5
:10EF700020719952668025F8082C995AB1F57A5F6C
:10EF80001CBF5B185A80DFE7645000243050002417
:10EF90002C500024605000242DE9F041002850D06E
:10EFA000C41C24F00304A4B20B2C04D9B4F57A5F7A
:10EFB00002D9002045E00C24A042FAD826486FF080
:10EFC0000708FBF7A3FE254B2548C4F57A5E1968B0
:10EFD0000268531A9BB2734503D31F48FBF7ACFE7C
:10EFE000E7E7CD18CF5A95F804C0BCF1000F30D137
:10EFF000A8EB03063E44A6422BD304F1140E76453B
:10F0000021D308341C44A6B211FA84F484F804C055
:10F010008F53638001232E802B718B5BB3F57A5F56
:10F0200001D00B445E80AA4206D10E4B1B681479B6
:10F030000CB193420AD102600748FBF77DFE05F14F
:10F040000800BDE8F08101232B71ECE712880A4427
:10F05000EDE73B46BFE700BF30500024605000247E
:10F060002C5000246450002410B50446FBF79EFE8B
:10F0700023681C680CB122681A60FBF7B1FE2046B9
:10F0800010BD436800228168033330B523F00303C9
:10F0900044880A60944200DC30BD0D6801321D6076
:10F0A00005880B602B44F5E738B5054D0E24013C6F
:10F0B00055F8040BFFF7E5FFA4B2002CF7D138BDDB
:10F0C000C08507080D2805D8034B53F820000830E9
:10F0D000FFF7CABF00207047C08507080D2838B564
:10F0E0000C460DD861B1074B53F82050FBF75EFE7C
:10F0F000AB681A6822601C60BDE83840FBF770BE40
:10F1000038BD00BFC08507086FF00B00704710B511
:10F1100090F83D30044603F00502052A11D1C907D5
:10F120000FD542686AB11A0702D5011DFEF78CFAA5
:10F1300094F83D309B0604D52046BDE81040FEF70C
:10F140006EBD10BD30B5044610460A6885B06368D0
:10F150000D469A4216D0036003A90392019000F075
:10F16000D9FE03A9019803F01DFC2B68012120465C
:10F170006360FFF7CCFFE3690BB12046984701209D
:10F1800005B030BD0020FBE770470000F7B5144F15
:10F190000446002914BF0D463D46002A14BF1646FA
:10F1A0003E46002B18BF1F462B68B3B901AA29465B
:10F1B000FFF7C8FF01233268A1688A42E16818BFDF
:10F1C000A2603A688A4218BFE26023B901AA2946C0
:10F1D0002046FFF7B7FF03B0F0BD0023EBE700BF09
:10F1E00008850708F8B5079E044610B90024204694
:10F1F000F8BD002EFAD00025254FDFF8A0C0C5606D
:10F200008586002B08BF634680F83D50002A08BF62
:10F2100062468562002908BF6146C5624564476150
:10F22000C0E90155C0E90755069D4562194D2F7883
:10F2300080F84070089F0761FFF7A8FF2046B0479D
:10F240000028D3D114490E6894F84030FF2B334680
:10F2500008BF84F8400094F8402073B9FE2A01D01A
:10F26000531CDBB22B7094F83D3026609B060C607B
:10F27000BDD52046FEF704FDB9E793F840709742EC
:10F2800003D1013284F84020DEE71B68E5E700BFC8
:10F2900009F10408A0500024041701240885070878
:10F2A000014B1860704700BF0817012410B50446D1
:10F2B00080B190F83D30DA070CD443F0010380F8B8
:10F2C0003D30C36903B1984720460321BDE8104093
:10F2D000FFF71DBF10BD10B5044688B190F83D3052
:10F2E000DA070DD523F001021B0780F83D2001D578
:10F2F000FEF708F9E3691BB12046BDE81040184746
:10F3000010BD000013B5044620B3436843B1043078
:10F310000021019000F0FEFD0021019803F042FB66
:10F3200094F83D309A0602D52046FEF763FC94F827
:10F330003D30DB0702D52046FFF7CDFF0B4B1A68A7
:10F34000A24204BF00221A60094A1368A34204D1F2
:10F350002368136002B010BD1346002BFAD01A6860
:10F36000A242F9D122681A60F4E700BF081701240D
:10F370000417012400B1C161704710B5044698B16B
:10F3800090F83D305A070FD443F0040380F83D3025
:10F39000FDF75EFD03212046FFF7B9FE236A1BB18E
:10F3A0002046BDE81040184710BD50B190F83D20F0
:10F3B000510706D522F00402036A80F83D2003B10C
:10F3C0001847704700B1016270470000034658B10A
:10F3D000064A106800B9704790F840200132D2B256
:10F3E0009A4201D00068F5E7704700BF0417012476
:10F3F00010B5044608B9002010BD02301FF028FCEB
:10F400000A4AC3B210680028F5D090F840209A420A
:10F4100009D1217890F83E20914204D1617890F88A
:10F420003F209142E8D00068EDE700BF04170124B7
:10F4300008B5FFF7DDFF18B190F840000130C0B209
:10F4400008BD000008B5FBF7B1FC084B00221A709C
:10F45000FBF7C6FC064B186800B908BD436F1BB12B
:10F46000BDE8084000F086BCC068F5E70C17012431
:10F470001417012430B5A0B1B1F5803F11D2D9B134
:10F4800003898CB213FA81F39BB29C4209D890F99C
:10F490000C50002D07DA4268511A00F11002914217
:10F4A00005D2012009E0002AFBD04268511A4289A6
:10F4B0004160144403814481002030BD70B506468C
:10F4C0000C200C461546FFF7FDFD40B100230481DA
:10F4D000448143730573C0E900360123C38170BDC5
:10F4E000033020F0030070B50E18BDF81450049CD2
:10F4F000AE420DD804B1044418460023C0E90034DC
:10F50000022301814181437301230273C38170BDD2
:10F510000020FCE70022FFF7ADBF10B588B1B1F5C0
:10F52000803F0ED259B18AB243899A4209D89B1AB8
:10F53000446843812144038941609B1A0381002070
:10F5400010BD0120FCE70B1E02DA5942FFF7E5BFB0
:10F550000122FFF78FBF70B5044660B30025FBF7AB
:10F5600025FCA67B013EF6B2A673FBF739FC4EB92B
:10F57000637B26689B0709D5236920469847013598
:10F58000EDB20EB9284670BD3446E8E7237B03F0A0
:10F590000F03022B04D121460D20FFF79FFDEEE75C
:10F5A000012B02D121460C20F7E7002BE7D12046A2
:10F5B000FFF7FCFBE3E70546E4E70000B2F5C17F97
:10F5C0002DE9F04706460F4685B230D007D822F025
:10F5D0004003012B26D000242046BDE8F087B2F579
:10F5E000207FF8D10335CB1C25F0030523F003035E
:10F5F0001D44ADB205F110009D4280B2EBD38342B1
:10F60000E9D8FFF7C9FC04460028E5D006440023EA
:10F61000078113360360284B26F003064781C36039
:10F620004660D9E70020BDE8F047FFF747BF002656
:10F63000DFF890903446B0460D20B246FFF742FD09
:10F640000646C8B91D4DFBF7B1FB01232F782B707F
:10F65000FFB2FBF7C5FB4FB931461948FCF746FE30
:10F6600020B1FBF7A3FB2E70FBF7BAFB002CB2D046
:10F670002046FFF770FFAEE7EB1C0544C0F80080A2
:10F6800023F0030313350781C3F5147325F0030535
:10F69000C0F80C909BB24560BB4228BF3B464381FB
:10F6A0003CB1CAF80000FB1A00259FB2002FC3D15D
:10F6B00092E70446F7E700BF800001000C17012421
:10F6C00045F404088200010038B5038904468B42E2
:10F6D0001CD90D46CB1A6189A94218D3237B1A077E
:10F6E0000CD1A9420AD0637B9B0707D461682046EE
:10F6F000091B294489B2FFF7D5FB044620686581C0
:10F70000258108B1FFF727FF0023236038BD228938
:10F710006D1A1A44ADB222812468DCE70346002248
:10F7200090B2013203B970471B68F9E710B504467F
:10F7300040B1FBF73BFBA37B0133A373BDE8104053
:10F74000FBF74EBB10BD10B500B109B910BD104696
:10F750000B890489026823449BB20381002AF6D1F5
:10F760000160F3E710B5FFF7EEFF0846BDE8104073
:10F77000FFF7DCBF2DE9F0410C46054610B309B395
:10F7800002890B899A421DD30026B04662896F898F
:10F79000921B6168A7EB08076868314497424044B0
:10F7A00028BF17463A463E44FBF7D5F86389B8446C
:10F7B0009E426B8924BF24680026984508D12D6895
:10F7C00025B9A4B16FF00F00BDE8F0814FF000083B
:10F7D0002CB1628923899A4201D123684BB96A8985
:10F7E0002B899A4201D12B681BB9002CCED120461F
:10F7F000EAE76FF00500E7E72DE9F8438846914610
:10F80000064620B329B30027B9F1000F00D016B97E
:10F810003846BDE8F88375892BB1AB4203D35B1B37
:10F820009BB23668F0E7EC1A716808EB0700A4B2E7
:10F8300019444C4528BF4C4622462744FBF78BF819
:10F84000A9EB0402BFB200231FFA82F9E9E70746D9
:10F85000DEE70F46DCE72DE9F0410F46144605468A
:10F86000B8B1B1B10389934216D34FF0000814B96F
:10F870002046BDE8F0816E8907EB08016868A64262
:10F8800028BF26463246A41BFBF765F8B0442D6816
:10F89000EDE76FF00F00ECE74FF0FF30E9E738B528
:10F8A00015460A462989FFF789FE044610B1294604
:10F8B000FFF760FF204638BD124A4FF48040F0B594
:10F8C00013884FF6FF7601330F4D04219BB2B342EC
:10F8D00008BF4FF4404355F8044B246834B901394C
:10F8E00011F0FF01F7D11846138007E0E78A9F4225
:10F8F00005D1013880B20028E5D11380F0BDE4685D
:10F90000ECE700BFEC0C00240886070810B5037D67
:10F910000446042B03D0072B0BD0032B07D102F096
:10F9200077FA58B905232046237502F059FB0020C9
:10F9300010BD02F06DFA08B90923F4E7431CF7D1B2
:10F94000638B43F008036383F1E7000008B5FBF71E
:10F95000D1FA6FEA8040024B6FEA9040188008BDF0
:10F96000EC0C002401460120FFF7B8BBF8B5244D8C
:10F970000446002918BF0D46002838D0037D002B0F
:10F9800038D1417A11F004010CBF4FF0040E4FF052
:10F99000030E32B9FFF790FF024650B96FF0010035
:10F9A00012E0184E56F8040B006870B901339E45FA
:10F9B000F8D12B6803B12360134BE2821A681C60F4
:10F9C000E26002F007FD0020F8BDC78A97420CD123
:10F9D00011B1477A7F0708D4D0F800C0BCF1000FFE
:10F9E0000BD02F684FB1BC4507D0C068DDE76FF082
:10F9F0000F00E9E76FF00500E6E76FF00700E3E7C7
:10FA000008850708088607081817012419B191F816
:10FA100040100131C9B201727047000070B516463E
:10FA2000044600284DD0037D002B4ED1437A5B075E
:10FA300003D52B4B1B68002B30D10220FFF742FB74
:10FA40000546002848D0236901220361E38A027534
:10FA5000C382627D4275627A427200220272E27A49
:10FA6000C272A27A8272226802603BB11D4A136898
:10FA7000A3421ED1E36813600023E3602046FFF732
:10FA800071FF194BAB61164B1A681D60EA6002F0FA
:10FA9000A1FC002306B13370284670BDD98AE28AE2
:10FAA000914203D119682268914212D0DB68C2E703
:10FAB0001346002BE0D0DA68A242F9D1E268DA609E
:10FAC000DAE705466FF00F03E4E76FF00E03002559
:10FAD000E0E76FF00703FAE74FF0FF33DAE700BF24
:10FAE0002017012418170124EBFE0408C16A0246FE
:10FAF00030B5058D446A6B1A1819538EB3F5866FAD
:10FB000094BFC31AA0F58663002B01DB558530BD79
:10FB1000631A0020002BD6BF091B50855185F6E7DC
:10FB200010B50446E0B1038D194489B2B1F5066FF2
:10FB300013D88B4288BF4FF4066120462185FFF71A
:10FB4000D5FFB0F5067F0BD3638B204643F002034D
:10FB50006383BDE8104002F043BA4FF40661ECE75E
:10FB600010BD10B5044648B1406808B1FFF7F3FC7A
:10FB700021460320BDE81040FFF7B0BA10BD10B514
:10FB800000B910BD0468FFF7ECFF2046F8E738B570
:10FB900004460320FFF796FA054660B12346024665
:10FBA00004F1100153F8040B8B4242F8040BF9D115
:10FBB0006868FFF7BBFD284638BD00B1016170479A
:10FBC00008B1C0F88410704708B1C0F880107047C1
:10FBD00008B1C0F89010704718B1037D012B08BF21
:10FBE0008161704710B1C0F88C1042777047038B69
:10FBF000021DC18AFBF79AB949B18B8E3BB1282B04
:10FC00008ABF283B00239BB2984228BF1846704702
:10FC10002DE9F8430E46914698460446002800F028
:10FC20009580002900F09280037D002B40F09180A8
:10FC30000B6802834360007A90B1FFF7C7FB05466B
:10FC4000002800F0898023680BB943682360E78AA5
:10FC500057B9FFF731FEE08218BB6FF0010559E09C
:10FC6000201DFEF785F9EAE7637A5B0719D53C4B5F
:10FC7000196891B1CB8ABB4201D0C968F9E70B8BF7
:10FC80004B45FAD10A6823689A42F6D14A6833682C
:10FC90009A42F2D16FF007053CE0324B1968002917
:10FCA0003BD12046FFF7A3FF00232F4A29462065BA
:10FCB0000138E3626064C4E90932C4E916004FF414
:10FCC00006634FF40670221DA4F860306086FFF7CB
:10FCD00093FF0123608602212046A4F84830C4F82F
:10FCE000888002F05AF80546A0B9022323752FB187
:10FCF0001E4A1368A34221D1E3681360184B1A68A7
:10FD00001C60E26002F066FB194B012220461A706B
:10FD100002F066F92846BDE8F883CB8ABB420AD1D7
:10FD20000B8B4B4507D10A6823689A4203D14A6876
:10FD300033689A42AED0C968B1E71346002BDDD0D4
:10FD4000DA68A242F9D1E268DA60D7E76FF00F050E
:10FD5000E0E76FF00905DDE76FF00305DAE700BFC4
:10FD600014170124101701246008600818170124D3
:10FD70002417012410B50446406F18B1FFF7FFFEA9
:10FD80000023636710BD10B50446D8B1037D012B75
:10FD900018D90A2B16D0806F18B1FFF7DCFB0023AF
:10FDA000A367636F13B12046FFF7E4FF4FF6FF73BD
:10FDB000E06E2386FFF7E3FE206FFFF7E0FE0023EF
:10FDC000C4E91B3310BD03688B4210B50C4619D132
:10FDD000CB68036000232046E360FFF7D4FF237D58
:10FDE0000A2B0AD0012B08D0638BDA0705D543F024
:10FDF00002032046638302F0F3F800232375E382B5
:10FE000010BD1346002BE5D0DA68A242F9D1E268B2
:10FE1000DA60DFE72DE9FF470E460446002855D09B
:10FE2000037D0A2B09D101462A48FFF7CCFF204663
:10FE300004B0BDE8F047FFF795BDD0F85090D0F87A
:10FE400024A0D0F89070D0F81080C58A9BB93DB13D
:10FE5000214A1368834206D1C36813600025E56018
:10FE60002E460FE01346002BF8D0DA68A242F9D1F3
:10FE7000E268DA60F2E701461848FFF7A4FF184B82
:10FE800001221A70206F08B1FFF779FEE06E08B109
:10FE9000FFF775FE606F08B1FFF771FE56B1238B57
:10FEA000524649462046CDE90153231D009323467F
:10FEB00002F03FF82046FFF755FD3FB16FF00C010F
:10FEC00040463B4604B0BDE8F047184704B0BDE8E3
:10FED000F08700BF101701241817012414170124FC
:10FEE000241701240121FFF795BF084608B5FFF745
:10FEF000F9FF6FF00C0008BD38B50446084600B99C
:10FF000038BD02682368C5689A4201D1FFF7EAFF4D
:10FF10002846F4E738B50D46044680B1036873B14E
:10FF20000B4B1968FFF7E8FF0A4B20461968FFF7EB
:10FF3000E3FF25B12B6813B1074B1B6803B938BD2C
:10FF400019682268914204BF2A681A60DB68F5E7E5
:10FF50001417012418170124201701240C4B002228
:10FF600019680C4B30B404461D68104619B968B1C5
:10FF700030BCFFF74FBF0B7DA34205D10B6AEB1AD4
:10FF8000934224BF1A460846C968EFE730BC704761
:10FF9000141701241C170124F8B504460120FFF7AB
:10FFA00091F80346002836D1414E306800285BD1D5
:10FFB000404B0146404D1B682F68002B5FD108B1B4
:10FFC000FFF790FF0120FFF77DF8034618BB0920DB
:10FFD000FFF7C4FF0120FFF775F80346D8B90820E2
:10FFE000FFF7BCFF0120FFF76DF8034698B9200624
:10FFF0004DD45CB121460139326800202E68C9B267
:020000040805ED
:10000000002A46D113B11846FFF76CFF0120FFF715
:1000100059F8034630B3A4220021184620F0C8FA4C
:100020004FF4866225490346A0F86420244A4475AB
:100030008262FF22C2720622A0F84020C287214AB3
:1000400002631D4A126802621F4A127882771F4AB1
:1000500082641F4AC0F884201E4AC0E92512092282
:10006000C0F89C201846F8BD438BC5681F0704D50F
:1000700023F008034383FFF749FC284696E71A6AF2
:10008000BA1A8A4224BF18461146DB6895E77F21D9
:10009000B1E7577D8F4204D307D1156A751B85429E
:1000A00003D3106A39461346301AD268A8E700BF56
:1000B00014170124101701241C17012400DD6D0002
:1000C00060086008FFFF1802A250002401003004FD
:1000D00015020508F82401004020FFF75DBF00006D
:1000E00030B5044685B0037D002935D0042B01D0FE
:1000F000072B31D1A26F1AB9228DB2F5066F2BD022
:10010000238B2046626A0293E38A216D0193231DAB
:100110000093234601F00DFF2046FFF734FE304ADE
:100120001368A34210D1E368136000230122E36047
:100130002C4B1A702C4B1B68A3421DD101F088FB7D
:10014000002005B030BD1346002BEED0DA68A24285
:10015000F9D1E268DA60E8E7012B1AD0022B30D03F
:10016000002B36D1E38A3BB1204A1368A34208D161
:10017000E36813600023E3602046FFF7F3FBDFE74B
:100180001346002BF6D0DA68A242F9D1E268DA60B1
:10019000F0E71749002051F8232012685AB90133BB
:1001A000042BF8D121461348FFF70DFE214602200B
:1001B000FEF794FFC4E7D56FAC4208BFD067D268A2
:1001C000ECE721460648FFF7FEFD064B01221A70B8
:1001D000D2E7204605B0BDE83040FFF797BB00BF2F
:1001E00014170124241701242817012418170124A7
:1001F000088607082017012448B1037D0121012B3F
:100200001EBF438B43F010034383FFF769BF6FF0BA
:100210000F00704710B50846144669B13AB111890C
:10022000FFF77EFC2046FFF796F9002010BD33B99A
:10023000BDE81040FFF7E0BF6FF00F00F6E7104693
:10024000F4E7F8B5044678B3866F0023D0F88450FD
:10025000777B8367DDB1014632460069A8470546D2
:10026000E0B9BB0611D5238DD4F88460B3F5066FD1
:100270001CBF0133238546B10023214620691A465D
:10028000B0470D3001D16FF00C052846F8BD01468E
:100290002B4632462846FFF7BDFFE0E70D35F2D08A
:1002A0006FF00405A667F0E76FF00F05EDE70000BB
:1002B0002DE9F8431B4D1C4F2B781C4E01332B703E
:1002C0003C684FF000080CB9BDE8F8832B78A27F9A
:1002D0009A4224D0A377638BD90709D543F0020350
:1002E0002046638301F07CFE638B23F0030363836A
:1002F000638B1A0705D523F0080320466383FFF7B5
:1003000005FBA36FD4F80C903BB1204686F8008023
:10031000FFF797FF3378002BD2D14C46D3E7D4F8C0
:100320000C90FAE7A250002414170124241701248A
:1003300038B51446054618B3037D012B18D089B192
:10034000438B43F01003438322B10121BDE83840C1
:10035000FFF7C6BE806F08B9002038BDFFF7FBF875
:10036000AC67F9E7002AF7D0042B04D8022B04D895
:100370006FF00A00F1E7072BFAD100212846E5E7E4
:100380006FF00F00E9E700002DE9F04FB64F4FF096
:10039000000989B03B68CB4601333B60B34B1A7808
:1003A000059301321A70B24B4FF00008DFF8D0A26B
:1003B0001C6806933CB9AF4E3568002D40F048816B
:1003C00009B0BDE8F08F059BA27F1B789A4203D14C
:1003D000E668A0463446EDE7A37794F84230052B53
:1003E00000F2F78094F8A150002D00F0A58094F859
:1003F000A230052B00F2ED809F4B1D4494F8A030F5
:1004000015F8012C93420FD3B4F86010002900F0C6
:100410008480204601F034FC002840F08380204690
:1004200001F0DEFD30B17DE00133DBB2934284F8B0
:10043000A030E9D20025217D062909D1638BDB0696
:1004400006D53B68226A9B1A282B84BF0135EDB282
:10045000667A16F0080617D0042902D0072940F062
:10046000CB80236A4FF4FA703968D4F89C20C91AFB
:10047000D4E9256302FB0362B2FBF0F2914240F241
:10048000AA8001350126EDB2636F63B13B68226A31
:10049000B4F940109B1A01EB4101B3EB410F02D3B9
:1004A0002046FFF767FC237D032B40F0A7803B68C5
:1004B000226A9B1A282B02D8002D00F0AA80204621
:1004C000D4F89050FFF75FFCE368B8F1000F00F03C
:1004D0009D80C8F80C305EB1238B20460293E38ADE
:1004E0000193231D00932346626A216D01F021FDD3
:1004F00023692046E6680793FFF734FA8AF80090EC
:100500004DB1079B6FF00C011846A8479AF80030D0
:10051000002B7FF448AF44465BE7204601F0C6FE5F
:10052000002887D194F8A13084F8A090062B81D8B8
:10053000013384F8A1307DE7238E47F6FE729342A3
:100540009CBF01332386B4F94030B4F930209A427D
:10055000FFF670AF204601F078FC38B1236F002B16
:100560007FF468AFE36E002B3FF464AF237D022B72
:1005700014D0B4F93C20B4F93E30404903EBE20317
:1005800094F842200C2A28BF0C228A5C934047F63C
:10059000FF729342A8BF1346A4F84030B4F860201D
:1005A000B4F84830618E9A42A4F83090A4F848100C
:1005B00028BF1A464B00A4F868B09BB25008B3EBB2
:1005C000520F98BF03462046A4F84A3001F046FE79
:1005D00031E701252FE794F8A32003FB0263B3FB67
:1005E000F0F3994208D9204601F04CFE20B994F866
:1005F000A330013384F8A330002645E7092B7FF4AC
:100600005BAF3B68226A9B1AF02B54E7069A136093
:1006100061E7237F627F0133E668DBB29A4223778A
:100620003FF6D7AED4F88C3025778AF800501BB946
:10063000204601F0D5FCCCE62146206998479AF87F
:100640000030002B7FF4AFAE00287FF4C2AEEFE79E
:100650003B682A6A9B1AF02B14D92846FFF793FBB4
:10066000EB6894B9336011E01C170124A2500024F8
:10067000141701241017012418860708F8850708A5
:10068000241701242C46ED6897E6E360D5F80C802A
:100690002846FFF767F945468FE600BF08B5FFF724
:1006A00007FE064A13780133DBB21370DB0703D56C
:1006B000BDE80840FFF768BE08BD00BFA150002498
:1006C000094A1388591C1180084A12681AB108494E
:1006D00009888B4204D2074A12681344187D704778
:1006E0005B1ADBB2D05C7047CC500024D850002499
:1006F000D4500024D0500024C3682DE9F0419B89D8
:1007000005465BBADA070C4618D4DFF8608001278B
:100710007FBAE668D8F800002B8971682289034403
:100720000A449A1A002A10DA5B1A002B0ADD091A09
:10073000686889B22981FEF7C7FF03E000240846F4
:10074000FFF71DFA2C60BDE8F081B38920465BBA43
:10075000DB07266848BFEA68344642BF93893B43BB
:100760009381FFF7FEF9002ED3D1EBE7C8500024A8
:10077000F8B51A4B07461E8866B1194D00232B8029
:100780002B88B34206D2FFF79BFF0128F8D002283E
:1007900001D0C8B9F8BDFFF793FF0428FAD12B8820
:1007A0000133B342F6DAFFF78BFF0402FFF788FF4D
:1007B000A4B244EA00039BB25A1EB2F5067F28BFDA
:1007C0004FF406733B80DBE7FFF77AFF0128E1D99E
:1007D0002B88023B18442880D2E700BFDC5000245D
:1007E000CC5000240D4B10B51B78044613F01003B9
:1007F00012D0438BDB0606D4D0F890301BB16FF0DB
:100800000E010069984721460548FFF7DCFA2046AB
:10081000FFF7A8F8012010BD1846FCE7C4500024DB
:10082000141701242DE9F04105460C46124F134ED2
:100830007CB1E36838685A689B8911BA22895BBA2F
:10084000121A13F003030A4418BF01231344002BA8
:1008500002DD2046BDE8F081D4E90080FEF75EFFAE
:100860002B883288181A288020462389444613444E
:100870003380FFF776F9DBE7A4500024BC50002456
:10088000A04B2DE9F0471B7804469F4E13F0100F44
:100890009E4F00F088803368B0F860109C4DD0E91E
:1008A000150C2A68A946A0EB030EBEF1000F0CDB65
:1008B000984203D1ACEB0200002806DB944513D12B
:1008C00094480068C08988420ED99248B4F8628082
:1008D0000068C0891FFA80FEA4F86000F045C4E9F2
:1008E000153238BFA4F86200606C131A002B00F3B5
:1008F00017813B88002B40F00081B4F860306144E0
:10090000A56D2B448B4240F0F880B4F93030002BB9
:10091000C0F2F380904240F0F08094F84330FF2B17
:100920001CBF013384F8433094F84330032B0FD9B4
:10093000B4F848204FF6FF71638E13449BB29A427D
:1009400088BF0B46A4F84830204601F0CEFA00E0FC
:10095000FAD0606B38B3A36BD9F800209B1A002B38
:1009600021DA6D4B80B2B4F93CC01A88CCF3CF05C4
:10097000111A491B0BB21CFA81F1002B09B2B8BF46
:10098000801AB4F93E20A187B8BF4019A2EBA20299
:10099000B8BF03B213449BB2E38703EBE103A4F8AF
:1009A0004030002363633D883368626A002D00F0A5
:1009B0009582217D062900F29182D11A012900F148
:1009C0003881C3F10100401B1044002800F331813D
:1009D000524D89B24FF0000C2B8968685B1A2B814D
:1009E00003895B1A9BB242898A42C0F01B81FEF7E1
:1009F00094FD636AEA68336053603368626A991AE7
:100A00000029C0F2BA8103F1010C218DACEB020088
:100A1000401A002800F3B181934240F0A8813F4D75
:100A2000D5F80CC0B5F808E0BCF80C0043BA13F0D8
:100A3000030218BF0122724492B291423A8020D23E
:100A4000DA0707D520F47C5003F03E035BBA03437A
:100A5000ACF80C302981BCF80C305BBA9807686898
:100A600044BF01F1FF3129812989FEF72DFEEB6892
:100A70002A899B895BBA13F0030318BF012313442F
:100A80003B80D4F87480B8F1000F00F0E180EB688F
:100A90009B895BBADA0700F1D8804FF0010999FA17
:100AA00099F9D8F80CC030683A88DCF80430B8F806
:100AB000081002441944511A002980F2E980D21A20
:100AC000002A40F305811B1AEA6868689BB22B81F3
:100AD000928952BA920744BF03F1FF332B812989CF
:100AE000FEF7F2FDEB682A899B895BBA13F00303DA
:100AF00018BF012313443B80EAE0002384F843300D
:100B000027E700BFA8500024C8500024DE5000246E
:100B1000A4500024D05000241C170124AC50002401
:100B2000216D511A002979DC618B480709D521F024
:100B300004016183B4F84A10A4F848100021A4F815
:100B40006810B4F93C00E18F626401EBE001227DA2
:100B5000A4F84010032A4FF00001A4F8421026D94F
:100B6000B4F848109BB2B4F84A208A4215D9628B77
:100B700012F4006F628E14BF0120022012FB00F2FB
:100B800092B29A4294BF8B18CB189BB2994201D96A
:100B90004FF6FF73A4F8483009E0B4F86820134416
:100BA0009BB29A4230D8994230D9A4F8683004F107
:100BB0006608216F4046FFF735FEE16E206740462C
:100BC000FFF730FE226F9949B2FA82F3E066098896
:100BD0005B095B42238600232377B4F864300B441F
:100BE000A4F86430638B19057FF5B3AEA2B938B1B0
:100BF000C268526811BAE26C521A002A3FF7A9AED5
:100C000023F400636383A4E64FF6FF735B1AA4F832
:100C10006830638E0B44B8E7D268EAE7204601F0FB
:100C2000C1F996E6891A0381A0F80AC089B2006862
:100C3000D9E69B1A002BBEBF638B43F0020363838C
:100C4000DBE603686367FEF78CFF606F0028F8D16E
:100C500039882046238D32685B1A0A4423856262F4
:100C6000FEF744FF6B681A891AB1714A13600023BA
:100C70006B60EB689B895BBAD80704D56D4A137823
:100C800043F0200313706A4D4FF00008694F54E0A1
:100C9000BCF80C305BBADB0710D5E9688A8953BA17
:100CA00098070BD442EA090293B28A815BBA13F027
:100CB00003032A8918BF012313443B80D8F800A0FE
:100CC0004046FEF74EFFD046BAF1000F7FF4E9AE82
:100CD000C4F87480BCE7B9F8080032608B8902441C
:100CE0005BBA13F0030318BF01231A4403442046E0
:100CF0006262228DD31A2385FEF7F8FED9F804101C
:100D00000B892BB1286858B3FEF71DFDC9F8048084
:100D1000D9F80C309B895BBAD90708D53B7843F0EA
:100D200020033B70237D042B04BF07232375D9F8D0
:100D3000003048466367FEF714FFD4F87490B9F1A9
:100D4000000F05D0D9F80C10636A4A689A42C2D0E5
:100D5000638BDA0706D523F0010343F0020303E0B7
:100D60002960D3E743F001036383BDE8F087656F33
:100D700045B93148FEF70BFF60672046BDE8F047F4
:100D800001F010B94FF0000803F1FF3EE868426837
:100D9000934215D128482B8902899A42EDD9FEF752
:100DA000F6FE0028E9D0B8F1000F07D0C8F800001F
:100DB0002946FFF7A1FCE0E70D46E7E76067F7E7A4
:100DC000B8F1000F09D1991A002937DA1A48FEF74D
:100DD000DEFE0028D1D06067EAE7D8F80C10496839
:100DE000AEEB0101002929DBACEB0201002925DC77
:100DF0001148FEF7CCFE07460028BED0D8F80C30CC
:100E000031685A68B8F8083013445B1A002B07DDC4
:100E1000891AD8F8040089B2A8F80810FEF754FC23
:100E200029463846C8F80070C3E700BFBC5000240C
:100E3000C0500024C4500024AC5000242968A846A7
:100E40000029B9D19B1A002B97DD83895BBADB0798
:100E500093D42848FEF79BFE286000288DD0EB68CD
:100E600031685A682B8913445B1A002B05DD891AF7
:100E7000686889B22981FEF727FC31683A88666A7A
:100E80000A44238D921BD21A002A7FF776AF286876
:100E9000D0F80CE0BEF80C2092FA92FC1CF0010F86
:100EA00009D022F47C520CF03E0C9CFA9CFC42EAE5
:100EB0000C02AEF80C20591A314489B20181406805
:100EC000FEF702FC2A68D36812899B895BBA13F08B
:100ED000030318BF012313443B804EE7991A0029EE
:100EE00006DB01339B1A228D9B1A002B7FF73DAF47
:100EF000638B32E7AC5000242DE9F04F43688DB08E
:100F0000AB4F05463B604389132B40F2A380A94EAB
:100F100031687069FDF72FFA002840F09B807369F3
:100F200003F0F003E02B00F0958006F11403062196
:100F30002846009306F110032A89FDF7D3FE002806
:100F400040F088803B68998949BA890A01F0FC0120
:100F500013297FD92B898AB28B427BD3DFF884A2F5
:100F6000A2F11403DFF88082CAF800009BB26889FE
:100F7000DFF878929042A8F8003043D32846A9F8C9
:100F80000030FEF7CAFA3B688B4C1A8852BA1FFA37
:100F900082F91A805A8852BA1FFA82FB5A805A681C
:100FA000864812BADFF848E2226099685A6009BAA6
:100FB000016007EE901AD88940BAD8819889996063
:100FC000089040BA00F03F0810F0030F5FFA80FC71
:100FD00005948EF80080B5F808E034D17848A0F880
:100FE00000E078484FF0000804680B900A94746899
:100FF000069434690994746907940A9C84BB724B03
:101000001868FAE014212846FEF787FA6C8928460A
:10101000A9F800402146B8F80090FEF77EFA28684B
:10102000A9EB040843891FFA88F8434512D34368A3
:101030004146CAF80030FEF770FA2B891C44A4EB35
:1010400009042C819FE70EF101005D4C80B28645BA
:101050002080C6D928460DB0BDE8F04FFEF77BBA18
:1010600094F808A0BAF1000F06D0069890F8400056
:101070000130C0B2824556D1208B484553D1E08A19
:10108000584550D16068099988424CD12068079929
:10109000884248D1B8F1000F06D0E268C8F80C20A9
:1010A0000A9AE260474A1460484A002148481CF006
:1010B000080F484E9046D3608146474B11609A46D0
:1010C000A2F808E0556019603170018003D06B7B95
:1010D00043F001036B73A36FDFF818B1002B00F02E
:1010E0004A812046FFF7ADF80D3008D0A36F002BE2
:1010F00000F04181324B1B88002B00F03C81638D56
:1011000013B9204600F04EFF0024D8F80400CBF8B5
:101110000040CAF8004018B1FEF71DFAC8F80440B4
:101120000DB0BDE8F08FA046E46867E7047A34B1FB
:10113000069B93F840300133DBB29C425CD1038BB9
:101140004B4559D1C38A5B4556D1436809999942A9
:1011500052D10368079999424ED11CF0040F7FF4D5
:1011600079AF174B1CF0020F1C8811D0436AD31AB9
:1011700014D4068D9B1B002B10DC184B224417EE59
:10118000901A00930433CDE901B900F0D2FE61E773
:101190001CF0010F1EBF124B1B680362002C3FF4B2
:1011A00059AF438B43F00203438300F019FF51E72B
:1011B000D050002488FD0024C8500024A4500024EE
:1011C000DE5000241417012410170124AC50002411
:1011D000BC500024C4500024C050002498FD0024BA
:1011E0001C170124D8500024DC500024D4500024C3
:1011F000A850002428170124C068002896D18F4BDE
:10120000044680461B68099323B9002C00F016831E
:1012100040461FE093F808A0BAF1000F08D00699E5
:1012200091F840E00EF1010E5FFA8EFEF2450DD10D
:10123000B3F816E0DE4509D1D3F800E0079971450F
:1012400007D0BEF1000F04BF1C4680461846DB687D
:10125000DAE71C4628B1E368C360099BE360774B7B
:101260001C601CF0040F7FF4F5AE1CF0100F0BD0C7
:10127000734B17EE901A1888724B02442046009365
:101280000433CDE901B980E71CF0020F3FF4E2AE70
:10129000607DFEF781FE804648B9A369002B3FF4CC
:1012A000D9AE01464FF0FF3220699847D2E6736904
:1012B0003A68036033694360E38AC38213785278E3
:1012C00043EA0223038303230375059B1B68013351
:1012D0004362C362FEF78BFC059BC8F858001B688D
:1012E000C8F85000013BC8F84400C8F85C00C8F8D2
:1012F00054302369C8F87C40C8F81030637A03F092
:101300000C0388F80930237A88F808300B9B1B6897
:10131000C8F80C300B9BC3F8008001F05BF8012289
:10132000494B08F132001A70FFF722FA3B6898F82F
:101330000800DB89A8F86030A8F86230FEF746F8AC
:1013400008F1040220B910460592FCF711FE059A37
:101350000146B8F83200FEF74FFC1221A8F832001F
:10136000404600F01AFD20B100214046FEF752FD34
:1013700070E6404619E7354DCBF800402B7858070A
:101380001FD5237D022B0DD1314B226D1B689A4254
:1013900022D1337843F008033370638B23F00103C9
:1013A000638319E02B4B626A1B689A42F1D09B1A47
:1013B00012D4228D9B1A002B0EDC638B43F00203A8
:1013C000EEE713F00202618B19D0207D023801286C
:1013D00015D941F0020161833378190740F1D381B7
:1013E000D4F890301BB16FF00D0120699847214669
:1013F0001948FEF7E8FC2046FEF7B4FA84E6C90671
:1014000004F132005EBF1549096821620021A4F889
:10141000A210CDE90632FFF7ABF9217D0239DDE9F3
:1014200006320729D8D8DFE811F01B009D00030120
:101430000701500103017901980100BF2017012421
:10144000DE50002498FD002424170124A850002415
:10145000A4500024C8500024141701241C17012490
:1014600003F01202122A5DD1A44A1168626C0132A3
:101470008A4257D1059B62641B68A14A591C013BF3
:1014800012686162E162D28963650423A4F8602076
:10149000A4F86220207A2375FDF798FF221D20B959
:1014A00010460592FCF764FD059A0146608EFEF732
:1014B000A3FB41F21C134200608681009A4215464C
:1014C00038BF1D46B5EB800F20D98BB2A4F8483049
:1014D000B4F86630206F013BA4F86630D0B9E06EF6
:1014E0000368E366FEF73DFB236FB3B94FF6FF7366
:1014F0002386D4F88830002B3FF45FAF00222146CA
:10150000206998470D307FF458AFFDE59A4288BFB7
:1015100093B2DBE703682367E4E70023238684F8BC
:101520004230E6E7D8067FF557AF3B68754A188822
:101530001188059A1268029020465B880A446F4918
:101540000193714B00930433096800F0F2FC94F8A6
:101550004230052B3FF640AF00232046238600F0A3
:1015600086FE39E7D90655D5644B1968636CDB43B1
:10157000CB423ED4236DCB1A002B3ADC04232375D7
:10158000E36F1BB92046FEF7ADFCBDE59B69002B60
:10159000F8D0002221462069984718B10D303FF459
:1015A000B3ADEFE72046FFF76BF9B9F8003013B1A0
:1015B000013BA9F80030618E41F21C134A008800FB
:1015C0009A42154638BF1D46B5EB810F0DD983B23F
:1015D000A4F8483033789A067FF5FEAE638B43F06B
:1015E0000203638307232375F6E69A4288BF93B20A
:1015F000EEE73B68434A1D881088059A12680295F9
:101600005B880244204601933F4B0093043300F073
:1016100090FCE1E6002A3FF4DFAE636A3B4A013BFF
:10162000126893427FF4D8AE204600F036FCD3E631
:101630002046FFF725F9CDE72046FFF721F933785B
:1016400013F0200F2B7831D013F0100F638B28D0BC
:101650002A4A216D1268914223D1E26E0ABB43F0FF
:10166000020320466383FEF78EFB294A13689C42DF
:1016700009D1E368136008E0DA68944202D1E268B5
:10168000DA6002E01346002BF6D1224B01221A70D9
:101690000A232375204B1A681C60E26000F09AFE52
:1016A0009AE643F00203638308239CE7DB067FF599
:1016B00093AE124B226D1B689A427FF48DAEE36E9F
:1016C000002B7FF489AE06238DE72046FFF7D8F87C
:1016D00033789F067FF580AE638B204643F002038C
:1016E0006383FEF750FB0A4A13689C42C1D0002B6B
:1016F000CBD0DA689442C2D01346F8E7A450002455
:10170000D0500024DE50002498FD0024C85000244E
:101710001417012424170124101701242046FFF771
:10172000AFF82B78DD067FF557AE474B226D1B686F
:101730009A427FF451AEE36E002B7FF44DAE20460B
:10174000FEF721FB414A13689C4292D0002B9CD0AB
:10175000DA68944293D01346F8E72046FFF790F8F2
:101760002B78D8067FF538AE374B226D1B689A422E
:101770007FF432AEE36E002B7FF42EAE337843F06D
:101780001003337028E6B9F800202AB1D4F880306D
:101790009BB90023A9F800302046FFF723F8002862
:1017A0007FF4B2ACDAF80020DAB1638B13F01003E7
:1017B00009D01046FDF7CFFEE4E6214620699847A0
:1017C0000D30E6D1A0E4D4F8845005B32146206959
:1017D000A84710F10D0F3FF497AC10B1DAF80030C4
:1017E000A36733789A0605D5A36FABB15A7B42F055
:1017F00020025A7300232046CBF80030FEF7F2FF98
:1018000000287FF481AC204600F0EAFB7CE42B4604
:101810002146FEF7FFFCDCE7238DD4F88450B3F5B6
:10182000066F1CBF01332385002DE3D00023214622
:1018300020691A46A8470D30DCD165E4089B5BBAE5
:101840005B073FF507AC13E5A450002414170124EF
:10185000024A137843F0100313707047C4500024F9
:101860002DE9F0479DF820A0814603200F464FEA5E
:101870008A0516469846FDF725FC05F00405044642
:1018800028B93846FDF767FE2046BDE8F08780F8A6
:101890000AA04FF0000A3B8914215B1BC0E900A796
:1018A00003813846FDF736FE20B120465446FEF748
:1018B00058F9E9E76368AD0898FA88F8596805357A
:1018C000B9F81630E16046EA05355BBA6DBA0B80AF
:1018D000B9F81830C1F804805BBA8D814B808874E8
:1018E000C874D1E714312DE9F84389B2044617468C
:1018F000466AB0F816904FF42072B0F81880458D03
:101900002220FDF75BFED0B1436836BA45F21002E3
:1019100052BA9A8100225F601A745A749A74DA7407
:101920009E60628D99FA99F998FA98F8A3F8009058
:10193000A3F802806DBADD81636A1344E362BDE8F7
:10194000F8832DE9F0430D4685B090461F460446C6
:1019500020B3007A10B3FDF739FD064620B3D5F861
:10196000049043462A89062128460097FDF7BAF9D4
:10197000A9F81000B4B1E37AA47A062241462846B9
:101980000296CDE900423A46FCF7D3FC04462846CD
:10199000FDF7E1FD204605B0BDE8F0833846FCF7D1
:1019A000E7FADAE7FF23E8E76FF00304EFE72DE952
:1019B000F04F2DED028B8BB09146054604910693B6
:1019C000002800F05381B0F86230428E5B089342E9
:1019D00028BF1346002B08BF13460593049B002B1A
:1019E00000F04481037D072B03D0023B022B00F261
:1019F0004481B9F1000F0ED0B5F864304B4506D2E2
:101A00006B8B43F080036B834FF0FF3030E1B5F810
:101A10006630072BF4D8B5F86630D5F86CA0039380
:101A2000BAF1000F00F0DA805746DAF800A0BAF1F8
:101A3000000FF9D1B9F1000F00F01281059BB7F842
:101A40000880A3EB0806BB7A9B0003F00403F61A98
:101A5000B6B2002E00F0C780B8F1000F00F0C680CB
:101A60004E45069BA8BF4E46DB07B046B6B221D511
:101A70004FF4207231465046FDF7A0FD0446002881
:101A800000F0F080424604994068F8F764FF204671
:101A9000FDF744FE039BBA464FF0000803449BB297
:101AA0000393069B4FF0000B03F00103CDF81CB02D
:101AB000089383E07C6822462468002CFBD1137BCA
:101AC00013F0C00F06D151895368049A0B449A420F
:101AD00000F08E80012231460020FDF76FFD0446A4
:101AE000002800F0BF80049B4360D1E7A9EB060308
:101AF000059A9BB2934228BF13469BB208EE103A58
:101B0000089BD3B14FF4207218EE101A3620FDF75F
:101B100055FD824640B3049B18EE102A406899197F
:101B2000F8F719FF5046FDF7F9FD039B03449BB2FC
:101B3000082B03932CD9504614E0012218EE101AFA
:101B40003620FDF73BFD78B1049A0990324408999C
:101B500042604FF420723620FDF730FD099B82462B
:101B600090B91846FDF7F7FC6B8B43F080036B834D
:101B700014B12046FDF7EFFCBBF1000F3FF444AF7A
:101B80005846FDF7FCFF3FE71946FDF7DCFDC9E7C6
:101B9000EB6D00225146284633440092FFF760FE69
:101BA00082460028E0D0BBF1000F15D0079B1860DB
:101BB00018EE103ACDF81CA01E44B6B24E4595D38F
:101BC000CCB121467868FDF7BEFD3B8922891344DC
:101BD0003B81C7F800B026E08346E9E75746544604
:101BE000D04656465DE7D04654465AE75646FBE790
:101BF000B046BA4655E7B8F1000F10D07B681A8995
